:020000040800F2
:100000000000022049040108CF020008CF020008C6
:10001000CF020008CF020008CF0200080000000055
:10002000000000000000000000000000CD020008F9
:10003000CD02000800000000CD020008CD0200083B
:10004000CF020008CF020008CF020008CF0200084C
:10005000CF020008CF020008CF020008CF0200083C
:10006000CF020008CF020008CF020008F1D4000838
:1000700001D5000811D50008CF020008CF02000802
:10008000CF020008CF020008CF020008CF0200080C
:10009000CF020008CF020008CF020008CF020008FC
:1000A000CF020008CF020008CF020008CF020008EC
:1000B000CF02000821D50008CF020008CF020008B7
:1000C000CF020008CF020008CF020008CF020008CC
:1000D000CF020008CF020008CF02000831D5000887
:1000E000CF020008CF02000800000000CF02000885
:1000F000CF020008CF02000841D50008CF02000857
:10010000CF02000851D50008CF020008CF02000836
:10011000CF020008CF020008CF02000861D5000816
:10012000CF020008CF020008CF020008CF0200086B
:10013000CF020008CF020008CF020008CF0200085B
:1001400000000000000000000000000000000000AF
:10015000CF020008CF020008CF020008CF0200083B
:10016000CF020008CF020008CF020008CF0200082B
:10017000CF020008CF020008CF02000800000000F4
:10018000CF020008CF020008CF020008CF0200080B
:1001900071D50008CF020008CF020008CF02000886
:1001A000CF020008CF020008CF02000800000000C4
:1001B000CF020008CF020008CF020008CF020008DB
:1001C000CF020008CF02000800000000000000007D
:1001D0000000000000000000CF0200080000000046
:1001E000000000000000000000000000000000000F
:1001F0000000000000000000CF020008CF0200084D
:10020000CF020008CF02000800000000CF02000863
:10021000CF020008CF020008CF020008CF0200087A
:10022000CF02000800000000CF020008000000001C
:10023000CF020008CF02000800000000CF02000833
:10024000CF020008CF020008CF020008CF0200084A
:10025000CF020008CF020008CF020008CF0200083A
:10026000CF020008CF020008CF020008CF0200082A
:10027000CF020008CF020008CF02000800000000F3
:10028000CF020008CF020008CF020008CF0200080A
:1002900000000000CF020008CF02000800000000AC
:1002A00000000000CF020008CF020008CF020008C3
:1002B000CF020008CF020008CF020008CF020008DA
:0C02C000CF020008CF020008CF020008A7
:0202CC00704779
:0202CE00FEE749
:1002D0002DE9F84F2DED068B84B0B5EE401BF1EE05
:1002E00010FA00F09180B4EE411BF1EE10FA80F1AB
:1002F0008B80B0EE408B50EC101B420042EAD17173
:1003000011F5001F9FED429B77D2B0EEC89BB0EE77
:10031000C1ABB4EE4A9BF1EE10FA02D5B0EE489BA9
:100320006BE0B4EE4A9BF1EE10FA05D100F000400C
:10033000002140EC191B60E002A8B0EE4A0B10F05F
:100340009DF8B4EE4A9BF1EE10FA4FDB59EC1A0B14
:100350000190029F09F0004A4AF0E04040F07F6BB4
:10036000C9F30A556FF31E5940F2FF78B0EE490BFE
:1003700003A810F083F80398C01B691EB0EE4A0B67
:1003800012D34545B0EE4A0B0ED0431940F2FE722F
:10039000002693425A4605DC012B5246A4BF49EA87
:1003A0000352019E42EC106BB4EE490BF1EE10FAD1
:1003B00015DDB0EE4A0B95B14545B0EE4A0B0ED0B7
:1003C000014440F2FE7000228142584605DC0129BA
:1003D0005046A4BF49EA0150019A40EC102B39EE77
:1003E000409BB4EE4A9BF1EE10FABFDAB5EE408BBB
:1003F000F1EE10FA48BFB1EE499BB0EE490B04B0E4
:10040000BDEC068BBDE8F88F9FED019BF5E700BFC3
:08041000000000000000F87F6D
:1004180050EC10CBC0F30A52531E40F2FE718B42CF
:1004280051D240F2FE318A4208D8BFEE000B9FED50
:100438002A1BB0F1FF3F31FE000B704740F23241FA
:100448008A4288BF7047F0B5A2F2FF33B3F12001AA
:100458004FF48017C3F1200407FA04F540F20006B0
:10046800CFF6F07606FA04F25CBF27FA01F546FAF1
:1004780001F202EA0C0E27FA03F24EBF1E410022D7
:100488004FF0FF36064015EB0E0572412CFA04F4C6
:1004980000FA03F73C43002958BF0CFA01F46FF344
:1004A8001F540CFA03F148BF0C43B4FA84F149090C
:1004B8000028A8BF41F0010100291CBF324675463B
:1004C80042EC105BF0BD002A04BF00F000409446E7
:1004D80040EC10CB704700BF000000000000000097
:1004E8000000000000002440000000000000594007
:1004F800000000000088C3400000000084D7974136
:100508000080E03779C34143176E05B5B5B8934607
:10051800F5F93FE9034F384D321D30F94877825AD3
:080528003CBF737FDD4F157528
:1005300001000000000000000A00000000000000B0
:100540006400000000000000E8030000000000005C
:100550001027000000000000A0860100000000003D
:1005600040420F000000000080969800000000004C
:1005700000E1F5050000000000CA9A3B0000000001
:1005800000E40B540200000000E876481700000069
:100590000010A5D4E800000000A0724E1809000069
:1005A00000407A10F35A00000080C6A47E8D03003C
:1005B0000000C16FF286230000008A5D7845630168
:1005C000000064A7B3B6E00D0000E8890423C78AE1
:1005D0002DE9F84F2DED0A8B8EB0069289468046A4
:1005E0000020C8F800000DF11D0003909FEDC6AB80
:1005F000B2EE048BB7EE00BB9FEDC5CB19F8011B23
:10060000252906D0002900F0DA8540460FF06EFF5C
:10061000F4E70026494619F8012BA2F12003102B1C
:100620000DD88020DFE803F0091B1B191B1B1B15CD
:100630001B1B30181B101B1B120040200DE05E2AF4
:100640000DD14FF4805008E0102006E04FF4007008
:1006500003E04FF4004000E020200643DAE701F118
:100660000109A2F1300009284FF000001BD819F849
:10067000011B00EB800002EB40003038A1F130029A
:100680000A2A0A46F3D30EE0069850F8042B069087
:10069000002A104648BF5042102303EAD262164394
:1006A0004A7801F102092E2A0DD1494611F8012B91
:1006B0002A2A0BD1069999F8012051F804AB06912A
:1006C00009F1020916E04FF0000A1CE0A2F1300324
:1006D000092B4FF0000A13D811F8013B0AEB8A09E5
:1006E00002EB4902A2F1300AA3F130020A2A1A46AB
:1006F000F2D38946BAF1000F58BF46F4807602E083
:1007000046F4807689466B2A0ADC4C2A03D0682A94
:1007100018D06A2A28D119F8012B46F0020623E0E6
:100720006C2A05D07A2A14BF742A19F8012B1BE011
:10073000494611F8012B6C2A10D199F8012009F1D2
:100740000209EAE7494611F8012B682A09D199F80C
:10075000012009F1020946F0080605E046F001060D
:1007600001E046F00406894620EAE077462A1FDDCC
:10077000A2F1630015282FD8DFE810F06000170001
:1007800045002300A40116001700160016001600ED
:100790001600700084004E00160016007F00160040
:1007A000480016001600360028E746F4804631E07F
:1007B000442A09DD452A24D0462A7FF41FAF46F497
:1007C000005646F4006B7FE1252A40F065824046E2
:1007D00025210FF08BFE11E7472A00F07181582A7E
:1007E0007FF40CAF46F40056F0054FEA066048BFB0
:1007F00026F4007643F25801782A08BF43F27801C4
:1008000047E046F4005646F4806B5DE1F00548BFD2
:1008100026F4007600213EE03006232101EAE07054
:10082000CDE9047046F48076069A002152F8040B54
:1008300006924FF0080A0DF11E04DEE00698A7F1BB
:10084000010A10F8044B06904046314652460CF01F
:100850006EFC404621460FF049FEAEE1069951F884
:10086000040B06913107D8F8001000F11982B20785
:1008700052BF0160002206C0C0E6069850F8044B43
:10088000069079E1F0054FEA066048BF26F400764D
:10089000302101EAE07170044FEA8670069DCDE9CF
:1008A000047104D4002808D42B1D00210BE000287B
:1008B00015D455F8040BC11717E0E81D20F0070503
:1008C00005F1080369680DF11E0428687507069391
:1008D00015D416F008051CBFC0B2002132E0E81D97
:1008E00020F00705696855F8080B0DF11E04730721
:1008F00012D4330744BF40F3C01140B20FE080B2BE
:1009000000211FE000BF00BFA0C8EB85F3CCE17F52
:10091000000000000000594040F3C03100B200293F
:10092000069507DBB3060BD47306059D48BF20254B
:10093000059507E00023404263EB01012D2300E011
:100940002B230593F30548BF26F40076F30558BF23
:100950004FF0010A00276E2A21DD6F3A092A00F2C2
:100960006D80DFE802F0054A6B6B6B6B226B6B4AA4
:1009700050EA010262D0C20842EA417206251346DB
:1009800065F3DF00E055013752EAD1004FEAD101AB
:100990004FEAD20040EA41721846F0D14EE0582AA0
:1009A0002BD0642A18BF692A48D150EA010245D0E9
:1009B0000C46054630040AD507F00300032806D18B
:1009C0000DF11E0B2C200BF80700013701E00DF193
:1009D0001E0B28460A22002302F0AAFD00EB80022B
:1009E000A5EB420242F030020BF807200137D5F1A7
:1009F00009020022A241DBD320E0002750EA0102D5
:100A00001CD0B20440F6B262C0F601025CBF40F6F0
:100A1000C262C0F60102030943EA017500F00F004B
:100A20002B46105CE055013755EA11104FEA1111C1
:100A30004FEA151040EA01751846EFD105994FF0BD
:100A4000FF30FF2988BF0138AAEB070222EAE27AC9
:100A500007EB0A03049AD41A002918BF0444B0050E
:100A600006D44046314622460CF061FB059900242D
:100A7000FF29039D05D9090A40460FF037FD059966
:100A800000E011B140460FF031FD404631462246AC
:100A90000CF04DFB4046302152460FF077FD012F00
:100AA00005DBE95D40460FF021FD013FF9D8F00676
:100AB0007FF5A4AD4046202122460FF067FD9DE55D
:100AC00046F4005646F4406B5FEACB5058BF4FF0F7
:100AD000060A0BF4406006990731A0F5406021F04A
:100AE0000701B0FA80F0BAF1000F08BF4FEA501AC0
:100AF000D1E9005646EC195B01F108000690B0EE12
:100B0000490B0CF0D5FA80B1B5EE409BF1EE10FA2E
:100B10001DD55FEA8B4040F6AA44C0F601045CBFD5
:100B200040F6AF44C0F6010424E0B0EE490B0FF0EC
:100B300097FC00284AD05FEA8B4040F6D264C0F6AA
:100B400001045CBF40F6D664C0F6010412E01BF459
:100B5000005040F6B442C0F6010240F6B941C0F67A
:100B60000101104612BF541C08464C1C5FEA8B6101
:100B700048BF04462BF48076002C04BF40F62E2498
:100B8000C0F60104F005204602D40FF091FD02E00A
:100B900051460FF0A3FD054626F40076A7EB000AA8
:100BA0004046314652460CF0C2FA35B114F8011BEA
:100BB00040460FF09BFC013DF8D1F0067FF51EADDD
:100BC0004046202152460FF0E1FC17E5B0EE490BFC
:100BD0000CF07BFA002804BF0646054646EC195B7C
:100BE000B0EE490B0FF044FC044686F0004040ECA8
:100BF000105B002C09FE009BB0EE490B0DA80FF016
:100C00003BFC0D9800EB400046F26761C6F266615E
:100C100050FB01F0002C18BF4BF0600B811001EB72
:100C2000D0700D90B5EE409BF1EE10FA16D0013069
:100C30000FF03EFCB4EE490BF1EE10FA0D9806D51C
:100C4000411C0D910230F3E70D9801380D900FF023
:100C50002FFCB4EE490BF1EE10FAF5DC0D990BF414
:100C60004064B4F5806F07D0B4F5406F0AD18A456F
:100C7000C8BF11F1050F05DCB1F59A7F13D189EEDC
:100C80000A9B15E05FEA4B5040F1E7800E2940F3E4
:100C9000C1804FF0000AE0E0002A7FF4AFACA1E28F
:100CA0000170FFF7ABBC48420FF002FC20EE099B3D
:100CB000B5EE409BF1EE10FA23D0B0EE490B0CF0EC
:100CC000F7F900287FF420AF0D98B4EE489BF1EEC1
:100CD00010FA08DB89EE089B0130B4EE489BF1EE78
:100CE00010FAF7DA0D90B4EE4B9BF1EE10FA08D53E
:100CF00029EE089B0138B4EE4B9BF1EE10FAF7D4C5
:100D00000D90B4F5406F544608BF013CBAF1000F96
:100D100018BFA246CAF100000FF0CAFB4FF0FF3027
:100D20000CF0E4F930EE090BB4EE480BF1EE10FADA
:100D3000A1BF0D9880EE080B01300D9050EC106BA8
:100D40000290BAF1000F35D005940BF40860B0F5AD
:100D5000006F31D1BAF1100FA8BF4FF0100A0298FE
:100D600040EC196B50460FF0A3FB20EE090B51EC41
:100D7000100B02F08FFB0446084300F007820D467B
:100D80004CF6CD42CCF6CC42A4FB0201531E04FB30
:100D9000031105FB0211C20742EA5102C90741EAE9
:100DA0005000D0F1993049F69910C1F69910904150
:100DB00080F0EE81CDF814A0059A0BF0800010436E
:100DC000A7EB02000D9D0CBF471F871F01245FEAA0
:100DD000CB4002D404950299BDE045F25650C5F2CD
:100DE000555055FB00F000EBD07000EB4000281A86
:100DF00002300299DFE800F003A1AB03A10041EC4F
:100E0000106B20EE080B51EC106B013D0D95013F6E
:100E100002249CE0C84350444FF0100A1028B8BF89
:100E200082465FEA0B6218D4B8B150460FF040FB1F
:100E3000B6EE001B00EE091BB0EE410BFFF7ECFA1B
:100E4000B0EE481BFFF744FAB5EE400BF1EE10FA96
:100E500002D1BAF1010AE8D10D99CDF814A0CAF176
:100E6000000010398142C8BF08460FF021FB4FF047
:100E7000FF300CF03BF930EE099B0D9801300FF07C
:100E800017FBB4EE490BF1EE10FA0D9898BF013044
:100E9000002814D411281AD3A0F110010D91C0F12B
:100EA00010000FF005FB20EE090B51EC100B02F0C7
:100EB000F1FA05460E460020CDE9010019E050EC9C
:100EC000191BCDE9011000250D95002611E051EC0C
:100ED000190B02F0DFFA05460E4602F0FBFA41EC70
:100EE000100B39EE400B50EC101BCDE90110002027
:100EF0000D902BF4806A40F23050C0F600000830AC
:100F0000002400F10801013405C8281A76EB02001C
:100F10000846F6D2059AB81A0BF0800111434FF03B
:100F2000FF321CBF1146013A1BF0600F08BF0A4692
:100F30000D99511A0844071B2AE041EC106B20EE72
:100F40000C0B51EC106B023D0D95023F032422EA7D
:100F5000E272CDE904522BF4006A41EC196B304681
:100F600002F098FA05460E4602F0B4FA41EC100B76
:100F700039EE400B50EC101BCDE901101BF0600F57
:100F800018BF013F04980FF08FFA6328C8BF013FD4
:100F900027EAE77B1AF4047F0DD1012F0BDB40F227
:100FA0003057C0F60007404620210FF09FFABBF1F2
:100FB000010BF8D103E040F23057C0F600075FEABA
:100FC0008A604FEA4A6003D4002808D5202103E054
:100FD0002D21002858BF2B2140460FF087FA5FEAE9
:100FE000CA6009D4BBF1000F06D0404630210FF093
:100FF0007DFABBF1010BF8D1013C07EBC40006C838
:10100000681A76EB0200302006D36D1A9641013043
:101010006B1A76EB0203F8D2C1B240460FF066FAC3
:10102000002CE9D15FEA0A540BD50D98012808DBA2
:1010300001380D90404630210FF058FA0D980028E5
:10104000F6DC0AF08000059D284343D040462E215F
:101050000FF04CFA1020102DB8BF2846002C0D9927
:1010600020EAE077384648BF401A0FF021FA012DF8
:1010700026DBDDE9011040EC111B20EE010B51ECE9
:10108000100B02F007FA04460D463E46013E40F2C0
:101090003050C0F6000000EBC60006C8601A75EBC1
:1010A0000200302006D3641A95410130631A75EBB3
:1010B0000203F8D2C1B240460FF018FA002EE5D173
:1010C0000599C81B06D07C1A404630210FF00EFA55
:1010D0000134F9D35FEA4A504BD545215FEA8A4093
:1010E00058BF652140460FF001FA0D980028404690
:1010F00004DB2B210FF0FAF90D9805E02D210FF0FC
:10110000F5F90D9840420D90642815DB48F21F5404
:10111000C5F2EB14A0FB0401302000EB5111404656
:101120000FF0E4F90D9850FB04F14A1102EBD17174
:10113000642201FB12000D9046F26764C6F26664F9
:1011400050FB04F0811001EBD07000F130014046FB
:101150000FF0CCF90D9850FB04F18A1002EBD1711D
:1011600001EB8101A0EB410000F1300140460FF09E
:10117000BDF9BBF1000F3FF441AA404620210FF01A
:10118000B5F9BBF1010BF8D1FFF738BA059013E6BA
:10119000CDF814A0204629460A22002302F0C8F9FF
:1011A00004460D460A22002302F0C2F905980138D0
:1011B00005903FF401AE52EA0300EBD0FCE5D8F80D
:1011C0000C0028B1D8E9001291423CBF00224254E1
:1011D00040460FF0CDF9D8F800000EB0BDEC0A8BF8
:1011E000BDE8F88F40460FF0C3F94FF0FF30F4E749
:1011F00085B0049000208DF80F0004988069E8B94C
:101200000498806A0290032817D80299DFE801F059
:10121000020B0214049890F82F00C00710B10120AF
:101220008DF80F0009E00498C06AB0F1C07F02D1C8
:1012300001208DF80F0000E0FFE73BE00498806993
:10124000B0F5005F20D10498806A019003281AD875
:101250000199DFE801F00206020F01208DF80F006E
:1012600011E0049890F82F00C00710B101208DF80C
:101270000F0008E00498C06AB0F1C07F02D10120DD
:101280008DF80F00FFE715E00498806A00900328AE
:1012900003D30098032804D00CE001208DF80F0040
:1012A00008E0049890F82F00C00710B101208DF8D5
:0C12B0000F00FFE79DF80F0005B070472D
:1012BC008AB044F21040C5F60200006800F0380015
:1012CC0001460191182800F25A810199DFE811F0CA
:1012DC001900570157015701570157015701570181
:1012EC003500570157015701570157015701570155
:1012FC003B0057015701570157015701570157013F
:10130C00410044F20040C5F602000068C0F34010F2
:10131C0068B144F20040C5F602000068C0F3C10198
:10132C0049F20000C0F2D030C840029004E049F20B
:10133C000000C0F2D030029026E140F60010C0F25E
:10134C003D00029020E147F64000C0F27D10029073
:10135C001AE144F22840C5F60200016801F00301CD
:10136C0008910068C0F30510079044F22C40C5F6B4
:10137C000200006800F001000690069844F2344127
:10138C00C5F60201096889B2C908484300EE100A83
:10139C00B8EE400A8DED040A0798002800F0EC80A6
:1013AC000898009038B10098012863D00098022862
:1013BC0000F08480A6E044F20040C5F6020000680C
:1013CC00C0F3401090B344F20040C5F60200006830
:1013DC00C0F3C10149F20000C0F2D030C840059002
:1013EC009DED050AB8EE400A9DED071AB8EE411ABC
:1013FC0080EE010A44F23040C5F6020000686FF33B
:10140C005F2001EE100AB8EE411A9DED042A9FED03
:10141C00613A82EE032A31EE021AB7EE002A31EE5F
:10142C00021A20EE010A8DED030A22E09DED070A57
:10143C00B8EE401A9FED590A80EE010A44F2304092
:10144C00C5F6020000686FF35F2001EE100AB8EEDB
:10145C00411A9DED042A9FED4F3A82EE032A31EE9C
:10146C00021AB7EE002A31EE021A20EE010A8DEDB7
:10147C00030A6AE09DED070AB8EE401A9FED460A92
:10148C0080EE010A44F23040C5F6020000686FF3AA
:10149C005F2001EE100AB8EE411A9DED042A9FED73
:1014AC003D3A82EE032A31EE021AB7EE002A31EEF3
:1014BC00021A20EE010A8DED030A46E09DED070AA3
:1014CC00B8EE401A9FED320A80EE010A44F2304029
:1014DC00C5F6020000686FF35F2001EE100AB8EE4B
:1014EC00411A9DED042A9FED2B3A82EE032A31EE30
:1014FC00021AB7EE002A31EE021A20EE010A8DED27
:10150C00030A22E09DED070AB8EE401A9FED220A6D
:10151C0080EE010A44F23040C5F6020000686FF319
:10152C005F2001EE100AB8EE411A9DED042A9FEDE2
:10153C00193A82EE032A31EE021AB7EE002A31EE86
:10154C00021A20EE010A8DED030A44F23040C5F672
:10155C000200006881B2012000EB512009909DED42
:10156C00030A9DED091AB8EE411A80EE010ABCEE91
:10157C00C00A8DED020A01E00020029004E040F662
:10158C000010C0F23D00029002980AB0704700BFF4
:10159C0020BCBE4B000000460024744A0024744C4E
:1015AC0080B59AB0189000208DF857008DF8560031
:1015BC001898C0780007002840D51898406E1490F1
:1015CC0060B11498B0F5801F11D01498B0F5001FBD
:1015DC0015D01498B0F5401F19D019E044F22C41E5
:1015EC00C5F60201086840F40030086013E0189852
:1015FC000830022106F01FFD8DF857000BE01898FB
:10160C002830022106F06EFE8DF8570003E002E050
:10161C0001208DF857009DF8570058B944F25041FD
:10162C00C5F60201086820F44010189A526E104357
:10163C00086003E09DF857008DF856001898407824
:10164C00C00700283BD01898806D1390042820D830
:10165C001399DFE801F0030C141C1D0044F22C411B
:10166C00C5F60201086840F40030086014E01898D0
:10167C000830002106F0DFFC8DF857000CE01898BC
:10168C002830002106F02EFE8DF8570004E003E010
:10169C0002E001208DF857009DF8570058B944F22C
:1016AC005041C5F60201086820F00700189A926DA7
:1016BC001043086003E09DF857008DF85600189809
:1016CC004078400700284CD51898D0F8A400129008
:1016DC00A0B11298B0F5001F19D01298B0F5800F78
:1016EC001DD01298B0F5C00F21D01298B0F5000F94
:1016FC001ED01298B0F5200F1BD01BE044F22C41E9
:10170C00C5F60201086840F40030086015E018982E
:10171C000830002106F08FFC8DF857000DE018986A
:10172C002830002106F0DEFD8DF8570005E004E0BE
:10173C0003E002E001208DF857009DF8570060B9D6
:10174C0044F25841C5F60201086820F46000189A6A
:10175C00D2F8A4201043086003E09DF857008DF8E0
:10176C00560018984078000700284CD51898D0F8E7
:10177C00A8001190A0B11198B0F1807F19D01198E8
:10178C00B0F1007F1DD01198B0F1407F21D011989D
:10179C00B0F1806F1ED01198B0F1A06F1BD01BE080
:1017AC0044F22C41C5F60201086840F40030086090
:1017BC0015E018980830002106F03DFC8DF8570014
:1017CC000DE018982830002106F08CFD8DF857009C
:1017DC0005E004E003E002E001208DF857009DF8DD
:1017EC00570060B944F25841C5F60201086820F070
:1017FC00E060189AD2F8A8201043086003E09DF826
:10180C0057008DF856001898C0788007002836D5F8
:10181C001898C06C1090D8B11098102806D0109859
:10182C0020280CD01098302811D012E044F22C4112
:10183C00C5F60201086840F4003008600CE0189806
:10184C000830022106F0F7FB8DF8570004E003E0A6
:10185C0002E001208DF857009DF8570058B944F26A
:10186C004C41C5F60201086820F03000189AD26C81
:10187C001043086003E09DF857008DF85600189847
:10188C004078C006002845D51898C06D0F9080B1DF
:10189C000F98B0F5805F15D00F98B0F5005F19D098
:1018AC000F98B0F5405F1DD00F98B0F5804F1AD04F
:1018BC001AE044F22C41C5F60201086840F40030ED
:1018CC00086014E018980830002106F0B4FB8DF87D
:1018DC0057000CE018982830002106F003FD8DF815
:1018EC00570004E003E002E001208DF857009DF85A
:1018FC00570058B944F25041C5F60201086820F46B
:10190C00E040189AD26D1043086003E09DF8570030
:10191C008DF85600189840788006002842D5189803
:10192C00006E0E90A0B10E98B0F5803F11D00E98BD
:10193C00B0F5003F15D00E98B0F5403F19D00E9879
:10194C00B0F5802F16D00E98B0F5A02F13D013E061
:10195C0015E018980830012106F06DFB8DF8570042
:10196C000DE018982830012106F0BCFC8DF85700CA
:10197C0005E004E003E002E001208DF857009DF83B
:10198C00570058B944F25041C5F60201086820F4DA
:10199C00E020189A126E1043086003E09DF857007F
:1019AC008DF85600189840784006002844D51898B1
:1019BC00D0F8AC000D90A0B10D98B0F1805F11D0B3
:1019CC000D98B0F1005F15D00D98B0F1405F19D0B3
:1019DC000D98B0F1804F16D00D98B0F1A04F13D0E8
:1019EC0013E015E018980830012106F024FB8DF85F
:1019FC0057000DE018982830012106F073FC8DF883
:101A0C00570005E004E003E002E001208DF85700E8
:101A1C009DF8570060B944F25841C5F602010868B8
:101A2C0020F0E040189AD2F8AC201043086003E094
:101A3C009DF857008DF8560018984078000600283D
:101A4C0034D51898C06E0C90C8B10C98B0F1805F6A
:101A5C0004D00C98B0F1005F09D011E044F22C4195
:101A6C00C5F60201086840F4003008600BE01898D5
:101A7C000830012106F0DFFA8DF8570003E002E090
:101A8C0001208DF857009DF8570058B944F2504189
:101A9C00C5F60201086820F04050189AD26E104327
:101AAC00086003E09DF857008DF856001898C07830
:101ABC00C00790B31898806C0B90032817D80B991B
:101ACC00DFE801F014020B1344F22C41C5F60201BD
:101ADC00086840F4003008600CE0189808300221C7
:101AEC0006F0A9FA8DF8570004E003E002E00120AB
:101AFC008DF857009DF8570058B944F24C41C5F683
:101B0C000201086820F00300189A926C10430860D8
:101B1C0003E09DF857008DF8560018988078400621
:101B2C00002840F1E6821898D0F8B000B0F5807F1C
:101B3C0000F03A821898D0F8B000B0F5007F00F0B1
:101B4C0033821898D0F8B000B0F50C5F00F02C82FE
:101B5C001898D0F8B000B0F54C5F00F025821898BA
:101B6C00D0F8B000B0F5864F00F01E821898D0F86F
:101B7C00B000B0F5A64F00F017821898D0F8B0005E
:101B8C00B0F5C64F00F010821898D0F8B000B0F540
:101B9C00E64F00F009821898D0F8B000B0F5034F6A
:101BAC0000F002821898D0F8B000B0F5134F00F096
:101BBC00FB811898D0F8B000B0F5234F00F0F481F9
:101BCC001898D0F8B000B0F5334F00F0ED811898AC
:101BDC00D0F8B000B0F5434F00F0E6811898D0F87B
:101BEC00B000B0F5534F00F0DF811898D0F8B0007A
:101BFC00B0F5634F00F0D8811898D0F8B000B0F56C
:101C0C00734F00F0D1811898D0F8B00040F2003139
:101C1C00C0F20101884200F0C7811898D0F8B000DA
:101C2C0041F20031C0F20101884200F0BD811898E8
:101C3C00D0F8B00042F20031C0F20101884200F04D
:101C4C00B3811898D0F8B00043F20031C0F2010112
:101C5C00884200F0A9811898D0F8B00044F2003105
:101C6C00C0F20101884200F09F811898D0F8B000B2
:101C7C0045F20031C0F20101884200F095811898BC
:101C8C00D0F8B00046F20031C0F20101884200F0F9
:101C9C008B811898D0F8B00047F20031C0F20101E6
:101CAC00884200F081811898D0F8B00048F20031D9
:101CBC00C0F20101884200F077811898D0F8B0008A
:101CCC0049F20031C0F20101884200F06D81189890
:101CDC00D0F8B0004AF20031C0F20101884200F0A5
:101CEC0063811898D0F8B0004BF20031C0F20101BA
:101CFC00884200F059811898D0F8B0004CF20031AD
:101D0C00C0F20101884200F04F811898D0F8B00061
:101D1C004DF20031C0F20101884200F04581189863
:101D2C00D0F8B0004EF20031C0F20101884200F050
:101D3C003B811898D0F8B0004FF20031C0F201018D
:101D4C00884200F031811898D0F8B00040F2003190
:101D5C00C0F20201884200F027811898D0F8B00038
:101D6C0041F20031C0F20201884200F01D81189846
:101D7C00D0F8B00042F20031C0F20201884200F00B
:101D8C0013811898D0F8B00043F20031C0F2020170
:101D9C00884200F009811898D0F8B00044F2003164
:101DAC00C0F20201884200F0FF801898D0F8B00011
:101DBC0045F20031C0F20201884200F0F58018981B
:101DCC00D0F8B00046F20031C0F20201884200F0B7
:101DDC00EB801898D0F8B00047F20031C0F2020145
:101DEC00884200F0E1801898D0F8B00048F2003139
:101DFC00C0F20201884200F0D7801898D0F8B000E9
:101E0C0049F20031C0F20201884200F0CD801898EE
:101E1C00D0F8B0004AF20031C0F20201884200F062
:101E2C00C3801898D0F8B0004BF20031C0F2020118
:101E3C00884200F0B9801898D0F8B0004CF200310C
:101E4C00C0F20201884200F0AF801898D0F8B000C0
:101E5C004DF20031C0F20201884200F0A5801898C2
:101E6C00D0F8B0004EF20031C0F20201884200F00E
:101E7C009B801898D0F8B0004FF20031C0F20201EC
:101E8C00884200F091801898D0F8B00040F20031F0
:101E9C00C0F20301884200F087801898D0F8B00097
:101EAC0041F20031C0F2030188427DD01898D0F87D
:101EBC00B00042F20031C0F20301884274D018988D
:101ECC00D0F8B00043F20031C0F2030188426BD06D
:101EDC001898D0F8B00044F20031C0F203018842E7
:101EEC0062D01898D0F8B00045F20031C0F203016E
:101EFC00884259D01898D0F8B00046F20031C0F2A0
:101F0C000301884250D01898D0F8B00047F2003145
:101F1C00C0F20301884247D01898D0F8B00048F2BC
:101F2C000031C0F2030188423ED01898D0F8B000BE
:101F3C0049F20031C0F20301884235D01898D0F82C
:101F4C00B0004AF20031C0F2030188422CD018983C
:101F5C00D0F8B0004BF20031C0F20301884223D01C
:101F6C001898D0F8B0004CF20031C0F2030188424E
:101F7C001AD01898D0F8B0004DF20031C0F203011D
:101F8C00884211D01898D0F8B0004EF20031C0F24F
:101F9C000301884208D01898D0F8B0004FF20031F5
:101FAC00C0F20301884200D107E040F67630C0F65B
:101FBC00010040F27D3102F0E9FB44F60001C5F668
:101FCC000201086840F4807008600BF0C5FB1690A5
:101FDC0044F60000C5F602000068C00500280AD4CB
:101FEC000BF0BAFB1699401A652803D303208DF821
:101FFC00570000E0ECE79DF85700002875D144F23B
:10200C007040C5F60200006800F440701899D1F8D1
:10201C00B01001F44071884211D044F27041C5F601
:10202C000201086820F440701790086840F4803072
:10203C000860086820F480300860179808601898C9
:10204C00D0F8B000B0F5807F17D10BF085FB16905F
:10205C0044F27040C5F602000068C0F3400060B95D
:10206C000BF07AFB1699401A41F28931884203D35E
:10207C0003208DF8570000E0EAE79DF8570078BB85
:10208C001898D0F8B00000F44070B0F5407F12D131
:10209C0044F21041C5F60201086820F47C50189AED
:1020AC00D2F8B0204FF6F043C0F6FF731A4040EA66
:1020BC001210086007E044F21041C5F602010868EE
:1020CC0020F47C5008601898D0F8B0206FF31F32C1
:1020DC0044F27041C5F6020108681043086003E041
:1020EC009DF857008DF8560003E09DF857008DF8C9
:1020FC00560018980068C007002800F04780189810
:10210C00806F0A9028282BD80A99DFE801F015294E
:10211C0029292929292916292929292929291E2941
:10212C002929292929292629292929292929272918
:10213C00292929292929280015E018980830012176
:10214C0005F079FF8DF857000DE018982830012123
:10215C0006F0C8F88DF8570005E004E003E002E053
:10216C0001208DF857009DF8570058B944F254419E
:10217C00C5F60201086820F03800189A926F1043D7
:10218C00086003E09DF857008DF856001898007809
:10219C008007002834D51898406F0990052819D865
:1021AC000999DFE801F003040C14151615E01898D2
:1021BC000830012105F03FFF8DF857000DE018980D
:1021CC002830012106F08EF88DF8570005E004E068
:1021DC0003E002E001208DF857009DF8570058B934
:1021EC0044F25441C5F60201086820F00700189A21
:1021FC00526F1043086003E09DF857008DF85600AD
:10220C00189800784007002836D51898D0F8900018
:10221C000890052819D80899DFE801F003040C147C
:10222C00151615E018980830012105F004FF8DF8FB
:10223C0057000DE018982830012106F053F88DF85E
:10224C00570005E004E003E002E001208DF85700A0
:10225C009DF8570060B944F25841C5F60201086870
:10226C0020F00700189AD2F890201043086003E081
:10227C009DF857008DF856001898007880060028B5
:10228C0044D51898D0F88C000790A0B10798B0F1FD
:10229C00805F11D00798B0F1005F15D00798B0F1AE
:1022AC00405F19D00798B0F1804F16D00798B0F165
:1022BC00A04F13D013E015E018980830002105F05A
:1022CC00BAFE8DF857000DE018982830022106F060
:1022DC0009F88DF8570005E004E003E002E0012066
:1022EC008DF857009DF8570060B944F25441C5F67B
:1022FC000201086820F0E040189AD2F88C201043B4
:10230C00086003E09DF857008DF856001898007887
:10231C004006002844D51898D0F898000690A0B133
:10232C000698B0F5806F11D00698B0F5006F15D0F7
:10233C000698B0F5406F19D00698B0F5805F16D0AE
:10234C000698B0F5A05F13D013E015E0189808308C
:10235C00002105F070FE8DF857000DE0189828301C
:10236C00022105F0BFFF8DF8570005E004E003E003
:10237C0002E001208DF857009DF8570060B944F237
:10238C005841C5F60201086820F4E050189AD2F8BA
:10239C0098201043086003E09DF857008DF8560014
:1023AC00189800780006002844D51898D0F89C009E
:1023BC000590A0B10598B0F5005F11D00598B0F567
:1023CC00804F15D00598B0F5C04F19D00598B0F5D1
:1023DC00004F16D00598B0F5204F13D013E015E040
:1023EC0018980830002105F026FE8DF857000DE0F6
:1023FC0018982830022105F075FF8DF8570005E07C
:10240C0004E003E002E001208DF857009DF857002E
:10241C0060B944F25841C5F60201086820F46040E6
:10242C00189AD2F89C201043086003E09DF85700DE
:10243C008DF85600189800780007002839D51898A0
:10244C00D0F88000B0F5805F0FD01898D0F88000DD
:10245C00B0F5005F09D01898D0F8800028B1189812
:10246C00D0F88000B0F5405F00D107E040F6763040
:10247C00C0F6010040F2FC4102F088F91898D0F83F
:10248C008000B0F5805F08D118982830022105F043
:10249C0029FF10B101208DF8560044F25441C5F6C5
:1024AC000201086820F44050189AD2F8802010439A
:1024BC00086018980078C006002839D51898D0F80C
:1024CC009400B0F5807F0FD01898D0F89400B0F538
:1024DC00007F09D01898D0F8940028B11898D0F83B
:1024EC009400B0F5407F00D107E040F67630C0F69E
:1024FC0001004FF4A46102F049F91898D0F8940047
:10250C00B0F5807F08D118982830022105F0EAFE3A
:10251C0010B101208DF8560044F25841C5F6020165
:10252C00086820F44070189AD2F894201043086080
:10253C00189880780007002835D51898D0F8A00096
:10254C00049040B10498B0F5803F0CD00498B0F5DD
:10255C00003F10D010E018980830002105F06BFDFA
:10256C008DF857000BE018982830022105F0BAFEC0
:10257C008DF8570003E002E001208DF857009DF81C
:10258C00570060B944F25841C5F60201086820F4BE
:10259C004030189AD2F8A0201043086003E09DF850
:1025AC0057008DF85600189880784007002838D5C9
:1025BC001898D0F884000390B0F5801F08D00398C9
:1025CC00B0F5001F0DD00398B0F5401F11D011E0ED
:1025DC0044F22C41C5F60201086840F40030086052
:1025EC000BE018982830012105F07CFE8DF857007F
:1025FC0003E002E001208DF857009DF8570060B908
:10260C0044F25441C5F60201086820F44010189AAF
:10261C00D2F884201043086003E09DF857008DF831
:10262C00560018988078C007002840D01898006D84
:10263C0020B11898006DB0F5803F00D107E040F64E
:10264C007630C0F6010040F2865102F09FF81898DF
:10265C00006D029020B10298B0F5803F09D010E0D7
:10266C0044F22C41C5F60201086840F400300860C1
:10267C000AE018980830022105F0DDFC8DF85700AF
:10268C0002E001208DF857009DF8570058B944F22C
:10269C004C41C5F60201086820F48030189A126D7E
:1026AC001043086003E09DF857008DF85600189809
:1026BC00C0788006002808D518982830022105F02B
:1026CC0011FE10B101208DF8560018988078800703
:1026DC00002832D51898C06F0190B8B10198B0F5A8
:1026EC00807F08D00198B0F5007F0DD00198B0F52F
:1026FC00407F0AD00BE044F22C41C5F60201086879
:10270C0040F40030086005E004E003E002E0012042
:10271C008DF857009DF8570058B944F25441C5F64E
:10272C000201086820F44070189AD26F10430860B8
:10273C0003E09DF857008DF8560018988078C00675
:10274C0000281BD51898006F20B11898006FB0F1B5
:10275C00004F00D107E040F67630C0F6010040F2A1
:10276C00E55102F013F844F25041C5F60201086835
:10277C0020F00040189A126F104308601898807867
:10278C00800600281BD51898806E20B11898806E92
:10279C00B0F1807F00D107E040F67630C0F6010042
:1027AC0040F2F95101F0F2FF44F25041C5F602013A
:1027BC00086820F08070189A926E10430860189880
:1027CC00C0784006002820D51898D0F8B40028B15D
:1027DC001898D0F8B400B0F5004F00D107E040F6DF
:1027EC007630C0F6010040F20F6101F0CFFF44F2E9
:1027FC001041C5F60201086820F4004008601898E2
:10280C00D0F8B4200868104308601898C078000607
:10281C00002820D51898406D48B11898406DB0F13B
:10282C00805F04D01898406DB0F1005F00D107E0D4
:10283C0040F67630C0F6010040F2196101F0A6FFB7
:10284C0044F24C41C5F60201086820F04050189A39
:10285C00526D10430860189880780006002824D523
:10286C001898D0F8880058B11898D0F88800B0F5AE
:10287C00800F05D01898D0F88800B0F5000F00D163
:10288C0007E040F67630C0F6010040F2236101F01B
:10289C007DFF44F25441C5F60201086820F4400063
:1028AC00189AD2F888201043086018980079C0074D
:1028BC0070B118980830002105F0BDFB8DF8570059
:1028CC009DF8570000B903E09DF857008DF85600AD
:1028DC0018980079800700280ED518980830012127
:1028EC0005F0A9FB8DF857009DF8570000B903E0DF
:1028FC009DF857008DF8560018980079400700286D
:10290C000ED518980830022105F095FB8DF857006C
:10291C009DF8570000B903E09DF857008DF856005C
:10292C0018980079000700280ED518982830002137
:10293C0005F0D8FC8DF857009DF8570000B903E05E
:10294C009DF857008DF8560018980079C00600289D
:10295C000ED518982830012105F0C4FC8DF85700CD
:10296C009DF8570000B903E09DF857008DF856000C
:10297C0018980079800600280ED518982830022166
:10298C0005F0B0FC8DF857009DF8570000B903E036
:10299C009DF857008DF856009DF8560018B9002088
:1029AC008DF8670002E001208DF867009DF8670044
:0429BC001AB080BD10
:1029C00088B0079044F22840C5F60200016801F083
:1029D000030106910068C0F30530059044F22C40D5
:1029E000C5F602000068C0F300100490049844F299
:1029F0003C41C5F60201096889B2C908484300EEA6
:102A0000100AB8EE400A8DED020A0598002800F081
:102A100012810698009038B10098012863D0009880
:102A2000022800F08480A6E044F20040C5F60200CF
:102A30000068C0F3401090B344F20040C5F60200B5
:102A40000068C0F3C10149F20000C0F2D030C840B4
:102A500003909DED030AB8EE400A9DED051AB8EE0D
:102A6000411A80EE010A44F23840C5F602000068BF
:102A70006FF35F2001EE100AB8EE411A9DED022AB5
:102A80009FED723A82EE032A31EE021AB7EE002A67
:102A900031EE021A20EE010A8DED010A22E09DEDD1
:102AA000050AB8EE401A9FED6B0A80EE010A44F267
:102AB0003840C5F6020000686FF35F2001EE100A8F
:102AC000B8EE411A9DED022A9FED603A82EE032A8C
:102AD00031EE021AB7EE002A31EE021A20EE010A98
:102AE0008DED010A6AE09DED050AB8EE401A9FEDF2
:102AF000580A80EE010A44F23840C5F60200006828
:102B00006FF35F2001EE100AB8EE411A9DED022A24
:102B10009FED4E3A82EE032A31EE021AB7EE002AFA
:102B200031EE021A20EE010A8DED010A46E09DED1C
:102B3000050AB8EE401A9FED440A80EE010A44F2FD
:102B40003840C5F6020000686FF35F2001EE100AFE
:102B5000B8EE411A9DED022A9FED3C3A82EE032A1F
:102B600031EE021AB7EE002A31EE021A20EE010A07
:102B70008DED010A22E09DED050AB8EE401A9FEDA9
:102B8000340A80EE010A44F23840C5F602000068BB
:102B90006FF35F2001EE100AB8EE411A9DED022A94
:102BA0009FED2A3A82EE032A31EE021AB7EE002A8E
:102BB00031EE021A20EE010A8DED010A9DED010AA7
:102BC00044F23840C5F60200016889B2490A01EEB4
:102BD000101AB8EE411AB7EE002A31EE021A80EE52
:102BE000010A0799BCEEC00A81ED000A9DED010AB9
:102BF0000168C1F3064101EE101AB8EE411A31EE38
:102C0000021A80EE010A0799BCEEC00A81ED010AA2
:102C10009DED010A0068C0F3066001EE100AB8EEEF
:102C2000411A31EE021A80EE010A0798BCEEC00A82
:102C300080ED020A06E007990020086007994860C5
:102C40000799886008B0704720BCBE4B0000004662
:082C50000024744A0024744CB6
:102C580088B0079044F22840C5F60200016801F0E8
:102C6800030106910068C0F30550059044F22C401A
:102C7800C5F602000068C0F300200490049844F2EE
:102C88004441C5F60201096889B2C908484300EE03
:102C9800100AB8EE400A8DED020A0598002800F0E7
:102CA80012810698009038B10098012863D00098E6
:102CB800022800F08480A6E044F20040C5F6020035
:102CC8000068C0F3401090B344F20040C5F602001B
:102CD8000068C0F3C10149F20000C0F2D030C8401A
:102CE80003909DED030AB8EE400A9DED051AB8EE73
:102CF800411A80EE010A44F24040C5F6020000681D
:102D08006FF35F2001EE100AB8EE411A9DED022A1A
:102D18009FED723A82EE032A31EE021AB7EE002ACC
:102D280031EE021A20EE010A8DED010A22E09DED36
:102D3800050AB8EE401A9FED6B0A80EE010A44F2CC
:102D48004040C5F6020000686FF35F2001EE100AEC
:102D5800B8EE411A9DED022A9FED603A82EE032AF1
:102D680031EE021AB7EE002A31EE021A20EE010AFD
:102D78008DED010A6AE09DED050AB8EE401A9FED57
:102D8800580A80EE010A44F24040C5F60200006885
:102D98006FF35F2001EE100AB8EE411A9DED022A8A
:102DA8009FED4E3A82EE032A31EE021AB7EE002A60
:102DB80031EE021A20EE010A8DED010A46E09DED82
:102DC800050AB8EE401A9FED440A80EE010A44F263
:102DD8004040C5F6020000686FF35F2001EE100A5C
:102DE800B8EE411A9DED022A9FED3C3A82EE032A85
:102DF80031EE021AB7EE002A31EE021A20EE010A6D
:102E08008DED010A22E09DED050AB8EE401A9FED0E
:102E1800340A80EE010A44F24040C5F60200006818
:102E28006FF35F2001EE100AB8EE411A9DED022AF9
:102E38009FED2A3A82EE032A31EE021AB7EE002AF3
:102E480031EE021A20EE010A8DED010A9DED010A0C
:102E580044F24040C5F60200016889B2490A01EE11
:102E6800101AB8EE411AB7EE002A31EE021A80EEB7
:102E7800010A0799BCEEC00A81ED000A9DED010A1E
:102E88000168C1F3064101EE101AB8EE411A31EE9D
:102E9800021A80EE010A0799BCEEC00A81ED010A08
:102EA8009DED010A0068C0F3066001EE100AB8EE55
:102EB800411A31EE021A80EE010A0798BCEEC00AE8
:102EC80080ED020A06E0079900200860079948602B
:102ED8000799886008B0704720BCBE4B00000046C8
:082EE8000024744A0024744C1C
:102EF00080B586B004900391029200208DF80700FF
:102F0000029888B1029804280ED0029808280BD0A5
:102F100002980C2808D00298102805D0029814288E
:102F200002D002983C2800D107E040F65C10C0F6C1
:102F3000010041F2B30101F02FFC03980068602802
:102F40001FD00398006870281BD0039800684021A8
:102F5000C0F20101884214D0039800685021C0F2E9
:102F6000010188420DD0039800686021C0F2010180
:102F7000884206D0039800687021C0F2010188429F
:102F800000D107E040F65C10C0F6010041F2B40148
:102F900001F002FC0398806818B103988068022849
:102FA00000D107E040F65C10C0F6010041F2B50127
:102FB00001F0F2FB0398006918B103980069042836
:102FC00000D107E040F65C10C0F6010041F2B60106
:102FD00001F0E2FB049890F83C00012803D10220A4
:102FE0008DF8170048E20499012081F83C0002980E
:102FF0000090142800F235820099DFE811F01500E6
:10300000320232023202A3003202320232021201D2
:103010003202320232027001320232023202CF0137
:103020003202320232020002049800680021C4F227
:103030000101884264D004980068B0F1804F5FD0ED
:103040000498006840F20041C4F20001884257D061
:103050000498006840F60001C4F2000188424FD095
:103060000498006840F60041C4F20001884247D04D
:103070000498006840F20041C4F2010188423FD048
:103080000498006841F60001C4F20001884237D07C
:103090000498006841F60041C4F2000188422FD034
:1030A0000498006842F20001C4F20001884227D06F
:1030B0000498006844F20001C4F2010188421FD064
:1030C0000498006844F20041C4F20101884217D01C
:1030D0000498006844F60001C4F2010188420FD050
:1030E000049800684EF20001C4F20001884207D043
:1030F000049800684EF20041C4F20001884200D1F9
:1031000007E040F65C10C0F601004FF4865101F074
:1031100043FB04980068039906F092FE0498016846
:10312000886940F00800886104980168886920F087
:103130000400886103980269049801688869104353
:10314000886191E1049800680021C4F2010188427D
:1031500044D004980068B0F1804F3FD004980068D4
:1031600040F20041C4F20001884237D00498006860
:1031700040F60001C4F2000188422FD00498006894
:1031800040F60041C4F20001884227D0049800684C
:1031900040F20041C4F2010188421FD00498006847
:1031A00041F60001C4F20001884217D0049800687B
:1031B00044F20001C4F2010188420FD00498006873
:1031C0004EF20001C4F20001884207D00498006862
:1031D0004EF20041C4F20001884200D107E040F6FF
:1031E0005C10C0F6010041F2D10101F0D5FA04985B
:1031F000006803990CF03CFC04980168886940F46D
:103200000060886104980168886920F480608861A2
:103210000398026904980168886940EA022088617D
:1032200022E1049800680021C4F20101884234D0F0
:1032300004980068B0F1804F2FD00498006840F2E5
:103240000041C4F20001884227D00498006840F68B
:103250000001C4F2000188421FD00498006840F6C3
:103260000041C4F20001884217D00498006840F27F
:103270000041C4F2010188420FD0049800684EF268
:103280000001C4F20001884207D0049800684EF2A1
:103290000041C4F20001884200D107E040F65C1012
:1032A000C0F6010041F2E20101F076FA04980068EC
:1032B000039906F094FE04980168C86940F008007C
:1032C000C86104980168C86920F00400C8610398C7
:1032D000026904980168C8691043C861C4E0049891
:1032E00000680021C4F20101884234D004980068CB
:1032F000B0F1804F2FD00498006840F20041C4F232
:103300000001884227D00498006840F60001C4F20A
:10331000000188421FD00498006840F60041C4F2C2
:103320000001884217D00498006840F20041C4F2BE
:10333000010188420FD0049800684EF20001C4F2E7
:103340000001884207D0049800684EF20041C4F2A0
:103350000001884200D107E040F65C10C0F6010091
:1033600041F2F30101F018FA04980068039906F09D
:103370000FFF04980168C86940F40060C8610498B0
:103380000168C86920F48060C861039802690498E4
:103390000168C86940EA0220C86165E004980068D5
:1033A0000021C4F20101884207D00498006840F26D
:1033B0000041C4F20101884200D107E040F65C10F0
:1033C000C0F6010041F2041101F0E6F9049800682A
:1033D00003990CF027FC04980168486D40F0080040
:1033E000486504980168486D20F00400486503981A
:1033F000026904980168486D1043486534E00498F8
:1034000000680021C4F20101884207D004980068D6
:1034100040F20041C4F20101884200D107E040F6C9
:103420005C10C0F6010041F2151101F0B5F90498E5
:103430000068039906F025FF04980168486D40F480
:103440000060486504980168486D20F48060486514
:103450000398026904980168486D40EA02204865B3
:1034600002E001208DF807000499002081F83C005B
:103470009DF807008DF817009DF8170006B080BD75
:10348000034C206804348047FBE701F0BEF8FEE7F8
:043490005C0F0108C4
:103494000A15C90241EA5051C00241F0004140F20C
:1034A4001E439A1A08DA20320DD4D141D040484044
:1034B4009140D14048407047202A28BF202231FA49
:1034C40002F0002170476FF000010846704700BF0A
:1034D400F9B140F23D42B1FA81F3D21AC3F1200CA2
:1034E40030FA0CFC9840994051EA0C0183054FEAEC
:1034F400D02040EA41504FEAD12101EB025138BFBC
:103504007047013041F100011B4208BF20F0010067
:10351400704748B140F21D42B0FA80F3D21A984085
:0C352400C10A400501EB0251704700BFD6
:10353000002B35D129B9B0FBF2FC0CFB120260461E
:103540007047914215D22DE9F041B2FA82F39A40C8
:103550009940D3F1200C30FA0CFC51EA0C01984050
:1035600000F04EF8280036FA03F200210023BDE8EF
:10357000F081F0B5B1FBF2FC0CFB1211B2FA82F350
:103580009A409940D3F1200630FA06F6314398402C
:1035900000F036F8614628003200DA400023F0BD22
:1035A000F3B5B3FA83FC49085FEA300013FA0CF371
:1035B000DCF1200432FA04F423430CB41A0000F0C6
:1035C0001FF80CBC33FA0CF3DCF11F0C35FA0CF5C8
:1035D00018BF013D03BCA5FB026705FB0377801BF9
:1035E000B941904271EB030C05D3821A71EB0303CE
:1035F000681C0021F0BD02000B0028000021F0BD76
:10360000940D4FF6C2752D02B5FBF4F4D60A0136BF
:1036100004FB04F5A5FB0656F64306EB0416550815
:1036200032BF00277708013505FB1677A6FB074751
:103630007F0807EBC63714001500E7FB02457F1B28
:103640004D1C0400E7FB014505FB1206A64284BFA2
:10365000013DB618964224BF0135B61A704700BF27
:103660005AB3844690EA01039B071FD1830707D012
:1036700011F8013B00F8013B013AF7D11CE0844608
:10368000203A09D32DE9F007B1E8F807A0E8F807D8
:10369000203AF9D2BDE8F0071C3205D451F8043BBA
:1036A00040F8043B043AF9D2043205D011F8013B4A
:0C36B00000F8013B013AF9D16046704778
:1036BC0000220B0011001A0084465AB3830704D071
:1036CC0000F8011B013AF9D124E0C9B241EA012109
:1036DC0041EA0141202A11D3203A2DE9F0030B468F
:1036EC000C460D460E460F4688468946A0E8FA035E
:1036FC00203AFBD2BDE8F00320320BD0042A05D3CC
:10370C0040F8041B043A05D0042AF9D200F8011B36
:08371C00013AFBD16046704741
:0C372400840C0108503700083037000802
:103730007507010895070108EBD20008A1070108E9
:1037400095070108EBD20008DDD200084107010807
:10375000860C0108380D0108380D0108380D0108E4
:10376000380D0108380D0108380D0108380D010821
:10377000380D0108380D0108FFFFFFFFFFFFFFFFB5
:10378000FFFFFFFFFFFF00004A0C0108EA0C0108E1
:10379000350A0108070D01088C0A0108D80C010838
:0837A000E10C0108930A010885
:1037A80080B59EB01D9000208DF867001D98406878
:1037B8004BF62041C0F2BE01884200D807E040F62F
:1037C800D250C0F6010040F6E23100F0E1FF1D984A
:1037D8008068B0F1805F07D01D98806820B11D987F
:1037E8008068B0F5805F00D107E040F6D250C0F69F
:1037F800010040F6E33100F0CBFF1D98006840F669
:103808000041C5F60001884211D11D98C06820B159
:103818001D98C068B0F5005F00D107E040F6D250AF
:10382800C0F6010040F6E63100F0B2FF2BE01D982B
:10383800C068B0F5805F0CD01D98C06848B11D986D
:10384800C068B0F5405F04D01D98C068B0F5005F4F
:1038580000D107E040F6D250C0F6010040F6EA3148
:1038680000F096FF1D98006A20B11D98006AB0F517
:10387800006F00D107E040F6D250C0F6010040F6D4
:10388800EB3100F085FF1D98006948B11D9800696B
:10389800B0F5806F04D01D980069B0F5C06F00D1F5
:1038A80007E040F6D250C0F6010040F6EE3100F0D5
:1038B8006FFF1D9840696FF00C01084203D11D98F5
:1038C800406900B107E040F6D250C0F6010040F66A
:1038D800EF3100F05DFF1D98806970B11D98806917
:1038E800B0F5807F09D01D988069B0F5007F04D0BD
:1038F8001D988069B0F5407F00D107E040F6D250AE
:10390800C0F601004FF43F6100F042FF1D98C06906
:1039180020B11D98C069B0F5004F00D107E040F60E
:10392800D250C0F6010040F6F13100F031FF1D9889
:10393800406A58B31D98406A012827D01D98406AEC
:10394800022823D01D98406A03281FD01D98406A7A
:1039580004281BD01D98406A052817D01D98406A76
:10396800062813D01D98406A07280FD01D98406A72
:1039780008280BD01D98406A092807D01D98406A6E
:103988000A2803D01D98406A0B2800D107E040F6AA
:10399800D250C0F6010040F6F23100F0F9FE1D9950
:1039A80088680B694A69C9691843104308431C9021
:1039B8001D980068006846F6F311CCF6FF710840C0
:1039C8001C9908431D99096808601D98006840689B
:1039D80020F440501D9A1168D268104348601D9821
:1039E80080691C901D98006840F60041C5F60001EA
:1039F800884204D01D98016A1C9808431C901D98A1
:103A0800006880684FF2FF41C1F2FF1108401C991D
:103A180008431D99096888601D980068C06A20F0ED
:103A28000F001D9A1168526A1043C8621D980068F9
:103A380041F20001C4F20101884240F03F8044F2A3
:103A48005440C5F60200006800F0380001461091A5
:103A580028282FD81099DFE801F0152D2D2D2D2DB0
:103A68002D2D192D2D2D2D2D2D2D1D2D2D2D2D2DA2
:103A78002D2D212D2D2D2D2D2D2D252D2D2D2D2D82
:103A88002D2D290001208DF86D0016E004208DF8F9
:103A98006D0012E008208DF86D000EE010208DF802
:103AA8006D000AE020208DF86D0006E040208DF8BA
:103AB8006D0002E080208DF86D004DE21D980068D1
:103AC80044F20041C4F2000188422CD144F254402F
:103AD800C5F60200006800F0070001460F910528AE
:103AE8001DD80F99DFE801F003070B0F131700200B
:103AF8008DF86D0016E004208DF86D0012E00820A6
:103B08008DF86D000EE010208DF86D000AE0202081
:103B18008DF86D0006E040208DF86D0002E08020F1
:103B28008DF86D0018E21D98006844F60001C4F293
:103B3800000188422CD144F25440C5F602000068C6
:103B480000F0070001460E9105281DD80E99DFE800
:103B580001F003070B0F131700208DF86D0016E016
:103B680004208DF86D0012E008208DF86D000EE03D
:103B780010208DF86D000AE020208DF86D0006E019
:103B880040208DF86D0002E080208DF86D00E3E1A3
:103B98001D98006844F60041C4F2000188422CD107
:103BA80044F25440C5F60200006800F007000146E0
:103BB8000D9105281DD80D99DFE801F003070B0FBB
:103BC800131700208DF86D0016E004208DF86D00A5
:103BD80012E008208DF86D000EE010208DF86D00C1
:103BE8000AE020208DF86D0006E040208DF86D0079
:103BF80002E080208DF86D00AEE11D98006845F266
:103C08000001C4F2000188422CD144F25440C5F6A8
:103C18000200006800F0070001460C9105281DD835
:103C28000C99DFE801F003070B0F131700208DF83C
:103C38006D0016E004208DF86D0012E008208DF864
:103C48006D000EE010208DF86D000AE020208DF840
:103C58006D0006E040208DF86D0002E080208DF8B0
:103C68006D0079E11D98006841F20041C4F201013C
:103C7800884240F03F8044F25440C5F60200006894
:103C880000F0380001460B9128282FD80B99DFE85F
:103C980001F0152D2D2D2D2D2D2D192D2D2D2D2DE1
:103CA8002D2D1D2D2D2D2D2D2D2D212D2D2D2D2D58
:103CB8002D2D252D2D2D2D2D2D2D290001208DF873
:103CC8006D0016E004208DF86D0012E008208DF8D4
:103CD8006D000EE010208DF86D000AE020208DF8B0
:103CE8006D0006E040208DF86D0002E080208DF820
:103CF8006D0031E11D98006847F60001C4F200012B
:103D080088422CD144F25440C5F60200006800F005
:103D1800070001460A9105281DD80A99DFE801F035
:103D280003070B0F131700208DF86D0016E0042011
:103D38008DF86D0012E008208DF86D000EE010205F
:103D48008DF86D000AE020208DF86D0006E0402017
:103D58008DF86D0002E080208DF86D00FCE01D9864
:103D6800006847F60041C4F2000188422CD144F2B1
:103D78005440C5F60200006800F0070001460991AA
:103D880005281DD80999DFE801F003070B0F131761
:103D980000208DF86D0016E004208DF86D0012E00B
:103DA80008208DF86D000EE010208DF86D000AE0F7
:103DB80020208DF86D0006E040208DF86D0002E0AF
:103DC80080208DF86D00C7E01D98006841F600015D
:103DD800C4F20101884240F03F8044F25440C5F6E5
:103DE8000200006800F038000146089128282FD802
:103DF8000899DFE801F0152D2D2D2D2D2D2D192DCC
:103E08002D2D2D2D2D2D1D2D2D2D2D2D2D2D212DF6
:103E18002D2D2D2D2D2D252D2D2D2D2D2D2D290003
:103E280001208DF86D0016E004208DF86D0012E079
:103E380008208DF86D000EE010208DF86D000AE066
:103E480020208DF86D0006E040208DF86D0002E01E
:103E580080208DF86D007FE01D98006841F60041D4
:103E6800C4F20101884240F03F8044F25440C5F654
:103E78000200006800F038000146079128282FD872
:103E88000799DFE801F0152D2D2D2D2D2D2D192D3C
:103E98002D2D2D2D2D2D1D2D2D2D2D2D2D2D212D66
:103EA8002D2D2D2D2D2D252D2D2D2D2D2D2D290073
:103EB80001208DF86D0016E004208DF86D0012E0E9
:103EC80008208DF86D000EE010208DF86D000AE0D6
:103ED80020208DF86D0006E040208DF86D0002E08E
:103EE80080208DF86D0037E01D98006840F600418D
:103EF800C5F6000188422CD144F25840C5F60200AC
:103F0800006800F007000146069105281DD80699AB
:103F1800DFE801F003070B0F131702208DF86D007F
:103F280016E004208DF86D0012E008208DF86D0071
:103F38000EE010208DF86D000AE020208DF86D004D
:103F480006E040208DF86D0002E080208DF86D00BD
:103F580002E080208DF86D001D98006840F6004151
:103F6800C5F60001884240F09E809DF86D0001462C
:103F7800059102280FD00598042810D00598082824
:103F880013D00598102816D0059820282FD005980A
:103F9800402832D035E004F002FB119036E015A835
:103FA800FEF70AFD1698119030E012A8FEF750FEB1
:103FB800139811902AE044F20040C5F60200006808
:103FC800C0F3401068B144F20040C5F60200006832
:103FD800C0F3C10149F20000C0F2D030C8401190CE
:103FE80004E049F20000C0F2D03011900EE040F633
:103FF8000010C0F23D00119008E04FF4004011900D
:1040080004E00020119001208DF867001198002825
:1040180048D011981D994A6A40F23041C0F6010112
:1040280031F81210B0FBF1F0189018981D994968F2
:1040380001EB4101884205D318981D994968B0EBF6
:10404800013F03D901208DF867002BE011981D99D5
:104058004A6803924A6A40F23041C0F6010131F8D9
:104068001220002304931946FFF75EFA039A049B73
:10407800090241EA1061000210EB520041F100010F
:10408800FFF752FA1A901A98B0F5407F07D31A989A
:10409800000D20B91A981D990968C86002E001202E
:1040A8008DF867002DE11D98C069B0F5004F40F00C
:1040B8009C809DF86D0001460291402800F25E80C8
:1040C8000299DFE801F021255B5B295B5B5B2F5BD5
:1040D8005B5B5B5B5B5B355B5B5B5B5B5B5B5B5B4E
:1040E8005B5B5B5B5B5B515B5B5B5B5B5B5B5B5B22
:1040F8005B5B5B5B5B5B5B5B5B5B5B5B5B5B5B5B08
:104108005B5B5B5B5B5B570003F071FF11903AE010
:1041180003F080FF119036E015A8FEF74DFC1698C5
:10412800119030E012A8FEF793FD139811902AE041
:1041380044F20040C5F602000068C0F3401068B1C0
:1041480044F20040C5F602000068C0F3C10149F21C
:104158000000C0F2D030C840119004E049F20000DD
:10416800C0F2D03011900EE040F60010C0F23D00D1
:10417800119008E04FF40040119004E000201190E5
:1041880001208DF86700119870B311981D9A516835
:10419800536A40F23042C0F6010232F81320B0FBF5
:1041A800F2F0400000EB5100B0FBF1F01A901A98C1
:1041B800102816D3BDF86A0098B91A9820F00F0095
:1041C800ADF86E001A9800F00E01BDF86E0040EAD6
:1041D8005100ADF86E00BDF86E001D990968C86001
:1041E80002E001208DF867008BE09DF86D00014624
:1041F8000191402800F25E800199DFE801F0212555
:104208005B5B295B5B5B2F5B5B5B5B5B5B5B355B7A
:104218005B5B5B5B5B5B5B5B5B5B5B5B5B5B515BF0
:104228005B5B5B5B5B5B5B5B5B5B5B5B5B5B5B5BD6
:104238005B5B5B5B5B5B5B5B5B5B5B5B5B5B570025
:1042480003F0D5FE11903AE003F0E4FE119036E059
:1042580015A8FEF7B1FB1698119030E012A8FEF7EA
:10426800F7FC139811902AE044F20040C5F60200CA
:104278000068C0F3401068B144F20040C5F602007F
:104288000068C0F3C10149F20000C0F2D030C84054
:10429800119004E049F20000C0F2D03011900EE015
:1042A80040F60010C0F23D00119008E04FF40040C5
:1042B800119004E00020119001208DF867001198FA
:1042C800F8B111981D9A5168536A40F23042C0F60D
:1042D800010232F81320B0FBF2F000EB5100B0FB02
:1042E800F1F01A901A98102808D3BDF86A0028B976
:1042F800BDF868001D990968C86002E001208DF8C2
:1043080067001D990120A1F86A001D99A1F86800AD
:104318001D99002048671D9988679DF867001EB0A1
:0243280080BD56
:10432A0080B586B044F2D840C5F60200016841F073
:10433A0001010160006800F00100059005980B205A
:10434A00019000220392114600F090FD019809F0B5
:10435A0062FA039A0C200290114600F087FD029837
:10436A0009F059FA039A0D200490114600F07EFDD7
:0A437A00049809F050FA06B080BD67
:1043840080B59AB000201990189017901690159047
:1043940044F2E040C5F60200016841F010010160FA
:1043A400006800F010001490149844F2E040C5F640
:1043B4000200016841F004010160006800F004009B
:1043C4001390139844F2E040C5F60200016841F0EE
:1043D40020010160006800F020001290129844F25D
:1043E400E040C5F60200016841F080010160006808
:1043F40000F080001190119844F2E040C5F60200EC
:10440400016841F001010160006800F001001090B2
:10441400109844F2E040C5F60200016841F0020140
:104424000160006800F002000F900F9844F2E04031
:10443400C5F60200016841F040010160006800F027
:1044440040000E900E9844F2E040C5F60200016868
:1044540041F008010160006800F008000D900D981B
:1044640041F20000C5F6020001904AF2C001009139
:10447400002209920AF0D8FE099A41F20040C5F6DA
:10448400020003904FF4004102910AF0CDFE099A14
:1044940041F60000C5F6020008904BF60361049152
:1044A4000AF0C2FE099A40F60040C5F602000690E2
:1044B4004FF4906105910AF0B7FE0198099940F212
:1044C4003F721592032207921692179115A90C9127
:1044D40002F0EEF8009B0198099A0C9915930123B8
:1044E4000A9316931792189202F0E2F8079A099821
:1044F4000C9942F23F0315931692179040F6000070
:10450400C5F6020002F0D4F80398079B099A0C99A7
:1045140047F6FF7CCDF854C01693179202F0C8F802
:10452400079A09980C9949F6FF6315931692179008
:104534000020C5F602000B9002F0BAF8079A099819
:104544000C994FF6FF7315931692179040F20040A2
:10455400C5F6020002F0ACF8DDF808C00398099A29
:104564000A9B0C99CDF854C016931792189202F036
:104574009FF8DDF810C00898099A0A9B0C99CDF8A9
:1045840054C016931792189202F092F8DDF814C0F2
:104594000698099A0A9B0C99CDF854C01693179261
:1045A400189202F085F80698099A0C994FF4005372
:1045B40015931692179202F07BF80698079B099AB6
:1045C4000C994CF27B0CCDF854C01693179202F060
:1045D4006FF8079B0898099A0C9944F2FC1CCDF8D3
:1045E40054C01693179202F063F8099B0A9A0B9829
:1045F4000C994FF4807CCDF854C01693179202F0B6
:0646040057F81AB080BD5A
:10460A0080B584B00020009040F68840C0F60100D2
:10461A0040F6A141C0F6010140F64652C0F6010239
:10462A0008F08EFD00F079F84EF61450CEF2000034
:10463A0000688003002800D519E0BFF34F8FBFF34D
:10464A006F8F4EF65071CEF2000100200860BFF362
:10465A004F8FBFF36F8F4EF61451CEF200010868E8
:10466A0040F400300860BFF34F8FBFF36F8F4EF6F0
:10467A001450CEF200000068C003002800D537E0CD
:10468A004EF68451CEF2000100200860BFF34F8F2E
:10469A004EF68050CEF20000006803900398C0F3F3
:1046AA004E3002900398C0F3C90001900299019814
:1046BA00800761F34D104EF66071CEF2000108607A
:1046CA000198411E01910028F0D10298411E0291E1
:1046DA000028E7D1BFF34F8F4EF61451CEF20001F6
:1046EA00086840F480300860BFF34F8FBFF36F8FC4
:1046FA0000F055FB08F0FBFDFFF73FFEFFF710FE49
:10470A0000F04AF800F08CF8FBF7DBFD00F053FAF2
:0A471A0000F0BBF908F039FFFEE7DC
:1047240080B586B00020019005900490039002901B
:1047340000F0EBFB019801218DF808108DF80900B9
:1047440003901F228DF8102087228DF811208DF8F8
:1047540012008DF813008DF814108DF815108DF8D3
:1047640016008DF8170002A809F09CF8042009F03F
:0647740081F806B080BDD3
:10477A0080B582B001900198006841F20041C4F20C
:0E478A000001884201D100F045FB02B080BD65
:0A47980082B00190009102B070475A
:1047A20080B582B040F28C40C2F20040019044F2E7
:1047B2000001C5F600010160002141607F22826094
:1047C200FF22C26001618161C161416103F0FDFEAE
:0A47D20008B108F0F8FD02B080BD48
:1047DC0080B5B0B02F906846B821FEF769FF2F98CE
:1047EC00006844F20001C5F60001884215D1002092
:1047FC0001904FF4800000904FF480702C9068462C
:10480C00FCF7CEFE08B108F0D9FD44F27041C5F6B4
:0E481C000201086840F40040086030B080BD22
:10482A0080B582B040F23C10C2F20040009043F2E0
:10483A000041C4F2010101604FF4800141604FF46C
:10484A00C02181600821C16000210191016141619B
:10485A004FF0005282614FF08052C26101624162A0
:10486A008162C1624FF0804242638163C163016425
:10487A0041648164C16401654165816504F097F909
:0A488A0008B108F09CFD02B080BDEB
:1048940080B590B00E900E980F280FD80E9937203F
:1048A4000090002200F0E5FA009808F0B7FF0E9897
:1048B40040F6E801C2F20041086003E001208DF8EF
:1048C4003F0048E044F2E840C5F60200016841F0C8
:1048D40020010160006800F020000190019806A802
:1048E40002A90AF029FD0B980490049818B903F062
:1048F40080FB059003E003F07CFB400005900598E5
:104904004DF68361C4F21B31A0FB01014FF0FF306F
:1049140000EB9140039040F2F430C2F2004041F2C7
:104924000041C4F20001016040F2E731C160039923
:10493400416000210161816004F0C9FC40B940F28A
:10494400F430C2F200400AF087FF8DF83F0002E025
:0E49540001208DF83F009DF83F0010B080BD9F
:104962004EF68851CEF20001086840F470000860EB
:1049720042F20000C5F20020006800F00F00062895
:1049820008D842F20001C5F200210868072262F34A
:104992000300086044F20041C5F60201086840F0D5
:1049A2000100086044F21042C5F6020200201060C5
:1049B20008684EF67F52CEF6F6221040086042F2A8
:1049C2000000C5F20020006800F00F00082808D39C
:1049D20042F20001C5F200210868072262F30300D7
:1049E200086044F21841C5F602010020086044F252
:1049F2001C41C5F60201086044F22041C5F60201DD
:104A0200086044F22842C5F6020240F20021C0F2D8
:104A12000221116044F22C42C5F602020021C0F2CA
:104A2200FF11116044F23042C5F6020240F28021C9
:104A3200C0F20111116044F23442C5F60202106064
:104A420044F23842C5F60202116044F23C42C5F615
:104A52000202106044F24042C5F60202116044F2C2
:104A62004441C5F60201086044F20042C5F6020262
:104A7200116821F48021116044F26041C5F60201FF
:104A8200086044F20001C5F2002143F2D20008603E
:024A920070476B
:104A940080B590B0002101910F910E910D910C9170
:104AA4000B910A910991089107910691059104913E
:104AB4000391029140F24040C2F2004040F20042B1
:104AC400C4F2000202600322426081604FF47A72F1
:104AD400C26001618021816104F0F9FB08B108F032
:104AE40071FC4FF480500C9040F24040C2F2004000
:104AF4000CA905F01AFF08B108F064FC40F240402C
:104B0400C2F2004004F0FDFD08B108F05BFC002097
:104B140009900B9040F24040C2F2004009A90BF00A
:104B2400A7F908B108F04EFC60200290C820039059
:104B3400022004900020069040F24040C2F200405F
:104B440002A90422FEF7D2F908B108F03BFC40F2B6
:0E4B54004040C2F2004000F002F810B080BDF8
:104B620080B588B0079000200690059004900390CD
:104B720002900798006840F20041C4F200018842A6
:104B82001BD144F2E040C5F60200016841F0040185
:104B92000160006800F004000190019880200290FA
:104BA20002200390002104910591069040F6000036
:0E4BB200C5F6020002A901F07CFD08B080BD2E
:104BC00080B582B040F2A800C2F20040019044F6E5
:104BD0000001C4F2000101604FF4E13141600021A5
:104BE0008160C16001610C2242618161C161016229
:104BF0004162282181624FF4004181634FF40051EA
:104C0000016406F090FF08B108F0DEFB40F2A80056
:104C1000C2F20040002107F008FF08B108F0D4FB01
:104C200040F2A800C2F20040002107F0BDFF08B129
:104C300008F0CAFB40F2A800C2F2004007F05CFE98
:0A4C400008B108F0C1FB02B080BD0E
:104C4A0080B5BAB0399000203890379036903590B8
:104C5A00349006A8B821FEF72CFD3998006844F66E
:104C6A000001C4F20001884240F0978000210791B8
:104C7A000220069019221092C8221192129008223C
:104C8A001392149015914FF4007216921791239073
:104C9A0006A8FCF786FC08B108F091FB44F2E8404C
:104CAA00C5F60200016841F480210160006800F441
:104CBA0080200590059844F2E040C5F6020001689C
:104CCA0041F008010160006800F0080004900498AF
:104CDA004FF4D8503490022035900020029036903C
:104CEA0037900720389040F60040C5F6020034A9F4
:104CFA0001F0DBFC029940F2B820C2F200400390B6
:104D0A002822C4F2020202602D2242608160C16040
:104D1A004FF48062026141618161C1610162416255
:104D2A0000F001F908B108F04AFB399840F2B821BD
:104D3A00C2F20041C0F880103998886340F24020DE
:104D4A00C2F2004001904021C4F2020101602E210A
:104D5A004160402181600021C1604FF4806202619C
:104D6A0041618161C1614FF400320262416200F027
:104D7A00DAF808B108F023FB399840F24021C2F270
:104D8A000041C167399888632720009000221146A4
:0E4D9A0000F06CF8009808F03EFD3AB080BDC5
:104DA80080B582B0032000F043F8FCF783FA44F2A0
:104DB8001842C5F602021168C1F3032340F6C25136
:104DC800C0F60101CB5C03F01F03D84000900098A7
:104DD800126802F00F02895C01F01F01C84040F61A
:104DE800F801C2F200410860009840F6FC01C2F2E6
:104DF800004108600F20FFF749FD18B101208DF828
:104E0800070004E008F060FB00208DF807009DF81B
:064E1800070002B080BD9E
:104E1E0040F60010C2F20040027840F2B041C2F2F9
:0A4E2E000041086810440860704756
:104E380080B582B00190019807280BD00198062808
:104E480008D00198052805D00198042802D00198B7
:104E5800032800D106E040F6A220C0F60100912107
:0E4E6800FFF796FC019808F07FFC02B080BDB9
:104E760080B586B0ADF816000491039203980F280A
:104E860000D806E040F6A220C0F60100A921FFF7EF
:104E960080FC04980F2800D806E040F6A220C0F651
:104EA6000100AA21FFF775FC08F07DFC0290BDF910
:104EB6001600019002980499039A08F07CFC0146BA
:0A4EC600019800F002F806B080BD6C
:104ED00082B0ADF806000091BDF90600002809D4A3
:104EE00000980001BDF906104EF20042CEF2000219
:104EF00088540AE000980001BDF8061001F00F0187
:0E4F00004EF61452CEF20002885402B07047F2
:104F0E00BFF35F8F4EF62451CEF20001086820F4F5
:104F1E00803008604EF69451CEF2000100200860F9
:024F2E007047CA
:104F300010B58EB00C9008F015FC0A900C9820B9B2
:104F400001208DF8370000F0F6BD0C9800681021A4
:104F5000C4F20201884200F0B8800C980068282151
:104F6000C4F20201884200F0B0800C980068402131
:104F7000C4F20201884200F0A8800C980068582111
:104F8000C4F20201884200F0A0800C9800687021F1
:104F9000C4F20201884200F098800C9800688821D1
:104FA000C4F20201884200F090800C980068A021B1
:104FB000C4F20201884200F088800C980068B82191
:104FC000C4F20201884200F080800C98006840F230
:104FD0001041C4F20201884277D00C98006840F278
:104FE0002841C4F2020188426FD00C98006840F258
:104FF0004041C4F20201884267D00C98006840F238
:105000005841C4F2020188425FD00C98006840F217
:105010007041C4F20201884257D00C98006840F2F7
:105020008841C4F2020188424FD00C98006840F2D7
:10503000A041C4F20201884247D00C98006840F2B7
:10504000B841C4F2020188423FD00C98006845F292
:105050000841C5F60201884237D00C98006845F235
:105060001C41C5F6020188422FD00C98006845F219
:105070003041C5F60201884227D00C98006845F2FD
:105080004441C5F6020188421FD00C98006845F2E1
:105090005841C5F60201884217D00C98006845F2C5
:1050A0006C41C5F6020188420FD00C98006845F2A9
:1050B0008041C5F60201884207D00C98006845F28D
:1050C0009441C5F60201884200D106E040F2C0706A
:1050D000C0F60100E621FFF75FFB0C98806838B14D
:1050E0000C988068402803D00C988068802800D1F4
:1050F00006E040F2C070C0F60100E721FFF74CFB6C
:105100000C98C068B0F5007F02D00C98C06800B958
:1051100006E040F2C070C0F60100E821FFF73CFB5A
:105120000C980069B0F5806F02D00C98006900B946
:1051300006E040F2C070C0F60100E921FFF72CFB49
:105140000C98406948B10C984069B0F5006F04D0E4
:105150000C984069B0F5805F00D106E040F2C07065
:10516000C0F60100EA21FFF717FB0C98806948B1EF
:105170000C988069B0F5005F04D00C988069B0F598
:10518000804F00D106E040F2C070C0F60100EB2174
:10519000FFF702FB0C98C06990B10C98C069B0F59C
:1051A000807F0DD00C98C069202809D00C98C06968
:1051B000B0F5802F04D00C98C069B0F5402F00D115
:1051C00006E040F2C070C0F60100EC21FFF7E4FAFF
:1051D0000C98006A70B10C98006AB0F5803F09D055
:1051E0000C98006AB0F5003F04D00C98006AB0F546
:1051F000403F00D106E040F2C070C0F60100ED2152
:10520000FFF7CAFA0C98016801201022C4F20202CA
:105210009142079000F091800C98016801202822AB
:10522000C4F202029142079000F087800C98016856
:1052300001204022C4F20202914207907DD00C98D6
:10524000016801205822C4F202029142079074D0F2
:105250000C98016801207022C4F20202914207906A
:105260006BD00C98016801208822C4F2020291429E
:10527000079062D00C9801680120A022C4F20202BB
:105280009142079059D00C9801680120B822C4F2CD
:1052900002029142079050D00C980168012040F220
:1052A0001042C4F202029142079046D00C98016865
:1052B000012040F22842C4F20202914207903CD001
:1052C0000C980168012040F24042C4F2020291426F
:1052D000079032D00C980168012040F25842C4F285
:1052E00002029142079028D00C980168012040F2F8
:1052F0007042C4F20202914207901ED00C980168DD
:10530000012040F28842C4F202029142079014D078
:105310000C980168012040F2A042C4F202029142BE
:1053200007900AD00C9800684FF64831CBF6FD7113
:105330000844B0FA80F0400907900798C007002899
:1053400000F0B1810C984068892800D806E040F24E
:10535000C070C0F60100F121FFF71EFA0C98406AF8
:1053600018B10C98406A042800D106E040F2C070E1
:10537000C0F60100F221FFF70FFA0C98406A0028EE
:105380004AD00C98806A58B10C98806A012807D0DE
:105390000C98806A022803D00C98806A032800D1F8
:1053A00006E040F2C070C0F60100F721FFF7F4F903
:1053B0000C98C06A70B10C98C06AB0F5000F09D0A3
:1053C0000C98C06AB0F1807F04D00C98C06AB0F12C
:1053D000C07F00D106E040F2C070C0F60100F821A5
:1053E000FFF7DAF90C98006B70B10C98006BB0F510
:1053F000001F09D00C98006BB0F5800F04D00C98FA
:10540000006BB0F5C00F00D106E040F2C070C0F6EE
:105410000100F921FFF7C0F90C99022081F835004D
:105420000C99002081F834000C9800681021C4F217
:105430000201884270D00C9800682821C4F2020151
:10544000884269D00C9800684021C4F20201884269
:1054500062D00C9800685821C4F2020188425BD0E7
:105460000C9800687021C4F20201884254D00C9854
:1054700000688821C4F2020188424DD00C9800686F
:10548000A021C4F20201884246D00C980068B821DD
:10549000C4F2020188423FD00C98006840F21041EB
:1054A000C4F20201884237D00C98006840F22841CB
:1054B000C4F2020188422FD00C98006840F24041AB
:1054C000C4F20201884227D00C98006840F258418B
:1054D000C4F2020188421FD00C98006840F270416B
:1054E000C4F20201884217D00C98006840F288414B
:1054F000C4F2020188420FD00C98006840F2A0412B
:10550000C4F20201884207D00C98006840F2B8410A
:10551000C4F20201884206D10C980168086820F0A4
:105520000100086005E00C980168086820F001009F
:1055300008600C9800680068C00788B108F012F98C
:105540000A99401A06280AD30C99202048650C991C
:10555000032081F8350001208DF83700EBE2E8E701
:105560000C98006800680B900B9848F23F01CFF64A
:10557000106108400B900C998868D1F80CC00B6939
:105580004A6940EA0C00184310438A691043CA690B
:105590001043096A01430B9808430B900C98406A2A
:1055A000042806D10C99C86A096B01430B9808437B
:1055B0000B900C984068292805D30C98416801206D
:1055C0002F2906902CD30C9840683F2805D30C98BF
:1055D000416801204329069022D30C98406847284F
:1055E00005D30C98416801204929069018D30C98DE
:1055F00040684F2805D30C98416801205329069034
:105600000ED30C98416800207429059006D30C989D
:1056100041680020782938BF012005900598069040
:105620000698C00718B10B9840F480100B900B98A7
:105630000C99096808600C98006840690B900B98F9
:1056400020F007000B900C98416A0B9808430B90D0
:105650000C98406A042815D10C98816A0B9808436D
:105660000B900C98C06A68B10C98FBF7C1FD48B16B
:105670000C99402048650C99012081F835008DF87F
:10568000370058E20B980C99096848610C9800F0B3
:1056900056FA09900C98C06D00F01F013F20884019
:1056A000099988601BE10C980168012045F20842C5
:1056B000C5F602029142049046D00C980168012080
:1056C00045F21C42C5F60202914204903CD00C986F
:1056D0000168012045F23042C5F602029142049071
:1056E00032D00C980168012045F24442C5F602020E
:1056F0009142049028D00C980168012045F258424C
:10570000C5F60202914204901ED00C980168012057
:1057100045F26C42C5F602029142049014D00C98F6
:105720000168012045F28042C5F6020291420490D0
:105730000AD00C9800684AF66C31CAF2FD71084430
:10574000B0FA80F0400904900498C007002800F0E7
:10575000BB800C980168012045F20842C5F60202A0
:105760009142039046D00C980168012045F21C42FA
:10577000C5F60202914203903CD00C9801680120CA
:1057800045F23042C5F602029142039032D00C98A5
:105790000168012045F24442C5F60202914203909D
:1057A00028D00C980168012045F25842C5F6020243
:1057B000914203901ED00C980168012045F26C4282
:1057C000C5F602029142039014D00C9801680120A2
:1057D00045F28042C5F60202914203900AD00C982D
:1057E00000684AF66C31CAF2FD710844B0FA80F0E4
:1057F000400903900398C00760B10C9840681128D5
:1058000000D807E040F2C070C0F6010040F26B1112
:10581000FEF7C2FF0C99022081F835000C99002098
:1058200081F834000C98006800680B900B986FF3B7
:1058300010100B900C988068402802D11020029024
:1058400007E00C9880688038B0FA80F04009800347
:10585000029002980C99CA680B69D1F814C0D1F86B
:1058600018E0CC694EEA040E4CEA0E0C43EA0C0335
:105870001A4340EAD200096A40EA11110B98084322
:105880000B900B980C99096808600C9908684AF607
:10589000F832CAF2FD7210444CF6CD42CCF6CC423E
:1058A000A0FB02026FF0030000EA9200C8650C98AA
:1058B00000F045F908900C98C06D00F01F01012020
:1058C0008840089948600AE00C99402048650C9986
:1058D000032081F8350001208DF837002BE10C986A
:1058E000016801201022C4F202029142019000F0EE
:1058F000EA800C98016801202822C4F20202914239
:10590000019000F0E0800C98016801204022C4F270
:1059100002029142019000F0D6800C9801680120AB
:105920005822C4F202029142019000F0CC800C98FF
:10593000016801207022C4F202029142019000F03D
:10594000C2800C98016801208822C4F202029142B0
:10595000019000F0B8800C9801680120A022C4F2E8
:1059600002029142019000F0AE800C980168012083
:10597000B822C4F202029142019000F0A4800C9877
:105980000168012040F21042C4F2020291420190EB
:1059900000F099800C980168012040F22842C4F27E
:1059A00002029142019000F08E800C980168012063
:1059B00040F24042C4F202029142019000F0838022
:1059C0000C980168012040F25842C4F20202914250
:1059D000019078D00C980168012040F27042C4F226
:1059E0000202914201906ED00C980168012040F2B1
:1059F0008842C4F202029142019064D00C9801687E
:105A0000012040F2A042C4F20202914201905AD019
:105A10000C980168012040F2B842C4F2020291429F
:105A2000019050D00C980168012045F20842C5F65B
:105A300002029142019046D00C980168012045F283
:105A40001C42C5F60202914201903CD00C980168BC
:105A5000012045F23042C5F602029142019032D057
:105A60000C980168012045F24442C5F602029142B9
:105A7000019028D00C980168012045F25842C5F6E3
:105A80000202914201901ED00C980168012045F25B
:105A90006C42C5F602029142019014D00C98016844
:105AA000012045F28042C5F60202914201900AD0DF
:105AB0000C9800684AF66C31CAF2FD710844B0FADD
:105AC00080F0400901900198C00758B30C9800F08D
:105AD00005F90C988068802802D10C990020486054
:105AE0000C990879096E08600C98416E806E4860C8
:105AF0000C98406878B10C98406808280BD80C982E
:105B000008F064F80C98C16E002008600C98016FD2
:105B1000406F486006E00C990020C8660C99086741
:105B20000C9948670C99002048650C9A012182F86D
:0E5B300035108DF837009DF837000EB010BD0F
:105B3E0083B002900298016801201022C4F2020282
:105B4E009142009000F09180029801680120282275
:105B5E00C4F202029142009000F087800298016820
:105B6E0001204022C4F20202914200907DD00298A0
:105B7E00016801205822C4F202029142009074D0B2
:105B8E000298016801207022C4F202029142009034
:105B9E006BD00298016801208822C4F20202914261
:105BAE00009062D0029801680120A022C4F2020285
:105BBE009142009059D0029801680120B822C4F297
:105BCE0002029142009050D002980168012040F2EA
:105BDE001042C4F202029142009046D0029801682F
:105BEE00012040F22842C4F20202914200903CD0C1
:105BFE0002980168012040F24042C4F20202914232
:105C0E00009032D002980168012040F25842C4F24E
:105C1E0002029142009028D002980168012040F2C1
:105C2E007042C4F20202914200901ED002980168A6
:105C3E00012040F28842C4F202029142009014D038
:105C4E0002980168012040F2A042C4F20202914281
:105C5E0000900AD0029800684FF64831CBF6FD71DD
:105C6E000844B0FA80F0400900900098C00728B3AD
:105C7E000298007810384AF6AB21CAF6AA21A0FB8A
:105C8E00011000090190019800F0070140F65250F2
:105C9E00C0F60100405C0299C8650198042806D33D
:105CAE0002990868042262F30900886505E00299EA
:105CBE00086840F2FF329043886504E00299086854
:0E5CCE0020F0FF0088650298806D03B07047DB
:105CDC0084B0039003980068019003980168012038
:105CEC0045F20842C5F602029142009046D0039854
:105CFC000168012045F21C42C5F602029142009057
:105D0C003CD003980168012045F23042C5F60202EE
:105D1C009142009032D003980168012045F2444230
:105D2C00C5F602029142009028D003980168012028
:105D3C0045F25842C5F60202914200901ED00398DB
:105D4C000168012045F26C42C5F6020291420090B6
:105D5C0014D003980168012045F28042C5F6020276
:105D6C00914200900AD0039800684AF66C31CAF24E
:105D7C00FD710844B0FA80F0400900900098C0070B
:105D8C0008B30398007808384CF6CD41CCF6CC41DA
:105D9C00A0FB011000090290029945F60000C5F61F
:105DAC00020000EB810003990866039945F6800018
:105DBC00C5F602004866029800F01F0101208840D9
:105DCC000399886631E00398007810384AF6AB21C5
:105DDC00CAF6AA21A0FB011000090290019840F21A
:105DEC00B841C4F20201884209D8019840F210412E
:105DFC00C4F20201884202D3029808300290029940
:105E0C0040F60000C4F2020000EB81000399086622
:105E1C00039940F68000C4F202004866029800F034
:0E5E2C001F01012088400399886604B070476A
:105E3A0080B58AB0089007F090FC0490089820B9C1
:105E4A0001208DF8270000F02CBC089890F8350046
:105E5A0002280BD00899802048650899002081F80B
:105E6A00340001208DF8270000F01BBC0898016857
:105E7A0001201022C4F202029142039000F09180A4
:105E8A000898016801202822C4F202029142039074
:105E9A0000F087800898016801204022C4F20202BB
:105EAA00914203907DD00898016801205822C4F2DB
:105EBA0002029142039074D008980168012070226E
:105ECA00C4F20202914203906BD008980168012043
:105EDA008822C4F202029142039062D008980168B3
:105EEA000120A022C4F202029142039059D00898DC
:105EFA0001680120B822C4F202029142039050D0F4
:105F0A0008980168012040F21042C4F2020291424C
:105F1A00039046D008980168012040F22842C4F252
:105F2A000202914203903CD008980168012040F295
:105F3A004042C4F202029142039032D008980168AA
:105F4A00012040F25842C4F202029142039028D042
:105F5A0008980168012040F27042C4F2020291429C
:105F6A0003901ED008980168012040F28842C4F2CA
:105F7A0002029142039014D008980168012040F26D
:105F8A00A042C4F20202914203900AD00898006823
:105F9A004FF64831CBF6FD710844B0FA80F040095B
:105FAA0003900398C00778B108980168086820F040
:105FBA001E00086008980168486920F0800048615E
:105FCA0008980068059008E008980168086820F0B9
:105FDA000E0008600898006805900898016801207A
:105FEA001022C4F202029142029000F0EA8008985C
:105FFA00016801202822C4F202029142029000F0B4
:10600A00E0800898016801204022C4F2020291420D
:10601A00029000F0D6800898016801205822C4F244
:10602A0002029142029000F0CC8008980168012097
:10603A007022C4F202029142029000F0C2800898D3
:10604A00016801208822C4F202029142029000F003
:10605A00B880089801680120A022C4F20202914285
:10606A00029000F0AE80089801680120B822C4F2BC
:10607A0002029142029000F0A4800898016801206F
:10608A0040F21042C4F202029142029000F099805A
:10609A0008980168012040F22842C4F202029142A3
:1060AA00029000F08E8008980168012040F2404278
:1060BA00C4F202029142029000F0838008980168BB
:1060CA00012040F25842C4F202029142029078D072
:1060DA0008980168012040F27042C4F2020291421B
:1060EA0002906ED008980168012040F28842C4F2FA
:1060FA0002029142029064D008980168012040F29D
:10610A00A042C4F20202914202905AD00898016851
:10611A00012040F2B842C4F202029142029050D0E9
:10612A0008980168012045F20842C5F60202914228
:10613A00029046D008980168012045F21C42C5F633
:10614A000202914202903CD008980168012045F26F
:10615A003042C5F602029142029032D00898016894
:10616A00012045F24442C5F602029142029028D02B
:10617A0008980168012045F25842C5F60202914288
:10618A0002901ED008980168012045F26C42C5F6BB
:10619A0002029142029014D008980168012045F247
:1061AA008042C5F60202914202900AD0089800681D
:1061BA004AF66C31CAF2FD710844B0FA80F040091F
:1061CA0002900298C00728B10898016E086820F466
:1061DA0080700860089800681021C4F202018842A1
:1061EA0070D0089800682821C4F20201884269D058
:1061FA00089800684021C4F20201884262D00898D7
:10620A0000685821C4F2020188425BD008980068ED
:10621A007021C4F20201884254D00898006888218B
:10622A00C4F2020188424DD008980068A021C4F245
:10623A000201884246D008980068B821C4F20201D7
:10624A0088423FD00898006840F21041C4F2020127
:10625A00884237D00898006840F22841C4F2020107
:10626A0088422FD00898006840F24041C4F20201E7
:10627A00884227D00898006840F25841C4F20201C7
:10628A0088421FD00898006840F27041C4F20201A7
:10629A00884217D00898006840F28841C4F2020187
:1062AA0088420FD00898006840F2A041C4F2020167
:1062BA00884207D00898006840F2B841C4F2020147
:1062CA00884206D108980168086820F00100086031
:1062DA0005E008980168086820F001000860059840
:1062EA000068C007A8B107F038FA0499401A0628CE
:1062FA000ED30899202048650899032081F83500B3
:10630A000899002081F8340001208DF82700C8E19F
:10631A00E5E70898016801201022C4F202029142BE
:10632A00019000F091800898016801202822C4F2A7
:10633A0002029142019000F08780089801680120CA
:10634A004022C4F20202914201907DD0089801686D
:10635A0001205822C4F202029142019074D0089896
:10636A00016801207022C4F20202914201906BD0AE
:10637A000898016801208822C4F202029142019021
:10638A0062D0089801680120A022C4F20202914258
:10639A00019059D0089801680120B822C4F202027B
:1063AA009142019050D008980168012040F21042B1
:1063BA00C4F202029142019046D008980168012075
:1063CA0040F22842C4F20202914201903CD008985D
:1063DA000168012040F24042C4F202029142019057
:1063EA0032D008980168012040F25842C4F20202F1
:1063FA009142019028D008980168012040F2704229
:10640A00C4F20202914201901ED00898016801204C
:10641A0040F28842C4F202029142019014D00898D4
:10642A000168012040F2A042C4F2020291420190A6
:10643A000AD0089800684FF64831CBF6FD71084437
:10644A00B0FA80F0400901900198C00758B1089845
:10645A00806D07900898C06D00F01F013F208840AA
:10646A00079988600AE00898806D06900898C06DC0
:10647A0000F01F01012088400699486008980168C9
:10648A0001201022C4F202029142009000F0EA8038
:10649A000898016801202822C4F202029142009061
:1064AA0000F0E0800898016801204022C4F202024C
:1064BA009142009000F0D680089801680120582285
:1064CA00C4F202029142009000F0CC800898016860
:1064DA0001207022C4F202029142009000F0C280B0
:1064EA000898016801208822C4F2020291420090B1
:1064FA0000F0B880089801680120A022C4F20202C4
:10650A009142009000F0AE80089801680120B822FC
:10651A00C4F202029142009000F0A4800898016837
:10652A00012040F21042C4F202029142009000F0AF
:10653A00998008980168012040F22842C4F20202B8
:10654A009142009000F08E8008980168012040F284
:10655A004042C4F202029142009000F083800898FF
:10656A000168012040F25842C4F2020291420090AE
:10657A0078D008980168012040F27042C4F2020201
:10658A00914200906ED008980168012040F288423A
:10659A00C4F202029142009064D008980168012076
:1065AA0040F2A042C4F20202914200905AD00898E6
:1065BA000168012040F2B842C4F2020291420090FE
:1065CA0050D008980168012045F20842C5F6020237
:1065DA009142009046D008980168012045F21C4279
:1065EA00C5F60202914200903CD008980168012049
:1065FA0045F23042C5F602029142009032D0089824
:10660A000168012045F24442C5F602029142009017
:10661A0028D008980168012045F25842C5F60202BE
:10662A00914200901ED008980168012045F26C4200
:10663A00C5F602029142009014D008980168012020
:10664A0045F28042C5F60202914200900AD00898AB
:10665A0000684AF66C31CAF2FD710844B0FA80F05B
:10666A00400900900098C00780B10898416E806E7A
:10667A0048600898C06E48B10898C16E086820F44E
:10668A00807008600898016F406F4860089901207F
:10669A0081F835000899002081F8340000208DF82F
:0A66AA0027009DF827000AB080BD0C
:1066B40080B590B00F900E9100200D908020C5F60B
:1066C40000000A900F980021C5F6020188423ED0CE
:1066D4000F9840F20041C5F60201884237D00F9866
:1066E40040F60001C5F60201884230D00F9840F60A
:1066F4000041C5F60201884229D00F9841F20001F9
:10670400C5F60201884222D00F9841F20041C5F635
:10671400020188421BD00F9841F60001C5F6020120
:10672400884214D00F9841F60041C5F60201884210
:106734000DD00F9842F20041C5F60201884206D0FE
:106744000F9842F60001C5F60201884200D106E026
:1067540040F65A50C0F60100B321FEF71BF80E981C
:10676400008818B10E98408800B906E040F65A50E7
:10677400C0F60100B421FEF70DF80E98406888B306
:106784000E98406801282DD00E984068112829D011
:106794000E984068022825D00E984068122821D00F
:1067A4000E984068B0F5881F1CD00E984068B0F56C
:1067B400041F17D00E984068B0F5441F12D00E98ED
:1067C4004068B0F5901F0DD00E984068B0F5081FD2
:1067D40008D00E984068B0F5481F03D00E98406862
:1067E400032800D106E040F65A50C0F60100B52156
:1067F400FDF7D0FF0E9800680D99C840002800F0FE
:106804001E820E9800680D9A0121914008400C9058
:106814000C98002800F00F820E98406800F00300E6
:10682400012805D00E98406800F00300022844D1E6
:106834000E98C06858B10E98C068012807D00E9809
:10684400C068022803D00E98C068032800D106E06F
:1068540040F65A50C0F60100C421FDF79BFF0F9883
:1068640080680B900D984100032000FA01F10B9809
:1068740088430B900E98C0680D99490000FA01F105
:106884000B9808430B900B980F9988600F984068F9
:106894000B900D99012000FA01F10B9888430B909D
:1068A4000E984068C0F300100D9900FA01F10B989E
:1068B40008430B900B980F9948600E98406800F0BD
:1068C4000300032829D00E98806838B10E98806898
:1068D400012803D00E988068022800D106E040F613
:1068E4005A50C0F60100D621FDF754FF0F98C06836
:1068F4000B900D984100032000FA01F10B98884396
:106904000B900E9880680D99490000FA01F10B98DC
:1069140008430B900B980F99C8600E98406800F0DC
:10692400030002287DD10F980021C5F60201884298
:106934003ED00F9840F20041C5F60201884237D09C
:106944000F9840F60001C5F60201884230D00F9836
:1069540040F60041C5F60201884229D00F9841F261
:106964000001C5F60201884222D00F9841F200418D
:10697400C5F6020188421BD00F9841F60001C5F606
:106984000201884214D00F9841F60041C5F6020175
:1069940088420DD00F9842F20041C5F602018842A8
:1069A40006D00F9842F60001C5F60201884200D1D4
:1069B40006E040F65A50C0F60100E321FDF7EAFE76
:1069C4000E9800690F2800D806E040F65A50C0F629
:1069D4000100E421FDF7DEFE0F980D996FF003022C
:1069E40002EA51010844006A0B900D9800F0070078
:1069F40081000F2000FA01F10B9888430B900E9848
:106A040000690D9901F00701890000FA01F10B9862
:106A140008430B900B980F990D9B02EA5302114403
:106A240008620F9800680B900D984100032000FA4B
:106A340001F10B9888430B900E98406800F0030016
:106A44000D99490000FA01F10B9808430B900B983B
:106A54000F9908600E9880798007002800F0EB8079
:106A640044F2F440C5F60200016841F002010160FD
:106A7400006800F00200099009980D9820F00300C6
:106A840040F20841C5F6000140580B900D9800F003
:106A9400030081000F2000FA01F10B9888430B904A
:106AA4000F980021C5F60201884202D10020089007
:106AB4005DE00F9840F20041C5F60201884202D120
:106AC4000120079051E00F9840F60001C5F602013D
:106AD400884202D10220069045E00F9840F600411A
:106AE400C5F60201884202D10320059039E00F98CF
:106AF40041F20001C5F60201884202D1042004904B
:106B04002DE00F9841F20041C5F60201884202D1FE
:106B14000520039021E00F9841F60001C5F602011B
:106B2400884202D10620029015E00F9841F60041F8
:106B3400C5F60201884202D10720019009E00F99AD
:106B440042F20042C5F602020A20914208BF09201F
:106B5400019001980290029803900398049004987D
:106B6400059005980690069807900798089008984D
:106B74000D9901F00301890000FA01F10B98084313
:106B84000B900B980D9921F0030140F20842C5F6D1
:106B9400000288504FF0B04000680B900C990B989D
:106BA40088430B900E988079C006002803D50C9971
:106BB4000B9808430B900B984FF0B04108600420E9
:106BC400C5F6000000680B900C990B9888430B9055
:106BD4000E9880798006002803D50C990B980843F9
:106BE4000B900B980421C5F6000108600A984068D0
:106BF4000B900C990B9888430B900E988079800722
:106C0400002803D50C990B9808430B900B980A990C
:106C140048600A9800680B900C990B9888430B9075
:106C24000E988079C00718B10C990B9808430B9003
:106C34000B980A9908600D9801300D90DAE510B0B0
:026C440080BD11
:106C460044F60001C5F60201086840F48070086049
:026C5600704785
:106C580080B58CB00A900A9820B901208DF82F00D1
:106C680000F0C1BD0A98006800B30A980078C00710
:106C7800E0B90A98006800F00200022816D00A98C5
:106C8800006800F01000102810D00A98006800F082
:106C9800080008280AD00A98006800F004000428B0
:106CA80004D00A9800788006002800D507E040F64E
:106CB8002700C0F6010040F2A111FDF769FD0A980E
:106CC8000078C007002800F0AE800A98406848B1F4
:106CD8000A984068B0F5803F04D00A984068B0F53B
:106CE800A02F00D107E040F62700C0F601004FF4BE
:106CF800D371FDF74DFD44F21040C5F6020000685F
:106D080000F03800069044F22840C5F602000068FA
:106D180005900698102807D00698182815D10598C8
:106D280000F00300022810D144F20040C5F602002A
:106D38000068C0F3404038B10A98406820B9012083
:106D48008DF82F0000F04FBD6DE00A984068B0F54F
:106D5800803F08D144F20041C5F60201086840F4BA
:106D6800803008602DE00A98406860B944F200411C
:106D7800C5F60201086820F480300860086820F42D
:106D8800802008601DE00A984068B0F5A02F0CD15B
:106D980044F20041C5F60201086840F4802008600A
:106DA800086840F4803008600BE044F20041C5F602
:106DB8000201086820F480300860086820F4802008
:106DC80008600A984068B8B106F0C8FC099044F217
:106DD8000040C5F602000068C0F3404058B906F00C
:106DE800BDFC0999401A652804D303208DF82F00AB
:106DF80000F0F9BCEBE716E006F0B0FC099044F2AD
:106E08000040C5F602000068C0F3404058B106F0E3
:106E1800A5FC0999401A652804D303208DF82F0092
:106E280000F0E1BCEBE70A9800788007002840F101
:106E3800D5800A98C06898B10A98C06801280FD010
:106E48000A98C06801280BD00A98C068092807D09A
:106E58000A98C068112803D00A98C068192800D178
:106E680007E040F62700C0F601004FF4ED71FDF78A
:106E78008FFC0A9800697F2800D807E040F62700B1
:106E8800C0F6010040F2DB11FDF782FC44F210402D
:106E9800C5F60200006800F03800049044F228406B
:106EA800C5F6020000680390049838B104981828C1
:106EB80043D19DF80C00800700283ED144F20040E1
:106EC800C5F602000068C0F3800038B10A98C068AF
:106ED80020B901208DF82F0000F085BC44F2004154
:106EE800C5F60201086820F019000A9AD268104312
:106EF800086006F033FC099044F20040C5F6020031
:106F08000068C0F3800058B906F028FC0999401AB7
:106F1800032804D303208DF82F0000F064BCEBE7AE
:106F280044F20441C5F60201086820F0FE400A9ABE
:106F3800126940EA0260086050E00A98C06870B3BD
:106F480044F20041C5F60201086820F019000A9AC7
:106F5800D2681043086006F001FC099044F2004032
:106F6800C5F602000068C0F3800058B906F0F6FBC9
:106F78000999401A032804D303208DF82F0000F044
:106F880032BCEBE744F20441C5F60201086820F080
:106F9800FE400A9A126940EA026008601EE044F264
:106FA8000041C5F60201086820F00100086006F0FB
:106FB800D5FB099044F20040C5F602000068C0F312
:106FC800800058B106F0CAFB0999401A032804D377
:106FD80003208DF82F0000F006BCEBE70A98007834
:106FE800C006002840F19F800A98C06918B10A9825
:106FF800C069802800D107E040F62700C0F60100EC
:1070080040F22B21FDF7C4FB0A98006A3F2800D8FC
:1070180007E040F62700C0F601004FF40B71FDF7BA
:10702800B7FB44F21040C5F60200006800F03800D3
:10703800029044F22840C5F60200006801900298C8
:10704800082807D00298182821D1019800F00300D9
:1070580001281CD144F20040C5F602000068C0F3C4
:10706800002038B10A98C069802803D001208DF823
:107078002F00B8E344F20C41C5F60201086820F07D
:107088007C500A9A126A40EA026008604BE00A984B
:10709800C06950B344F20041C5F60201086840F0E7
:1070A8008000086006F05AFB099044F20040C5F6DB
:1070B80002000068C0F3002050B906F04FFB0999A0
:1070C800401A032803D303208DF82F008BE3ECE745
:1070D80044F20C41C5F60201086820F07C500A9A77
:1070E800126A40EA026008601DE044F20041C5F6F9
:1070F8000201086820F08000086006F02FFB099064
:1071080044F20040C5F602000068C0F3002050B108
:1071180006F024FB0999401A032803D303208DF8AD
:107128002F0060E3ECE70A980078000700284FD5A5
:107138000A98406918B10A984069012800D107E007
:1071480040F62700C0F6010040F26D21FDF720FB54
:107158000A984069F0B144F27441C5F60201086822
:1071680040F00100086006F0F9FA099044F2744012
:10717800C5F602000068C0F3400050B906F0EEFA08
:107188000999401A032803D303208DF82F002AE316
:10719800ECE71DE044F27441C5F60201086820F0EE
:1071A8000100086006F0DAFA099044F27440C5F666
:1071B80002000068C0F3400050B106F0CFFA099908
:1071C800401A032803D303208DF82F000BE3ECE7C4
:1071D8000A980078800600284FD50A98806918B167
:1071E8000A988069012800D107E040F62700C0F618
:1071F80001004FF42671FDF7CBFA0A988069F0B1C7
:1072080044F20041C5F60201086840F48050086065
:1072180006F0A4FA099044F20040C5F6020000689E
:10722800C0F3403050B906F099FA0999401A03287A
:1072380003D303208DF82F00D5E2ECE71DE044F2DC
:107248000041C5F60201086820F48050086006F085
:1072580085FA099044F20040C5F602000068C0F3C0
:10726800403050B106F07AFA0999401A032803D33E
:1072780003208DF82F00B6E2ECE70A980078400763
:10728800002840F1A0800A98806838B10A98806880
:10729800012803D00A988068052800D107E040F645
:1072A8002700C0F6010040F2C221FDF771FA44F64A
:1072B8000001C5F60201086840F48070086006F015
:1072C8004DFA099044F60000C5F602000068C005B2
:1072D80000280AD406F042FA0999401A652803D30F
:1072E80003208DF82F007EE2ECE70A9880680128D9
:1072F80008D144F27041C5F60201086840F0010067
:1073080008602CE00A98806860B944F27041C5F6BC
:107318000201086820F001000860086820F00400F5
:1073280008601CE00A98806805280CD144F2704176
:10733800C5F60201086840F004000860086840F0DB
:10734800010008600BE044F27041C5F602010868CC
:1073580020F001000860086820F0040008600A981E
:107368008068C0B106F0FAF9099044F27040C5F699
:1073780002000068C0F3400060B906F0EFF909990F
:10738800401A41F28931884203D303208DF82F0037
:1073980029E2EAE717E006F0E1F9099044F27040C3
:1073A800C5F602000068C0F3400060B106F0D6F9E7
:1073B8000999401A41F28931884203D303208DF894
:1073C8002F0010E2EAE70A98406A38B10A98406A42
:1073D800012803D00A98406A022800D107E040F645
:1073E8002700C0F601004FF43D71FDF7D1F90A9866
:1073F800406A002800F0F48144F21040C5F602000B
:10740800006800F03800182800F068810A98406A7F
:10741800022840F044810A98806A01280AD00A9814
:10742800806A38B10A98806A032803D00A98806A6B
:10743800022800D107E040F62700C0F6010040F21C
:10744800FD21FDF7A5F90A98006C58B10A98006C5F
:10745800042807D00A98006C082803D00A98006C02
:107468000C2800D107E040F62700C0F6010040F2E2
:10747800FE21FDF78DF90A98406C18B10A98406C06
:10748800022800D107E040F62700C0F6010040F2CC
:10749800FF21FDF77DF90A98C06A20B10A98C06AF1
:1074A8003F2800D807E040F62700C0F601004FF457
:1074B8004071FDF76DF90A98006B042805D30A9806
:1074C800006BB0F5007F00D807E040F62700C0F653
:1074D800010040F20131FDF75BF90A98406B20B1D9
:1074E8000A98406B802800D807E040F62700C0F6CD
:1074F800010040F20231FDF74BF90A98806B20B188
:107508000A98806B802800D807E040F62700C0F66C
:10751800010040F20331FDF73BF90A98C06B20B136
:107528000A98C06B802800D807E040F62700C0F60C
:1075380001004FF44171FDF72BF90A98806C400B5C
:1075480000B907E040F62700C0F6010040F2053117
:10755800FDF71EF944F20041C5F60201086820F063
:107568008070086006F0FAF8099044F20040C5F609
:1075780002000068C0F3406050B106F0EFF80999C6
:10758800401A032803D303208DF82F002BE1ECE7E2
:1075980044F22841C5F60201086840F2F3329043EC
:1075A8000A9B9A6ADB6A42EA0312104308600A9946
:1075B800086BD1F834C08B6BCA6B01386FF35F204E
:1075C8004FF60061CFF6FF7101EB4C2189B20844F8
:1075D8000021CFF6FF7101EB034101F4FE010844DD
:1075E8004FF07F4101EB026101F0FE41084444F293
:1075F8003041C5F60201086044F22C41C5F602018B
:107608000091086820F00100086044F23442C5F691
:10761800020210684FF6F87398430A9B9B6C40EA85
:10762800C3001060086820F00C000A9A126C10431E
:107638000860086820F002000A9A526C104308603B
:10764800086840F480300860086840F4003008603A
:10765800086840F480200860086840F0010008606D
:1076680044F20041C5F60201086840F080700860E5
:1076780006F074F8099044F20040C5F6020000686C
:10768800C0F3406050B906F069F80999401A032818
:1076980003D303208DF82F00A5E0ECE71DE044F2AA
:1076A8000041C5F60201086820F08070086006F005
:1076B80055F8099044F20040C5F602000068C0F38E
:1076C800406050B106F04AF80999401A032803D3DC
:1076D80003208DF82F0086E0ECE781E044F2284093
:1076E800C5F602000068089044F23040C5F6020072
:1076F800006807900A98406A01282DD0089800F081
:1077080003000A99896A884226D10898C0F30511AE
:107718000A98C06A88421FD107986FF35F200A99B8
:10772800096B0139884217D1BDF81C00410A0A9833
:10773800406B013888420FD10798C0F306410A9878
:10774800806B0138884207D10798C0F306610A9810
:10775800C06B0138884203D001208DF82F0042E029
:1077680044F23440C5F60200006880B2C0080890B0
:107778000A98806C0899884232D00A98806C400B2D
:1077880000B907E040F62700C0F601004FF45B712E
:10779800FCF7FEFF44F22C41C5F60201086820F010
:1077A8000100086005F0DAFF099005F0D7FF099994
:1077B800401A00B9F9E744F23441C5F602010868F5
:1077C8004FF6F87290430A9A926C40EAC200086039
:1077D80044F22C41C5F60201086840F00100086037
:0E77E80000208DF82F009DF82F000CB080BD02
:1077F60080B586B004900391049818B901208DF8DD
:107806001700C6E30498006820B1049800683F2872
:1078160000D807E040F62700C0F6010040F2A73185
:10782600FCF7B7FF039860B30398012829D00398A3
:10783600022826D00398032823D00398042820D0B2
:10784600039805281DD0039806281AD00398072800
:1078560017D00398082814D00398092811D0039844
:107866000A280ED003980B280BD003980C2808D0B2
:1078760003980D2805D003980E2802D003980F28E8
:1078860000D107E040F62700C0F601004FF46A7108
:10789600FCF77FFF039842F20001C5F20021096858
:1078A60001F00F01884213D942F20000C5F2002010
:1078B600016821F00F01039A11430160006800F08E
:1078C6000F000399884203D001208DF8170060E36A
:1078D600049800784007002831D50498006944F2DE
:1078E6001841C5F60201096801F07001884226D9DF
:1078F6000498006978B10498006940280BD0049870
:107906000069502807D004980069602803D00498BD
:107916000069702800D107E040F62700C0F6010094
:107926004FF47171FCF735FF44F21841C5F60201B8
:10793600086820F07000049A1269104308600498E1
:1079460000780007002831D50498406944F21C41AC
:10795600C5F60201096801F07001884226D904982B
:10796600406978B10498406940280BD00498406972
:10797600502807D004984069602803D004984069CD
:10798600702800D107E040F62700C0F6010040F25B
:10799600D631FCF7FEFE44F21C41C5F6020108682A
:1079A60020F07000049A5269104308600498007829
:1079B600C006002835D50498806944F21C41C5F6F6
:1079C6000201096801F4E06188422AD904988069B5
:1079D60098B104988069B0F5806F0ED004988069DC
:1079E600B0F5A06F09D004988069B0F5C06F04D0D7
:1079F60004988069B0F5E06F00D107E040F62700F3
:107A0600C0F6010040F2E731FCF7C3FE44F21C4128
:107A1600C5F60201086820F4E060049A92691043F2
:107A26000860049800788006002831D50498C0695B
:107A360044F22041C5F60201096801F0700188424E
:107A460026D90498C06978B10498C06940280BD03B
:107A56000498C069502807D00498C069602803D0EC
:107A66000498C069702800D107E040F62700C0F6E8
:107A7600010040F2F931FCF78CFE44F22041C5F6D4
:107A86000201086820F07000049AD2691043086069
:107A9600049800788007002841D50498C06844F20D
:107AA6001841C5F60201096801F00F01884236D96E
:107AB6000498C068F8B10498C06808281BD00498D8
:107AC600C068092817D00498C0680A2813D00498FB
:107AD600C0680B280FD00498C0680C280BD00498F7
:107AE600C0680D2807D00498C0680E2803D00498F3
:107AF600C0680F2800D107E040F62700C0F6010055
:107B060040F20C41FCF745FE44F21841C5F602016D
:107B1600086820F00F00049AD268104308600498A1
:107B26000078C007002800F0BD800498806838B34C
:107B360004988068B0F5006F22D004988068B0F58C
:107B4600106F1DD004988068B0F5206F18D0049887
:107B56008068B0F5306F13D004988068B0F5406F38
:107B66000ED004988068B0F5506F09D004988068EC
:107B7600B0F5606F04D004988068B0F5706F00D1DE
:107B860007E040F62700C0F6010040F21C41FCF772
:107B960000FE0498406801280AD00498406838B16D
:107BA60004984068022803D004984068032800D14E
:107BB60007E040F62700C0F6010040F21D41FCF741
:107BC600E8FD44F21841C5F60201086820F4706029
:107BD600049A9268104308600498406802280CD101
:107BE60044F20040C5F602000068C0F3404018B9F0
:107BF60001208DF81700CCE12DE004984068032899
:107C06000CD144F20040C5F602000068C0F34060A3
:107C160018B901208DF81700BBE11CE004984068F4
:107C260001280CD144F20040C5F602000068C0F3FA
:107C3600002018B901208DF81700AAE10BE044F2E4
:107C46000040C5F602000068C0F3800018B90120A4
:107C56008DF817009DE144F21041C5F6020108684F
:107C660020F00700049A52681043086005F077FD7B
:107C7600019044F21040C5F60200006800F038009A
:107C860004994968C90088420CD005F068FD01993D
:107C9600401A41F28931884203D303208DF8170038
:107CA60077E1E6E7049800788007002841D5049834
:107CB600C06844F21841C5F60201096801F00F01D7
:107CC600884236D20498C068F8B10498C06808287B
:107CD6001BD00498C068092817D00498C0680A28E1
:107CE60013D00498C0680B280FD00498C0680C28DD
:107CF6000BD00498C0680D2807D00498C0680E28D9
:107D060003D00498C0680F2800D107E040F627008A
:107D1600C0F6010040F25E41FCF73BFD44F218411B
:107D2600C5F60201086820F00F00049AD2681043D5
:107D36000860039842F20001C5F20021096801F0CB
:107D46000F01884213D242F20000C5F200200168FA
:107D560021F00F01039A11430160006800F00F0043
:107D66000399884203D001208DF8170011E1049889
:107D760000784007002831D50498006944F218417C
:107D8600C5F60201096801F07001884226D20498FE
:107D9600006978B10498006940280BD004980069FE
:107DA600502807D004980069602803D00498006919
:107DB600702800D107E040F62700C0F6010040F227
:107DC6007F41FCF7E6FC44F21841C5F6020108685B
:107DD60020F07000049A1269104308600498007835
:107DE6000007002831D50498406944F21C41C5F6C5
:107DF6000201096801F07001884226D204984069A0
:107E060078B10498406940280BD0049840695028FE
:107E160007D004984069602803D004984069702808
:107E260000D107E040F62700C0F6010040F291417C
:107E3600FCF7AFFC44F21C41C5F60201086820F0CD
:107E46007000049A52691043086004980078C006CE
:107E5600002835D50498806944F21C41C5F6020114
:107E6600096801F4E06188422AD20498806998B1D1
:107E760004988069B0F5806F0ED004988069B0F5DB
:107E8600A06F09D004988069B0F5C06F04D004983B
:107E96008069B0F5E06F00D107E040F62700C0F634
:107EA600010040F2A341FCF774FC44F21C41C5F604
:107EB6000201086820F4E060049A926910430860A1
:107EC600049800788006002831D50498C06944F2E9
:107ED6002041C5F60201096801F07001884226D2E8
:107EE6000498C06978B10498C06940280BD00498FA
:107EF600C069502807D00498C069602803D0049848
:107F0600C069702800D107E040F62700C0F60100DE
:107F160040F2B541FCF73DFC44F22041C5F60201B2
:107F2600086820F07000049AD26910430860F9F7D7
:107F3600C2F944F21842C5F602021168C1F30323DE
:107F460040F6C251C0F60101CB5C03F01F03D840D6
:107F560000900098126802F00F02895C01F01F0180
:107F6600C84040F6F801C2F200410860009840F6A9
:107F7600FC01C2F20041086040F6E800C2F200408F
:107F86000068FCF784FC8DF80B009DF80B008DF85B
:0A7F960017009DF8170006B080BD2B
:107FA00080B582B0F9F78AF944F21842C5F60202A8
:107FB0001168C1F3032340F6C251C0F60101CB5C46
:107FC00003F01F03D84001900198126802F00F02DD
:107FD000895C01F01F0120FA01F140F6F800C2F2BD
:107FE00000400160019940F6FC02C2F200421160BB
:067FF000006802B080BD34
:107FF60080B5FFF7D2FF44F21C41C5F602010968BD
:10800600C1F3021240F6C251C0F60101895C01F0CB
:068016001F01C84080BDFF
:10801C0080B5FFF7BFFF44F21C41C5F602010968A9
:10802C00C1F3022240F6C251C0F60101895C01F095
:06803C001F01C84080BDD9
:1080420080B586B00490039100208DF80700049853
:10805200006820B1049800683F2800D807E040F685
:108062007630C0F6010040F67261FCF794FB04988A
:108072004068042805D304984068B0F5007F00D812
:1080820007E040F67630C0F6010040F67361FCF777
:1080920082FB0498806820B104988068802800D808
:1080A20007E040F67630C0F6010040F67461FCF756
:1080B20072FB0498006920B104980069802800D8F6
:1080C20007E040F67630C0F6010040F67561FCF735
:1080D20062FB0498C06820B10498C068802800D868
:1080E20007E040F67630C0F6010040F67661FCF714
:1080F20052FB0498406958B104984069402807D05F
:1081020004984069802803D004984069C02800D1AF
:1081120007E040F67630C0F6010040F67761FCF7E2
:108122003AFB0498806918B104988069202800D12C
:1081320007E040F67630C0F6010040F67861FCF7C1
:108142002AFB0498C069400B00B907E040F676307C
:10815200C0F6010040F67961FCF71DFB44F22840AD
:10816200C5F60200006800F00300032803D10120D5
:108172008DF81700B7E044F20041C5F60201086825
:1081820020F08060086005F0ECFA029044F20040B2
:10819200C5F602000068C0F3C06050B105F0E1FA14
:1081A2000299401A032803D303208DF817009AE09E
:1081B200ECE744F22841C5F60201086820F47C305D
:1081C200049A126840EA0230086004994868D1F8BB
:1081D20008C0CB680A6901386FF35F204FF600616F
:1081E200CFF6FF7101EB4C2189B208440021CFF692
:1081F200FF7101EB034101F4FE0108444FF07F419E
:1082020001EB026101F0FE41084444F23841C5F637
:108212000201086044F22C41C5F60201009108688F
:1082220020F0C000049A526910430860086820F0E8
:108232002000049A926910430860086820F0100038
:10824200086044F23C42C5F6020210684FF6F87329
:108252009843049BDB6940EAC3001060086840F061
:1082620010000860039840B944F22C41C5F602019F
:10827200086840F40020086013E00398012808D140
:1082820044F22C41C5F60201086840F480100860EF
:1082920007E044F22C41C5F60201086840F40010E0
:1082A200086044F20041C5F60201086840F08060AF
:1082B200086005F056FA029044F20040C5F602004A
:1082C2000068C0F3C06050B905F04BFA0299401A39
:1082D200032803D303208DF8170004E0ECE79DF890
:0E82E20007008DF817009DF8170006B080BD4C
:1082F00080B586B00490039100208DF807000498A3
:10830000006820B1049800683F2800D807E040F6D4
:108310007630C0F6010040F6DA61FCF73DFA0498C9
:108320004068042805D304984068B0F5007F00D861
:1083300007E040F67630C0F6010040F6DB61FCF75E
:108340002BFA0498806820B104988068802800D8AF
:1083500007E040F67630C0F6010040F6DC61FCF73D
:108360001BFA0498006920B104980069802800D89D
:1083700007E040F67630C0F6010040F6DD61FCF71C
:108380000BFA0498C06820B10498C068802800D80F
:1083900007E040F67630C0F6010040F6DE61FCF7FB
:1083A000FBF90498406970B104984069B0F5806F9A
:1083B00009D004984069B0F5006F04D00498406972
:1083C000B0F5406F00D107E040F67630C0F601000E
:1083D00040F6DF61FCF7E0F90498806920B1049869
:1083E0008069B0F5007F00D107E040F67630C0F636
:1083F00001004FF46E61FCF7CFF90498C069400B9F
:1084000000B907E040F67630C0F6010040F6E161C1
:10841000FCF7C2F944F22840C5F60200006800F0FB
:108420000300032803D101208DF81700B7E044F2C0
:108430000041C5F60201086820F08050086005F090
:1084400091F9029044F20040C5F602000068C0F3C2
:10845000407050B105F086F90299401A032803D301
:1084600003208DF817009AE0ECE744F22841C5F6A6
:108470000201086820F07C70049A126840EA0250F9
:10848000086004994868D1F808C0CB680A690138C7
:108490006FF35F204FF60061CFF6FF7101EB4C21C7
:1084A00089B208440021CFF6FF7101EB034101F4CA
:1084B000FE0108444FF07F4101EB026101F0FE41F3
:1084C000084444F24041C5F60201086044F22C41E0
:1084D000C5F602010091086820F44060049A5269D0
:1084E00010430860086820F40070049A92691043F1
:1084F0000860086820F48070086044F24442C5F6C1
:10850000020210684FF6F8739843049BDB6940EA57
:10851000C3001060086840F480700860039840B998
:1085200044F22C41C5F60201086840F4800008605E
:1085300013E00398012808D144F22C41C5F602014A
:10854000086840F40000086007E044F22C41C5F6DA
:108550000201086840F08070086044F20041C5F6EE
:108560000201086840F08050086005F0FBF80290B6
:1085700044F20040C5F602000068C0F3407050B9F4
:1085800005F0F0F80299401A032803D303208DF870
:10859000170004E0ECE79DF807008DF817009DF840
:0685A000170006B080BDCB
:1085A60080B5FFF7FAFC44F22041C5F602010968DE
:1085B600C1F3021240F6C251C0F60101895C01F016
:0685C6001F01C84080BD4A
:1085CC0080B582B0019001208DF80300019800283D
:1085DC0000F0E9800198006844F20001C5F6000142
:1085EC00884200D106E040F68E00C0F60100FD2165
:1085FC00FCF7CCF801984068402802D001984068FC
:10860C0000B906E040F68E00C0F60100FE21FCF732
:10861C00BDF8019880687F2800D806E040F68E00EF
:10862C00C0F60100FF21FCF7B1F80198C068C00B3F
:10863C0000B907E040F68E00C0F601004FF48071DF
:10864C00FCF7A4F80198006970B101980069B0F5C5
:10865C00001F09D001980069B0F5800F04D0019873
:10866C000069B0F5C00F00D107E040F68E00C0F6EF
:10867C00010040F20111FCF789F80198406918B12A
:10868C0001984069022800D107E040F68E00C0F640
:10869C0001004FF48171FCF779F80198806920B1E1
:1086AC0001988069B0F5801F00D107E040F68E007C
:1086BC00C0F6010040F20311FCF768F80198C0699C
:1086CC0018B10198C069012800D107E040F68E006E
:1086DC00C0F601004FF48271FCF758F8019890F83D
:1086EC00210030B90199002081F820000198FCF795
:1086FC006FF80199022081F8210001980068C06888
:10870C00C0F30010002844D101980168CA204862C7
:10871C000198016853204862019800F048F88DF8E0
:10872C0003009DF80300F0B90198016888684FF6C2
:10873C00BF72CFF68F7210408860019A1168506832
:10874C001369926918430243886810438860019842
:10875C0001688268C06840EA02400861019800F034
:10876C005DF88DF803009DF8030068B90198016865
:10877C00C86C20F00300C864019801684269C069A4
:10878C000243C86C1043C86401980168FF2048621A
:10879C0002E000208DF803009DF8030018B9019940
:0E87AC00012081F821009DF8030002B080BD7D
:1087BA0080B584B0039000208DF807000398006804
:1087CA00C0684006002826D4039801684FF0FF309D
:1087DA00C86004F0C2FF029003980068C1680020D4
:1087EA0049060029009005D49DF80700033818BFF0
:1087FA00012000900098C00768B104F0AEFF02990A
:10880A00401AB0F57A7F05D903208DF8070003993D
:0E881A0081F82100E0E79DF8070004B080BD62
:1088280080B582B0019000208DF8030044F20C015D
:10883800C5F60001086820F08000086044F20800CE
:10884800C5F600000068800600280AD4019806F0E2
:10885800B5FD28B10199032081F821008DF80300A6
:1088680019E044F20801C5F60001086820F020006C
:108878000860019806F0A2FD28B10199032081F84B
:1088880021008DF8030044F20801C5F600010868CC
:0E88980040F0200008609DF8030002B080BD93
:1088A60080B584B003900398C06A0190039800686D
:1088B600406B80B2C00B40B19DF804000007002851
:1088C60003D5039806F0A1FD71E103980068406B9B
:1088D600C0F30020002800F09F80039801684FF441
:1088E6008070886303980168C86B4CF23A12904313
:1088F600C86303980168C86B20F08050C86303986A
:108906000168C86820F04000C8609DF804000007B0
:10891600002837D59DF804008007002804D49DF868
:108926000400800600280ED50398006807F049FD6C
:108936000290029838B1029A0399486B1043486333
:10894600039804F020FE0398016840F63A70C1F6D9
:10895600000088630399012081F830000399002004
:10896600C8629DF80400C00720B99DF8040080077E
:10897600002803D5039804F006FE02E0039804F0ED
:1089860002FE48E09DF804000006002843D503983F
:1089960001680020886203990968C862039909681A
:1089A60008659DF804008007002804D49DF804009B
:1089B600800600280ED50398006807F002FD029095
:1089C600029838B1029A0399486B1043486303989A
:1089D60004F0D9FD0399012081F8300003990020A5
:1089E600C8629DF80400C006002804D49DF804005F
:1089F6008006002802D5039804F0C5FD9DF8040002
:108A0600C00720B99DF804008007002802D5039806
:108A160004F0B9FDFFE7CAE003980068406BC0F3B5
:108A2600803040B19DF804000007002803D5039864
:108A360006F027FDBBE003980068406B10F03A0F84
:108A460000F08A8003980068406BC0F3400020B1B4
:108A56000399486B40F00200486303980068406B36
:108A6600C0F3C00020B10399486B40F0080048638A
:108A760003980068406BC0F3401020B10399486B1F
:108A860040F02000486303980068406BC0F3001074
:108A960020B10399486B40F01000486303980168C1
:108AA60040F63A70C1F60000886303980168C86B07
:108AB60020F49D70C86303980168C86820F04000E0
:108AC600C86003980168C86A40F40050C8620398F9
:108AD6000168C86840F08000C8600398006807F025
:108AE60070FC02460399486B10434863039801687B
:108AF600C86820F08000C860039801684FF40060E1
:108B060088639DF80400000700280AD50399012010
:108B160081F8300003990020C862039804F033FD01
:108B260019E09DF804000006002814D50398406B50
:108B360080B103980168C86B20F08050C863039821
:108B46000168002008650399012081F83000039828
:108B560004F019FDFFE72AE003980068406BC0F3B4
:108B6600007020B3039801684FF080508863039823
:108B76000068006D400700280CD49DF804008006AC
:108B8600002803D5039804F0FEFC02E0039804F0E5
:108B9600FAFC0BE09DF804008006002803D5039834
:108BA60004F0F1FC02E0039804F0EDFCFFE704B0EA
:028BB60080BD80
:108BB80080B586B00490049818B901208DF8170084
:108BC800EBE20498006843F20001C4F20101884214
:108BD80027D00498006843F60001C4F200018842D7
:108BE8001FD00498006843F60041C4F2000188428F
:108BF80017D00498006843F20041C4F2010188428A
:108C08000FD00498006845F20001C4F201018842BF
:108C180007D00498006841F20041C5F60001884277
:108C280000D106E040F6F500C0F60100FE21FBF792
:108C3800AFFD0498406820B104984068B0F5800FF3
:108C480000D106E040F6F500C0F60100FF21FBF771
:108C58009FFD0498806870B104988068B0F5802FF3
:108C680009D004988068B0F5C02F04D004988068B3
:108C7800B0F5003F00D107E040F6F500C0F601006E
:108C88004FF48071FBF784FD0498C0681F2873D0E7
:108C98000498C0681E286FD00498C0681D286BD03F
:108CA8000498C0681C2867D00498C0681B2863D043
:108CB8000498C0681A285FD00498C06819285BD047
:108CC8000498C068182857D00498C068172853D04B
:108CD8000498C06816284FD00498C06815284BD04F
:108CE8000498C068142847D00498C068132843D053
:108CF8000498C06815283FD00498C06812283BD053
:108D08000498C068112837D00498C068102833D058
:108D18000498C0680F282FD00498C0680E282BD05C
:108D28000498C0680D2827D00498C0680C2823D060
:108D38000498C0680B281FD00498C0680A281BD064
:108D48000498C068092817D00498C068082813D068
:108D58000498C06807280FD00498C06806280BD06C
:108D68000498C068052807D00498C068042803D070
:108D78000498C068032800D107E040F6F500C0F663
:108D8800010040F20111FBF703FD0498C06B0028B5
:108D980043D00498C06B20283FD00498C06B40286B
:108DA8003BD00498C06B602837D00498C06B8028EB
:108DB80033D00498C06BA0282FD00498C06BC0286B
:108DC8002BD00498C06BE02827D00498C06BB0F56E
:108DD800807F22D00498C06BB0F5907F1DD0049896
:108DE800C06BB0F5A07F18D00498C06BB0F5B07F09
:108DF80013D00498C06BB0F5C07F0ED00498C06B38
:108E0800B0F5D07F09D00498C06BB0F5E07F04D0EE
:108E18000498C06BB0F5F07F00D107E040F6F5008C
:108E2800C0F601004FF48171FBF7B2FC0498806929
:108E3800B0F1806F07D00498806920B104988069E8
:108E4800B0F1005F00D107E040F6F500C0F6010080
:108E580040F20311FBF79CFC0498406BB0F1804F83
:108E680002D00498406B00B907E040F6F500C0F660
:108E780001004FF48271FBF78BFC0498C06910B3B2
:108E88000498C069B0F1805F1DD00498C069B0F142
:108E9800005F18D00498C069B0F1405F13D00498FF
:108EA800C069B0F1804F0ED00498C069B0F1A04FEE
:108EB80009D00498C069B0F1C04F04D00498C069C3
:108EC800B0F1E04F00D107E040F6F500C0F6010030
:108ED80040F20511FBF75CFC0498006A20B1049885
:108EE800006AB0F5000F00D107E040F6F500C0F6C3
:108EF80001004FF48371FBF74BFC0498406A20B1E2
:108F08000498406AB0F5002F00D107E040F6F5005C
:108F1800C0F6010040F20711FBF73AFC0498406ADA
:108F280008BB0498006920B104980069B0F1007F7B
:108F380000D107E040F6F500C0F601004FF4857156
:108F4800FBF726FC0498406920B104984069B0F109
:108F5800807F00D107E040F6F500C0F6010040F23E
:108F68000B11FBF715FC049900208862049800682F
:108F780043F20001C4F20101884217D00498006846
:108F880043F60001C4F2000188420FD0049800683B
:108F980043F60041C4F20001884207D00498C06833
:108FA800102803D301208DF81700F6E0049800F08C
:108FB800F8F802900498006843F20001C4F2010135
:108FC800884212D00498006843F60001C4F20001F8
:108FD80088420AD00498006843F60041C4F20001B0
:108FE800884202D0029808281AD80498006843F2E8
:108FF8000001C4F2010188420FD00498006843F6CA
:109008000001C4F20001884207D00498006843F6C2
:109018000041C4F20001884206D10298112803D306
:1090280001208DF81700B8E0049890F8810030B955
:109038000499002081F88000049804F0C3F9049989
:10904800022081F8810004980168086820F0010076
:10905800086004980068806800F4F8100390049889
:109068008069B0F1806F15D104984068B0F5800F21
:1090780002D10498806B38B10498406850B90498BC
:10908800806BB0F1805F05D104980168086840F4EE
:109098008050086004988079400600280ED504980E
:1090A800C06807280AD304980068006820F4807014
:1090B800049A1168126D1043086005E0049801686D
:1090C800086820F480700860049B1968DA68D86919
:1090D800D3F828C040EA0C00DDF80CC040EA0C00C8
:1090E800DB6B184310438860049A0192506B516AF5
:1090F8000843916B0843916908431168D2F804C08A
:109108009368D2F810E040EA0E00D2F814E040EA82
:109118000E00D2F820E040EA0E0040EA0C00D2F837
:109128004CC040EA0C001843936C1843926D1043EE
:10913800C8600498406888B904980068806801216C
:1091480061F3CC20049909688860049800688068F5
:10915800022161F34A20049909688860049801682B
:10916800086D20F001000865049880794006002801
:1091780009D504980068C06820F00040049A116876
:10918800526D1043C86004990020C1F88400049A05
:10919800012182F881108DF817009DF8170006B09C
:0291A80080BD88
:1091AA0083B002900298C16B012000EB511001902C
:1091BA000298C0680130009000980730C0080090FB
:0A91CA0000980199484303B0704774
:1091D40082B001900198006840690090019801688C
:1091E400886940F00800886101980168886940F046
:1091F4001000886101980168086820F00100086087
:1092040001980168086940F26F329043086101983F
:109214000168886820F440408860019890F88100D3
:10922400042811D09DF80000800600280CD501996F
:10923400D1F8840040F08000C1F8840001980168EE
:10924400886940F020008861019890F88100032823
:1092540011D09DF80000400600280CD50199D1F8E2
:10926400840040F00400C1F8840001980168886912
:1092740040F0400088619DF80100800700280CD56B
:109284000199D1F8840040F00100C1F884000198EC
:109294000168886940F4007088619DF80100C00786
:1092A40060B10199D1F8840040F00800C1F884004D
:1092B40001980168886940F48070886101990020F0
:0E92C400A1F862000199A1F86A0002B070479B
:1092D20080B584B00290029818B901208DF80F0071
:1092E20043E1029800680021C4F20101884274D06F
:1092F20002980068B0F1804F6FD00298006840F287
:109302000041C4F20001884267D00298006840F62A
:109312000001C4F2000188425FD00298006840F662
:109322000041C4F20001884257D00298006841F21D
:109332000001C4F2000188424FD00298006841F255
:109342000041C4F20001884247D00298006840F20E
:109352000041C4F2010188423FD00298006841F600
:109362000001C4F20001884237D00298006841F639
:109372000041C4F2000188422FD00298006842F2F4
:109382000001C4F20001884227D00298006844F22A
:109392000001C4F2010188421FD00298006844F221
:1093A2000041C4F20101884217D00298006844F6D5
:1093B2000001C4F2010188420FD0029800684EF207
:1093C2000001C4F20001884207D0029800684EF200
:1093D2000041C4F20001884200D107E040F65C106F
:1093E200C0F601004FF48B71FBF7D5F90298806843
:1093F20078B10298806810280BD0029880682028E3
:1094020007D002988068402803D0029880686028BC
:1094120000D107E040F65C10C0F6010040F21711DF
:10942200FBF7B9F90298006948B102980069B0F5F2
:10943200807F04D002980069B0F5007F00D107E078
:1094420040F65C10C0F601004FF48C71FBF7A3F9F3
:10945200029801680120B1F1804F01901ED002985C
:109462000168012040F60042C4F2000291420190DC
:1094720014D00298016801204EF20002C4F20002E8
:10948200914201900AD00298006841F60041CBF661
:10949200FF710844B0FA80F0400901900198C007BA
:1094A20040B90298C06848B10298C068B0F5803FE0
:1094B20003D303E00298C06800B107E040F65C10F5
:1094C200C0F6010040F21911FBF765F902988069B4
:1094D20018B102988069802800D107E040F65C103C
:1094E200C0F601004FF48D71FBF755F9029890F820
:1094F2003D0030B90299002081F83C00029804F046
:10950200BEF80299022081F83D00029951F8040B3D
:1095120000F02FF80299012081F8480002990120F9
:1095220081F83E00029981F83F00029981F84000DB
:10953200029981F84100029981F84200029981F86A
:1095420043000299012081F84400029981F8450004
:10955200029981F84600029981F847000299012098
:1095620081F83D0000208DF80F009DF80F0004B037
:0295720080BDBA
:1095740083B0029001910298006800900298002143
:10958400C4F2010188421FD00298B0F1804F1BD071
:10959400029840F20041C4F20001884214D00298BB
:1095A40040F60001C4F2000188420DD0029840F652
:1095B4000041C4F20001884206D0029840F2004102
:1095C400C4F20101884208D1009820F07000009094
:1095D4000198416800980843009002980021C4F261
:1095E4000101884242D00298B0F1804F3ED00298E7
:1095F40040F20041C4F20001884237D0029840F69C
:109604000001C4F20001884230D0029840F60041C3
:10961400C4F20001884229D0029840F20041C4F209
:109624000101884222D0029844F20001C4F20101EF
:1096340088421BD0029844F20041C4F201018842DE
:1096440014D0029844F60001C4F2010188420DD0FE
:1096540002984EF20001C4F20001884206D002983A
:109664004EF20041C4F20001884208D1009820F46F
:10967400407000900198C1680098084300900098D9
:1096840020F080000199496908430090019880689E
:109694000299C862019800680299886202980021C0
:1096A400C4F2010188421BD0029840F20041C4F286
:1096B4000101884214D0029844F20001C4F201016D
:1096C40088420DD0029844F20041C4F2010188425C
:1096D40006D0029844F60001C4F20101884203D185
:1096E40001980069029908630299086840F004002F
:1096F400086002990120486100980299086003B04B
:029704007047AC
:1097060080B584B00290029818B901208DF80F0038
:1097160043E1029800680021C4F20101884274D036
:1097260002980068B0F1804F6FD00298006840F24E
:109736000041C4F20001884267D00298006840F6F2
:109746000001C4F2000188425FD00298006840F62A
:109756000041C4F20001884257D00298006841F2E5
:109766000001C4F2000188424FD00298006841F21D
:109776000041C4F20001884247D00298006840F2D6
:109786000041C4F2010188423FD00298006841F6C8
:109796000001C4F20001884237D00298006841F601
:1097A6000041C4F2000188422FD00298006842F2BC
:1097B6000001C4F20001884227D00298006844F2F2
:1097C6000001C4F2010188421FD00298006844F2E9
:1097D6000041C4F20101884217D00298006844F69D
:1097E6000001C4F2010188420FD0029800684EF2CF
:1097F6000001C4F20001884207D0029800684EF2C8
:109806000041C4F20001884200D107E040F65C1036
:10981600C0F6010040F23351FAF7BBFF02988068A8
:1098260078B10298806810280BD0029880682028AA
:1098360007D002988068402803D002988068602884
:1098460000D107E040F65C10C0F6010040F234514A
:10985600FAF79FFF0298006948B102980069B0F5CF
:10986600807F04D002980069B0F5007F00D107E040
:1098760040F65C10C0F6010040F23551FAF789FF58
:10988600029801680120B1F1804F01901ED0029824
:109896000168012040F60042C4F2000291420190A4
:1098A60014D00298016801204EF20002C4F20002B0
:1098B600914201900AD00298006841F60041CBF629
:1098C600FF710844B0FA80F0400901900198C00782
:1098D60040B90298C06848B10298C068B0F5803FA8
:1098E60003D303E00298C06800B107E040F65C10BD
:1098F600C0F6010040F23651FAF74BFF0298806934
:1099060018B102988069802800D107E040F65C1003
:10991600C0F6010040F23751FAF73BFF029890F883
:109926003D0030B90299002081F83C00029803F00E
:109936002AFE0299022081F83D00029951F8040B93
:10994600FFF715FE0299012081F8480002990120CF
:1099560081F83E00029981F83F00029981F84000A3
:10996600029981F84100029981F84200029981F832
:1099760043000299012081F84400029981F84500CC
:10998600029981F84600029981F847000299012060
:1099960081F83D0000208DF80F009DF80F0004B0FF
:0299A60080BD82
:1099A80080B584B00290029818B901208DF80F0094
:1099B80043E1029800680021C4F20101884274D092
:1099C80002980068B0F1804F6FD00298006840F2AA
:1099D8000041C4F20001884267D00298006840F64E
:1099E8000001C4F2000188425FD00298006840F686
:1099F8000041C4F20001884257D00298006841F241
:109A08000001C4F2000188424FD00298006841F278
:109A18000041C4F20001884247D00298006840F231
:109A28000041C4F2010188423FD00298006841F623
:109A38000001C4F20001884237D00298006841F65C
:109A48000041C4F2000188422FD00298006842F217
:109A58000001C4F20001884227D00298006844F24D
:109A68000001C4F2010188421FD00298006844F244
:109A78000041C4F20101884217D00298006844F6F8
:109A88000001C4F2010188420FD0029800684EF22A
:109A98000001C4F20001884207D0029800684EF223
:109AA8000041C4F20001884200D107E040F65C1092
:109AB800C0F6010040F2CF71FAF76AFE029880689A
:109AC80078B10298806810280BD002988068202806
:109AD80007D002988068402803D0029880686028E0
:109AE80000D107E040F65C10C0F601004FF4FA61BF
:109AF800FAF74EFE0298006948B102980069B0F57D
:109B0800807F04D002980069B0F5007F00D107E09B
:109B180040F65C10C0F6010040F2D171FAF738FE49
:109B2800029801680120B1F1804F01901ED002987F
:109B38000168012040F60042C4F2000291420190FF
:109B480014D00298016801204EF20002C4F200020B
:109B5800914201900AD00298006841F60041CBF684
:109B6800FF710844B0FA80F0400901900198C007DD
:109B780040B90298C06848B10298C068B0F5803F03
:109B880003D303E00298C06800B107E040F65C1018
:109B9800C0F6010040F2D271FAF7FAFD0298806926
:109BA80018B102988069802800D107E040F65C105F
:109BB800C0F6010040F2D371FAF7EAFD029890F876
:109BC8003D0030B90299002081F83C00029803F06A
:109BD800D9FC0299022081F83D00029951F8040B42
:109BE800FFF7C4FC0299012081F84800029901207E
:109BF80081F83E00029981F83F00029981F84000FF
:109C0800029981F84100029981F84200029981F88D
:109C180043000299012081F84400029981F8450027
:109C2800029981F84600029981F8470002990120BB
:109C380081F83D0000208DF80F009DF80F0004B05A
:029C480080BDDD
:109C4A0080B584B0039003980068C06802900398B6
:109C5A000068006901909DF80400800700281ED55D
:109C6A009DF808008007002819D5039801686FF04D
:109C7A000200086103990120087703980068806947
:109C8A00800718B1039803F07CFC05E0039803F001
:109C9A0078FC039803F075FC0399002008779DF877
:109CAA000400400700281FD59DF808004007002837
:109CBA001AD5039801686FF004000861039902201D
:109CCA00087703980068806910F4407F03D00398EE
:109CDA0003F057FC05E0039803F053FC039803F0E4
:109CEA0050FC0399002008779DF80400000700281B
:109CFA001ED59DF808000007002819D503980168A9
:109D0A006FF0080008610399042008770398006837
:109D1A00C069800718B1039803F033FC05E0039883
:109D2A0003F02FFC039803F02CFC0399002008771A
:109D3A009DF80400C00600281FD59DF80800C0063B
:109D4A0000281AD5039801686FF01000086103997A
:109D5A000820087703980068C06910F4407F03D090
:109D6A00039803F00EFC05E0039803F00AFC03983D
:109D7A0003F007FC0399002008779DF80400C00748
:109D8A0058B19DF80800C00738B1039801686FF010
:109D9A00010008610398FAF7EBFC019800F08000D3
:109DAA00802804D09DF80500800600280CD59DF86F
:109DBA0008000006002807D5039801686FF40250CE
:109DCA000861039803F0DDFB9DF80500C00760B148
:109DDA009DF808000006002807D5039801686FF46B
:109DEA0080700861039803F0CCFB9DF804004006DC
:109DFA0000280CD59DF808004006002807D50398CE
:109E0A0001686FF040000861039803F0BAFB9DF8FF
:109E1A000400800600280CD59DF80800800600285A
:109E2A0007D5039801686FF020000861039803F0D2
:069E3A00A8FB04B080BD8E
:109E400080B586B0059004910598006A0290059946
:109E5000086A20F0010008620598406801900598A2
:109E60008069039003984FF68F71CFF6FE7108401A
:109E70000390039820F0030003900498016803986E
:109E800008430390029820F0020002900498816831
:109E900002980843029005980021C4F2010188420B
:109EA0001BD0059840F20041C4F20101884214D051
:109EB000059844F20001C4F2010188420DD00598D2
:109EC00044F20041C4F20101884206D0059844F6EC
:109ED0000001C4F2010188421CD10498C06818B185
:109EE0000498C068082800D107E040F65C10C0F66E
:109EF000010041F66B31FAF74FFC029820F00800A0
:109F000002900498C168029808430290029820F0D9
:109F10000400029005980021C4F2010188421BD080
:109F2000059840F20041C4F20101884214D005981E
:109F300044F20001C4F2010188420DD0059844F2B8
:109F40000041C4F20101884206D0059844F60001A0
:109F5000C4F20101884233D104988069B0F5007FD2
:109F600002D00498806900B907E040F65C10C0F6A2
:109F7000010041F67831FAF70FFC04984069B0F51A
:109F8000807F02D00498406900B907E040F65C1079
:109F9000C0F6010041F67931FAF7FEFB019820F492
:109FA00080700190019820F400700190049841693C
:109FB0000198084301900498816901980843019031
:109FC000019805994860039805998861049840684C
:0E9FD0000599486302980599086206B080BDA5
:109FDE0080B586B0059004910598006A02900599A7
:109FEE00086A20F480700862059840680190059810
:109FFE00C069039003984FF68F71CFF6FE7108403B
:10A00E000390039820F003000390049801680398CE
:10A01E0008430390029820F400700290049881681F
:10A02E00029840EA0120029005980021C4F2010135
:10A03E00884221D0059840F20041C4F201018842C5
:10A04E001AD0059844F20001C4F20101884201D1F0
:10A05E00002088B9059844F20041C4F201018842FB
:10A06E0001D1002040B9059844F60001C4F2010167
:10A07E0088421FD10120E8B90498C06818B104982D
:10A08E00C068082800D107E040F65C10C0F6010059
:10A09E0041F60241FAF779FB029820F40060029033
:10A0AE000498C168029840EA01200290029820F4B8
:10A0BE008060029005980021C4F2010188421BD0F5
:10A0CE00059840F20041C4F20101884214D005986F
:10A0DE0044F20001C4F2010188420DD0059844F209
:10A0EE000041C4F20101884206D0059844F60001F1
:10A0FE00C4F20101884235D104988069B0F5007F21
:10A10E0002D00498806900B907E040F65C10C0F6F2
:10A11E00010041F60F41FAF738FB04984069B0F59B
:10A12E00807F02D00498406900B907E040F65C10C9
:10A13E00C0F6010041F61041FAF727FB019820F412
:10A14E0080500190019820F40050019004984169CC
:10A15E00019840EA0110019004988169019840EA43
:10A16E000110019001980599486003980599C861FE
:10A17E00049840680599C86302980599086206B06C
:02A18E0080BD92
:10A1900080B586B0059004910598006A02900599F3
:10A1A000086A20F48050086205984068019005987C
:10A1B000C0690390039848F6FF71CFF6FF6108402D
:10A1C0000390039820F4407003900498016803986A
:10A1D00040EA01200390029820F400500290049875
:10A1E0008168029840EA0130029005980021C4F28B
:10A1F000010188421BD0059840F20041C4F20101E0
:10A20000884214D0059844F20001C4F2010188424A
:10A210000DD0059844F20041C4F20101884206D0F5
:10A22000059844F60001C4F2010188421AD104984D
:10A230004069B0F5807F02D00498406900B907E01A
:10A2400040F65C10C0F6010041F64F41FAF7A4FA5F
:10A25000019820F48040019004984169019840EAF7
:10A260008110019001980599486003980599C8618B
:10A27000049840680599086402980599086206B038
:02A2800080BD9F
:10A2820085B0049003910498006A01900499086AC9
:10A2920020F4801008620498406800900498406D91
:10A2A2000290029848F6FF71CFF6FF6108400290D3
:10A2B20003980168029840EA01200290019820F474
:10A2C2000010019003988168019840EA01500190C2
:10A2D20004980021C4F2010188421BD0049840F284
:10A2E2000041C4F20101884214D0049844F20001F2
:10A2F200C4F2010188420DD0049844F20041C4F234
:10A302000101884206D0049844F60001C4F201011A
:10A31200884209D1009820F4802000900398416976
:10A32200009840EA812000900098049948600298C1
:10A3320004994865039840680499C865019804998E
:06A34200086205B070473F
:10A3480080B586B004900391029200208DF8070032
:10A35800049800680021C4F20101884264D004987E
:10A368000068B0F1804F5FD00498006840F2004167
:10A37800C4F20001884257D00498006840F60001F2
:10A38800C4F2000188424FD00498006840F60041AA
:10A39800C4F20001884247D00498006840F20041A6
:10A3A800C4F2010188423FD00498006841F60001D8
:10A3B800C4F20001884237D00498006841F6004191
:10A3C800C4F2000188422FD00498006842F20001CC
:10A3D800C4F20001884227D00498006844F20001C2
:10A3E800C4F2010188421FD00498006844F2004179
:10A3F800C4F20101884217D00498006844F60001AD
:10A40800C4F2010188420FD0049800684EF200019E
:10A41800C4F20001884207D0049800684EF2004157
:10A42800C4F20001884200D107E040F65C10C0F693
:10A43800010041F24C01FAF7ABF90398006838B112
:10A4480003980068022803D0039800680A2800D1FE
:10A4580007E040F65C10C0F6010041F24D01FAF742
:10A4680097F903984068012807D0039840680228A4
:10A4780003D003984068032800D107E040F65C1039
:10A48800C0F6010041F24E01FAF782F9039880689C
:10A4980058B103988068042807D003988068082872
:10A4A80003D0039880680C2800D107E040F65C10C0
:10A4B800C0F6010041F24F01FAF76AF90398C06843
:10A4C8000F2800D807E040F65C10C0F6010041F202
:10A4D8005001FAF75DF9049890F83C00012803D17F
:10A4E80002208DF8170052E10499012081F83C0000
:10A4F8000298A8B904980068039B19685A68DB6831
:10A5080000F049F904980168886920F00C00886116
:10A5180003988268049801688869104388612EE16D
:10A52800029804286BD1049800680021C4F2010144
:10A53800884244D004980068B0F1804F3FD0049816
:10A54800006840F20041C4F20001884237D0049804
:10A55800006840F60001C4F2000188422FD0049838
:10A56800006840F60041C4F20001884227D00498F0
:10A57800006840F20041C4F2010188421FD00498EB
:10A58800006841F60001C4F20001884217D004981F
:10A59800006844F20001C4F2010188420FD0049817
:10A5A80000684EF20001C4F20001884207D0049806
:10A5B80000684EF20041C4F20001884200D107E071
:10A5C80040F65C10C0F6010041F26601FAF7E0F8C7
:10A5D80004980068039B19685A68DB6805F080FBDB
:10A5E80004980168886920F440608861039882684B
:10A5F80004980168886940EA02208861BFE00298EF
:10A6080008285AD1049800680021C4F20101884240
:10A6180034D004980068B0F1804F2FD004980068B7
:10A6280040F20041C4F20001884227D00498006833
:10A6380040F60001C4F2000188421FD00498006867
:10A6480040F60041C4F20001884217D0049800681F
:10A6580040F20041C4F2010188420FD0049800681A
:10A668004EF20001C4F20001884207D00498006845
:10A678004EF20041C4F20001884200D107E040F6E2
:10A688005C10C0F6010041F27601FAF781F80498EF
:10A698000068039B19685A68DB6800F00FF9049892
:10A6A8000168C86920F00C00C861039882680498A2
:10A6B8000168C8691043C86161E002980C285BD141
:10A6C800049800680021C4F20101884234D004983B
:10A6D8000068B0F1804F2FD00498006840F2004124
:10A6E800C4F20001884227D00498006840F60001AF
:10A6F800C4F2000188421FD00498006840F6004167
:10A70800C4F20001884217D00498006840F2004162
:10A71800C4F2010188420FD0049800684EF200018B
:10A72800C4F20001884207D0049800684EF2004144
:10A73800C4F20001884200D107E040F65C10C0F680
:10A74800010041F28601FAF723F804980068039B98
:10A7580019685A68DB6805F0F9FA04980168C8694D
:10A7680020F44060C8610398826804980168C86949
:10A7780040EA0220C86102E001208DF80700049930
:10A78800002081F83C009DF807008DF817009DF81F
:06A79800170006B080BDB1
:10A79E0087B006900591049203930698006A019083
:10A7AE000699086A20F001000862069880690290F6
:10A7BE00069901200022C4F20102914200904ED06F
:10A7CE0006990120B1F1804F009048D006990120E2
:10A7DE0040F20042C4F20002914200903FD006992E
:10A7EE00012040F60002C4F200029142009036D0E1
:10A7FE000699012040F60042C4F2000291420090F8
:10A80E002DD00699012040F20042C4F2010291427D
:10A81E00009024D00699012041F60002C4F20002F5
:10A82E00914200901BD00699012044F20002C4F21E
:10A83E0001029142009012D0069901204EF20002C0
:10A84E00C4F200029142009009D0069841F60041F0
:10A85E00CBF6FF710844B0FA80F0400900900098E2
:10A86E00C00740B1029820F00300029004990298AC
:10A87E000843029003E0029840F001000290029813
:10A88E0020F0F000029003980001C1B20298084334
:10A89E000290019820F00A000190059800F00A013C
:10A8AE0001980843019002980699886101980699CB
:06A8BE00086207B07047BC
:10A8C40086B005900491039202930598006A009063
:10A8D4000599086A20F4807008620598C06901909F
:10A8E400019820F003000190039901980843019016
:10A8F400019820F0F000019002980001C1B2019883
:10A9040008430190009820F420600090049800F01F
:10A914000A01009840EA0120009001980599C86155
:0AA9240000980599086206B070471C
:10A92E0080B586B00490039100208DF80B0004983A
:10A93E0090F83C00012804D102208DF8170000F099
:10A94E0060BC0499012081F83C000499022081F832
:10A95E003D0003980068B0F5805F23D0039800682F
:10A96E0070281FD003980068B0F5005F1AD00398C6
:10A97E000068402816D003980068502812D003981B
:10A98E00006860280ED00398006858B103980068DC
:10A99E00102807D003980068202803D00398006879
:10A9AE00302800D107E040F65C10C0F6010041F2FD
:10A9BE005151F9F7EAFE04980068806801900198F9
:10A9CE004FF68871CFF6CE7108400190019820F4B1
:10A9DE007F40019001980499096888600398006887
:10A9EE000090002800F0A2830098102800F09E83AB
:10A9FE000098202800F09A830098302800F0968363
:10AA0E000098402800F007830098502800F0ED8150
:10AA1E000098602800F074820098702800F0AF80D3
:10AA2E000098B0F5805F24D00098B0F5005F00F07C
:10AA3E0044810098B0F5801F00F078830098B0F143
:10AA4E00101F00F0738300982021C0F2100188427D
:10AA5E0000F06C8300983021C0F21001884200F0A3
:10AA6E00658300984021C0F21001884200F05E8399
:10AA7E00B8E3049800680021C4F20101884274D042
:10AA8E0004980068B0F1804F6FD00498006840F2CF
:10AA9E000041C4F20001884267D00498006840F675
:10AAAE000001C4F2000188425FD00498006840F6AD
:10AABE000041C4F20001884257D00498006841F268
:10AACE000001C4F2000188424FD00498006841F2A0
:10AADE000041C4F20001884247D00498006840F259
:10AAEE000041C4F2010188423FD00498006841F64B
:10AAFE000001C4F20001884237D00498006841F684
:10AB0E000041C4F2000188422FD00498006842F23E
:10AB1E000001C4F20001884227D00498006844F274
:10AB2E000001C4F2010188421FD00498006844F26B
:10AB3E000041C4F20101884217D00498006844F61F
:10AB4E000001C4F2010188420FD0049800684EF251
:10AB5E000001C4F20001884207D0049800684EF24A
:10AB6E000041C4F20001884200D107E040F65C10BB
:10AB7E00C0F6010041F25D51F9F707FE35E3049886
:10AB8E0000680021C4F20101884234D004980068A4
:10AB9E00B0F1804F2FD00498006840F20041C4F20B
:10ABAE000001884227D00498006840F60001C4F2E4
:10ABBE00000188421FD00498006840F60041C4F29C
:10ABCE000001884217D00498006840F20041C4F298
:10ABDE00010188420FD0049800684EF20001C4F2C1
:10ABEE000001884207D0049800684EF20041C4F27A
:10ABFE000001884200D107E040F65C10C0F601006B
:10AC0E0041F26451F9F7C1FD0398806870B1039861
:10AC1E008068B0F5805F09D003988068B0F5005F5A
:10AC2E0004D003988068B0F5405F00D107E040F68D
:10AC3E005C10C0F6010041F26751F9F7A6FD0398CA
:10AC4E004068B0F5004F0DD00398406850B103989E
:10AC5E00406838B103984068022803D003984068D2
:10AC6E000A2800D107E040F65C10C0F6010041F260
:10AC7E006851F9F78AFD0398C0680F2800D807E0DD
:10AC8E0040F65C10C0F6010041F26951F9F77DFD06
:10AC9E0004980068039B5A689968DB6805F089F888
:10ACAE000498006880680190019840F07700019048
:10ACBE00019804990968886097E204980068002159
:10ACCE00C4F20101884234D004980068B0F1804F7C
:10ACDE002FD00498006840F20041C4F2000188426F
:10ACEE0027D00498006840F60001C4F200018842A3
:10ACFE001FD00498006840F60041C4F2000188425B
:10AD0E0017D00498006840F20041C4F20101884255
:10AD1E000FD0049800684EF20001C4F20001884280
:10AD2E0007D0049800684EF20041C4F20001884238
:10AD3E0000D107E040F65C10C0F6010041F27C51F4
:10AD4E00F9F723FD0398806870B103988068B0F519
:10AD5E00805F09D003988068B0F5005F04D0039837
:10AD6E008068B0F5405F00D107E040F65C10C0F699
:10AD7E00010041F27F51F9F708FD03984068B0F5E4
:10AD8E00004F0DD00398406850B10398406838B119
:10AD9E0003984068022803D0039840680A2800D11F
:10ADAE0007E040F65C10C0F601004FF4AC51F9F725
:10ADBE00ECFC0398C0680F2800D807E040F65C1042
:10ADCE00C0F6010041F28151F9F7DFFC04980068EA
:10ADDE00039B5A689968DB6804F0EBFF04980168DE
:10ADEE00886840F480408860FFE104980068002184
:10ADFE00C4F20101884244D004980068B0F1804F3B
:10AE0E003FD00498006840F20041C4F2000188422D
:10AE1E0037D00498006840F60001C4F20001884261
:10AE2E002FD00498006840F60041C4F20001884219
:10AE3E0027D00498006840F20041C4F20101884214
:10AE4E001FD00498006841F60001C4F20001884248
:10AE5E0017D00498006844F20001C4F20101884240
:10AE6E000FD0049800684EF20001C4F2000188422F
:10AE7E0007D0049800684EF20041C4F200018842E7
:10AE8E0000D107E040F65C10C0F6010041F290518F
:10AE9E00F9F77BFC03984068B0F5004F0DD003988E
:10AEAE00406850B10398406838B103984068022852
:10AEBE0003D0039840680A2800D107E040F65C10E2
:10AECE00C0F6010041F29351F9F75FFC0398C06898
:10AEDE000F2800D807E040F65C10C0F6010041F2E2
:10AEEE009451F9F752FC04980068039A5168D2689D
:10AEFE0004F079FF04980068502104F09CFF74E17F
:10AF0E00049800680021C4F20101884244D00498DC
:10AF1E000068B0F1804F3FD00498006840F20041C5
:10AF2E00C4F20001884237D00498006840F6000150
:10AF3E00C4F2000188422FD00498006840F6004108
:10AF4E00C4F20001884227D00498006840F2004104
:10AF5E00C4F2010188421FD00498006841F6000136
:10AF6E00C4F20001884217D00498006844F2000130
:10AF7E00C4F2010188420FD0049800684EF200011D
:10AF8E00C4F20001884207D0049800684EF20041D6
:10AF9E00C4F20001884200D107E040F65C10C0F612
:10AFAE0001004FF4AD51F9F7F0FB03984068B0F58E
:10AFBE00004F0DD00398406850B10398406838B1E7
:10AFCE0003984068022803D0039840680A2800D1ED
:10AFDE0007E040F65C10C0F6010041F2A351F9F70C
:10AFEE00D4FB0398C0680F2800D807E040F65C1029
:10AFFE00C0F6010041F2A451F9F7C7FB04980068AE
:10B00E00039A5168D26800F000F904980068602134
:10B01E0004F011FFE9E0049800680021C4F2010178
:10B02E00884244D004980068B0F1804F3FD0049815
:10B03E00006840F20041C4F20001884237D0049803
:10B04E00006840F60001C4F2000188422FD0049837
:10B05E00006840F60041C4F20001884227D00498EF
:10B06E00006840F20041C4F2010188421FD00498EA
:10B07E00006841F60001C4F20001884217D004981E
:10B08E00006844F20001C4F2010188420FD0049816
:10B09E0000684EF20001C4F20001884207D0049805
:10B0AE0000684EF20041C4F20001884200D107E070
:10B0BE0040F65C10C0F6010041F2B051F9F765FBA5
:10B0CE0003984068B0F5004F0DD00398406850B11A
:10B0DE000398406838B103984068022803D003985B
:10B0EE0040680A2800D107E040F65C10C0F6010067
:10B0FE0041F2B351F9F749FB0398C0680F2800D805
:10B10E0007E040F65C10C0F6010041F2B451F9F7C9
:10B11E003CFB04980068039A5168D26804F063FE01
:10B12E0004980068402104F086FE5EE004980068F2
:10B13E000021C4F20101884244D004980068B0F1A5
:10B14E00804F3FD00498006840F20041C4F20001E5
:10B15E00884237D00498006840F60001C4F200011E
:10B16E0088422FD00498006840F60041C4F20001D6
:10B17E00884227D00498006840F20041C4F20101D1
:10B18E0088421FD00498006841F60001C4F2000105
:10B19E00884217D00498006844F20001C4F20101FD
:10B1AE0088420FD0049800684EF20001C4F20001EC
:10B1BE00884207D0049800684EF20041C4F20001A4
:10B1CE00884200D107E040F65C10C0F6010041F263
:10B1DE00C851F9F7DAFA049800680399096804F07F
:10B1EE002AFE02E001208DF80B000499012081F85F
:10B1FE003D000499002081F83C009DF80B008DF86D
:0AB20E0017009DF8170006B080BD80
:10B2180085B00490039102920498006A0090049902
:10B22800086A20F01000086204988069019001986B
:10B2380020F4704001900299019840EA0130019091
:10B24800009820F0A00000900399009840EA0110AF
:10B25800009001980499886100980499086205B0E3
:02B2680070472D
:10B26A0080B584B002900191029800680021C4F26E
:10B27A000101884244D002980068B0F1804F3FD063
:10B28A000298006840F20041C4F20001884237D0B7
:10B29A000298006840F60001C4F2000188422FD0EB
:10B2AA000298006840F60041C4F20001884227D0A3
:10B2BA000298006840F20041C4F2010188421FD09E
:10B2CA000298006841F60001C4F20001884217D0D2
:10B2DA000298006844F20001C4F2010188420FD0CA
:10B2EA00029800684EF20001C4F20001884207D0B9
:10B2FA00029800684EF20041C4F20001884200D16F
:10B30A0007E040F65C10C0F6010041F20861F9F767
:10B31A003EFA01980068A0B101980068042810D08C
:10B32A000198006805280CD001980068062808D002
:10B33A0001980068072804D001980068B0F5803F9A
:10B34A0000D107E040F65C10C0F6010041F2096145
:10B35A00F9F71DFA01984068002846D0019840681C
:10B36A00102842D00198406820283ED001984068B1
:10B37A0030283AD001984068B0F5801F35D001983E
:10B38A004068B0F1101F30D0019840682021C0F207
:10B39A001001884229D0019840683021C0F210017A
:10B3AA00884222D0019840684021C0F210018842A8
:10B3BA001BD001984068B0F5001F16D0019840686C
:10B3CA001021C0F2200188420FD00198406840281D
:10B3DA000BD001984068502807D00198406860282F
:10B3EA0003D001984068702800D107E040F65C104D
:10B3FA00C0F6010041F20A61F9F7C9F9029890F81A
:10B40A003C00012803D102208DF80F002FE0029999
:10B41A00012081F83C000299022081F83D0002983F
:10B42A00019900F028F858B10299012081F83D00ED
:10B43A000299002081F83C0001208DF80F0016E0E7
:10B44A0002980168C86820F04000C8600298016844
:10B45A00C86820F48040C8600299012081F83D0044
:10B46A000299002081F83C0000208DF80F009DF819
:06B47A000F0004B080BDCC
:10B4800080B588B00690059100208DF813000698CD
:10B4900000688068039003984FF68F71CFF6CF71E4
:10B4A0000840039005984168039808430390039867
:10B4B0004FF6F871CFF6FE710840039005980168C9
:10B4C00003980843039003980699096888600598D3
:10B4D00040680090002800F0C5820098102800F015
:10B4E000C1820098202800F0BD820098302800F02A
:10B4F000B9820098402800F0DE800098502800F0C3
:10B5000085810098602800F027820098702840D03C
:10B510000098B0F5801F00F0A5820098B0F1101FD0
:10B5200000F0A08200982021C0F21001884200F0B3
:10B53000998200983021C0F21001884200F0928276
:10B5400000984021C0F21001884200F08B820098E0
:10B550005021C0F21001884200F0848200986021DE
:10B56000C0F21001884200F07D8200987021C0F284
:10B570001001884200F076820098B0F5001F00F0BC
:10B58000718200981021C0F22001884200F06A8286
:10B59000BEE2069800680021C4F20101884234D05E
:10B5A00006980068B0F1804F2FD00698006840F2EE
:10B5B0000041C4F20001884227D00698006840F696
:10B5C0000001C4F2000188421FD00698006840F6CE
:10B5D0000041C4F20001884217D00698006840F28A
:10B5E0000041C4F2010188420FD0069800684EF273
:10B5F0000001C4F20001884207D0069800684EF2AC
:10B600000041C4F20001884200D107E040F65C101E
:10B61000C0F6010041F6F641F9F7BEF80598C0689A
:10B6200070B10598C068B0F5805F09D00598C06812
:10B63000B0F5005F04D00598C068B0F5405F00D158
:10B6400007E040F65C10C0F6010041F6F741F9F75B
:10B65000A3F805988068B0F5004F0DD00598806874
:10B6600050B10598806838B105988068022803D0E9
:10B67000059880680A2800D107E040F65C10C0F603
:10B68000010041F6F841F9F787F8059800690F289D
:10B6900000D807E040F65C10C0F6010041F6F94121
:10B6A000F9F77AF806980068059B9A68D9681B69CB
:10B6B00004F086FB2FE2069800680021C4F2010125
:10B6C000884264D006980068B0F1804F5FD0069839
:10B6D000006840F20041C4F20001884257D0069849
:10B6E000006840F60001C4F2000188424FD006987D
:10B6F000006840F60041C4F20001884247D0069835
:10B70000006840F20041C4F2010188423FD006982F
:10B71000006841F60001C4F20001884237D0069863
:10B72000006841F60041C4F2000188422FD006981B
:10B73000006842F20001C4F20001884227D0069856
:10B74000006844F20001C4F2010188421FD006984B
:10B75000006844F20041C4F20101884217D0069803
:10B76000006844F60001C4F2010188420FD0069837
:10B7700000684EF20001C4F20001884207D006982A
:10B7800000684EF20041C4F20001884200D107E097
:10B7900040F65C10C0F6010041F60551F8F7FCFFD9
:10B7A000059800690F2800D807E040F65C10C0F645
:10B7B000010041F60651F8F7EFFF059800680528EB
:10B7C00003D101208DF81F00A9E106980068006AE6
:10B7D000019006980168086A20F001000862069846
:10B7E000006880690290029820F0F00002900598AD
:10B7F0000169029840EA01100290029806990968CE
:10B800008861019806990968086284E106980068D1
:10B810000021C4F20101884264D006980068B0F1AA
:10B82000804F5FD00698006840F20041C4F20001EA
:10B83000884257D00698006840F60001C4F2000123
:10B8400088424FD00698006840F60041C4F20001DB
:10B85000884247D00698006840F20041C4F20101D6
:10B8600088423FD00698006841F60001C4F200010A
:10B87000884237D00698006841F60041C4F20001C2
:10B8800088422FD00698006842F20001C4F20001FD
:10B89000884227D00698006844F20001C4F20101F2
:10B8A00088421FD00698006844F20041C4F20101AA
:10B8B000884217D00698006844F60001C4F20101DE
:10B8C00088420FD0069800684EF20001C4F20001D1
:10B8D000884207D0069800684EF20041C4F2000189
:10B8E000884200D107E040F65C10C0F6010041F646
:10B8F0001F51F8F751FF05988068B0F5004F0DD043
:10B900000598806850B10598806838B105988068BE
:10B91000022803D0059880680A2800D107E040F685
:10B920005C10C0F601004FF4E951F8F735FF0598B7
:10B9300000690F2800D807E040F65C10C0F601004F
:10B9400041F62151F8F728FF06980068059A91689A
:10B95000126904F04FFADEE0069800680021C4F294
:10B960000101884244D006980068B0F1804F3FD072
:10B970000698006840F20041C4F20001884237D0C6
:10B980000698006840F60001C4F2000188422FD0FA
:10B990000698006840F60041C4F20001884227D0B2
:10B9A0000698006840F20041C4F2010188421FD0AD
:10B9B0000698006841F60001C4F20001884217D0E1
:10B9C0000698006844F20001C4F2010188420FD0D9
:10B9D000069800684EF20001C4F20001884207D0C8
:10B9E000069800684EF20041C4F20001884200D17E
:10B9F00007E040F65C10C0F6010041F62D51F8F763
:10BA0000CBFE05988068B0F5004F0DD00598806892
:10BA100050B10598806838B105988068022803D035
:10BA2000059880680A2800D107E040F65C10C0F64F
:10BA3000010041F62E51F8F7AFFE059800690F2876
:10BA400000D807E040F65C10C0F6010041F62F5127
:10BA5000F8F7A2FE06980068059A91681269FFF748
:10BA6000DBFB58E0069800680021C4F2010188421F
:10BA700044D006980068B0F1804F3FD00698006827
:10BA800040F20041C4F20001884237D006980068B5
:10BA900040F60001C4F2000188422FD006980068E9
:10BAA00040F60041C4F20001884227D006980068A1
:10BAB00040F20041C4F2010188421FD0069800689C
:10BAC00041F60001C4F20001884217D006980068D0
:10BAD00044F20001C4F2010188420FD006980068C8
:10BAE0004EF20001C4F20001884207D006980068B7
:10BAF0004EF20041C4F20001884200D107E040F656
:10BB00005C10C0F6010041F64851F8F745FE02E02E
:10BB100001208DF813009DF813008DF81F009DF88B
:06BB20001F0008B080BD0B
:10BB260080B582B00090009818B901208DF8070002
:10BB360001E100988069002861D00098006841F210
:10BB46000001C4F2010188424FD00098006844F217
:10BB56000041C4F20001884247D00098006844F6CC
:10BB66000001C4F2000188423FD00098006844F604
:10BB76000041C4F20001884237D00098006845F2BF
:10BB86000001C4F2000188422FD00098006841F2FB
:10BB96000041C4F20101884227D00098006847F6A8
:10BBA6000001C4F2000188421FD00098006847F6E1
:10BBB6000041C4F20001884217D00098006841F69F
:10BBC6000001C4F2010188420FD00098006841F6D6
:10BBD6000041C4F20101884207D00098006840F68F
:10BBE6000041C5F60001884200D107E040F6D25078
:10BBF600C0F601004FF49F71F8F7CBFD60E00098A6
:10BC0600006841F20001C4F2010188424FD0009859
:10BC1600006844F20041C4F20001884247D000980F
:10BC2600006844F60001C4F2000188423FD0009843
:10BC3600006844F60041C4F20001884237D00098FB
:10BC4600006845F20001C4F2000188422FD0009836
:10BC5600006841F20041C4F20101884227D00098F1
:10BC6600006847F60001C4F2000188421FD0009820
:10BC7600006847F60041C4F20001884217D00098D8
:10BC8600006841F60001C4F2010188420FD0009815
:10BC9600006841F60041C4F20101884207D00098CD
:10BCA600006840F60041C5F60001884200D107E071
:10BCB60040F6D250C0F6010040F24311F8F769FD94
:10BCC6000098D0F8880030B90099002081F88400E7
:10BCD6000098F8F7B7FF00992420C1F8880000986B
:10BCE6000168086820F0010008600098806A10B1B9
:10BCF600009800F024F80098F7F753FD012803D1C7
:10BD060001208DF8070016E000980168486820F4C5
:10BD16009040486000980168886820F02A00886092
:10BD260000980168086840F001000860009804F077
:0EBD360042FA8DF807009DF8070002B080BDAC
:10BD440080B582B001900198806AFF2800D807E08E
:10BD540040F6D250C0F601004FF44E61F8F71AFDD8
:10BD6400019890F82800000700281AD50198806BE4
:10BD740020B10198806BB0F5004F00D107E040F688
:10BD8400D250C0F6010040F6E541F8F703FD0198F2
:10BD94000068406820F40040019A1168926B1043D7
:10BDA4004860019890F82800C007D0B10198C06A93
:10BDB40020B10198C06AB0F5003F00D107E040F619
:10BDC400D250C0F6010040F6EC41F8F7E3FC0198CC
:10BDD4000068406820F40030019A1168D26A104368
:10BDE4004860019890F82800800700281AD5019827
:10BDF400006B20B10198006BB0F5803F00D107E0E3
:10BE040040F6D250C0F6010040F6F341F8F7C2FC08
:10BE140001980068406820F48030019A1168126B20
:10BE240010434860019890F82800400700281AD56C
:10BE34000198406B20B10198406BB0F5802F00D180
:10BE440007E040F6D250C0F6010040F6FA41F8F798
:10BE5400A1FC01980068406820F48020019A1168D0
:10BE6400526B10434860019890F82800C0060028DF
:10BE74001AD50198C06B20B10198C06BB0F5805FF2
:10BE840000D107E040F6D250C0F6010040F601515F
:10BE9400F8F780FC01980068806820F48050019ACB
:10BEA4001168D26B10438860019890F828008006CE
:10BEB40000281AD50198006C20B10198006CB0F5E7
:10BEC400005F00D107E040F6D250C0F6010040F612
:10BED4000851F8F75FFC01980068806820F400506E
:10BEE400019A1168126C10438860019890F8280038
:10BEF4004006002840F19E800198006841F200014C
:10BF0400C4F20101884247D00198006844F200411C
:10BF1400C4F2000188423FD00198006844F6000151
:10BF2400C4F20001884237D00198006844F6004109
:10BF3400C4F2000188422FD00198006845F2000144
:10BF4400C4F20001884227D00198006841F2004100
:10BF5400C4F2010188421FD00198006847F600012D
:10BF6400C4F20001884217D00198006847F60041E6
:10BF7400C4F2000188420FD00198006841F6000124
:10BF8400C4F20101884207D00198006841F60041DB
:10BF9400C4F20101884200D107E040F6D250C0F655
:10BFA400010040F60F51F8F7F5FB0198406C20B101
:10BFB4000198406CB0F5801F00D107E040F6D250E4
:10BFC400C0F601004FF45161F8F7E4FB01980068F2
:10BFD400406820F48010019A1168526C1043486044
:10BFE4000198406CB0F5801F24D10198806C70B129
:10BFF4000198806CB0F5001F09D00198806CB0F5F1
:10C00400800F04D00198806CB0F5C00F00D107E018
:10C0140040F6D250C0F6010040F61551F8F7BAFBCD
:10C0240001980068406820F4C000019A1168926C7D
:10C0340010434860019890F82800000600281AD59B
:10C044000198C06C20B10198C06CB0F5002F00D1EC
:10C0540007E040F6D250C0F6010040F61D51F8F753
:10C0640099FB01980068406820F40020019A116847
:0AC07400D26C1043486002B080BD9A
:10C07E0080B586B0DDF820C0049003918DF80B20BA
:10C08E00019304980068C06903990840401AB0FAF9
:10C09E0080F040099DF80B10884253D1089801306A
:10C0AE0000284ED001F057FB0199401A089988429A
:10C0BE0001D8089818B903208DF8170045E00498A8
:10C0CE0000680068400700283BD50398802838D0C8
:10C0DE000398402835D004980068C069C0F3C000AA
:10C0EE00012813D104980168082000900862049872
:10C0FE0004F005F900980499C1F890000499002005
:10C10E0081F8840001208DF817001EE00498006865
:10C11E00C069C0F3C020012813D1049801684FF400
:10C12E0000600862049804F0EAF804992020C1F82F
:10C13E0090000499002081F8840003208DF81700E8
:10C14E0003E09EE700208DF817009DF8170006B05B
:02C15E0080BDA2
:10C1600080B5BAB0119011980068C069109011980C
:10C17000006800680F901198006880680E90109811
:10C1800040F60F0108400D900D98A8B99DF84000A9
:10C190008006002810D59DF83C008006002804D4B5
:10C1A0009DF83B00C006002806D51198406F10B1DD
:10C1B0001198416F884726E30D98002800F0EF8022
:10C1C0000E980121C1F20001084207D10F9840F2F8
:10C1D0002011C0F20041084200F0E1809DF84000CB
:10C1E000C00770B19DF83D00C00750B111980168BB
:10C1F000012008621199D1F8900040F00100C1F8C7
:10C2000090009DF84000800700280ED59DF838006A
:10C21000C00750B111980168022008621199D1F845
:10C22000900040F00400C1F890009DF840004007E5
:10C2300000280ED59DF83800C00750B1119801684C
:10C24000042008621199D1F8900040F00200C1F872
:10C2500090009DF840000007002815D59DF83C008F
:10C260008006002805D40E980121C1F20001084281
:10C270000AD011980168082008621199D1F890003D
:10C2800040F00800C1F890009DF841000007002828
:10C2900010D59DF83F00400700280BD51198016884
:10C2A0004FF4006008621199D1F8900040F020002E
:10C2B000C1F890001198D0F8900000286ED09DF839
:10C2C0004000800600280FD59DF83C00800600281D
:10C2D00004D49DF83B00C006002805D51198406F96
:10C2E00010B11198416F88471198D0F890000C90C8
:10C2F00011980068806800F04000402804D09DF844
:10C30000300010F0280F42D0119803F0FFFF119871
:10C31000006880684006002835D51198006808300C
:10C320002190219850E8000F2090209820F04000A4
:10C330000B900B9911980068083039913890389912
:10C34000399A41E80020379037980028E5D11198B4
:10C35000D0F8800098B11198D0F880104CF60B00FE
:10C36000C0F6000008651198D0F8800001F0B4FC18
:10C3700020B11198D0F88000016D884702E0119833
:10C3800001F004F902E0119801F000F906E01198BB
:10C3900001F0FCF811990020C1F8900033E21198E7
:10C3A000C06E012840F0DE819DF84000C0060028E4
:10C3B00040F1D8819DF83C00C006002840F1D281B0
:10C3C0001198016810200862119800688068400682
:10C3D000002840F157811198D0F8800000681021A2
:10C3E000C4F20201884200F090801198D0F88000D9
:10C3F00000682821C4F20201884200F0868011986A
:10C40000D0F8800000684021C4F2020188427CD04C
:10C410001198D0F8800000685821C4F202018842C7
:10C4200073D01198D0F8800000687021C4F2020126
:10C4300088426AD01198D0F8800000688821C4F240
:10C440000201884261D01198D0F880000068A021D4
:10C45000C4F20201884258D01198D0F880000068D8
:10C46000B821C4F2020188424FD01198D0F8800060
:10C47000006840F21041C4F20201884245D0119890
:10C48000D0F88000006840F22841C4F202018842DE
:10C490003BD01198D0F88000006840F24041C4F2CF
:10C4A0000201884231D01198D0F88000006840F233
:10C4B0005841C4F20201884227D01198D0F8800078
:10C4C000006840F27041C4F2020188421DD0119808
:10C4D000D0F88000006840F28841C4F2020188422E
:10C4E00013D01198D0F88000006840F2A041C4F247
:10C4F0000201884209D01198D0F88000006840F20B
:10C50000B841C4F20201884206D11198D0F88000E7
:10C5100000684068019005E01198D0F8800000683C
:10C52000406801900198ADF82A00BDF82A00002863
:10C5300000F09180BDF82A001199B1F85C10884292
:10C5400080F28980BDF82A001199A1F85E00119847
:10C55000D0F88000C069B0F5807F6FD01198006876
:10C560001F901F9850E8000F1E901E9820F48070B6
:10C570000990099911980068369135903599369A45
:10C5800041E80020349034980028E7D111980068E1
:10C5900008301D901D9850E8000F1C901C9820F04A
:10C5A0000100089008991198006808303391329082
:10C5B0003299339A41E80020319031980028E5D132
:10C5C0001198006808301B901B9850E8000F1A90D3
:10C5D0001A9820F0400007900799119800680830D9
:10C5E00030912F902F99309A41E800202E902E986C
:10C5F0000028E5D111992020C1F88C001199002064
:10C60000C866119800681990199850E8000F1890A2
:10C61000189820F0100006900699119800682D9146
:10C620002C902C992D9A41E800202B902B980028D3
:10C63000E7D11198D0F88000F9F7FFFB119902209B
:10C6400008671198B0F85C10B0F85E20891A89B2BA
:10C6500000F096FF15E0BDF82A001199B1F85C10C2
:10C6600088420ED11198D0F88000C069B0F5807F63
:10C6700007D11199022008671198B0F85C1000F0FA
:10C680007FFFC0E01199B1F85C00B1F85E10401A6C
:10C69000ADF816001198B0F85E00002861D0BDF822
:10C6A000160000285DD0119800681790179850E880
:10C6B000000F1690169820F4907004900499119829
:10C6C00000682A91299029992A9A41E80020289007
:10C6D00028980028E7D1119800680830159015981F
:10C6E00050E8000F149014984FF6FE71CEF6FF71CB
:10C6F000084003900399119800680830279126900C
:10C700002699279A41E80020259025980028E2D113
:10C7100011992020C1F88C0011990020C866119948
:10C720004867119800681390139850E8000F129012
:10C73000129820F01000029002991198006824913C
:10C7400023902399249A41E80020229022980028DF
:10C75000E7D11199022008671198BDF8161000F072
:10C760000FFF50E09DF84200C00600280DD59DF84F
:10C770003A004006002808D5119801684FF480104F
:10C780000862119800F002FF3DE09DF840000006AD
:10C79000002810D59DF83C000006002804D49DF820
:10C7A0003A000006002806D51198806F10B1119844
:10C7B000816F884727E09DF840004006002808D593
:10C7C0009DF83C004006002803D5119800F02CF895
:10C7D00019E09DF842000006002808D59DF83F00AA
:10C7E0004006002803D5119800F0D0FE0BE09DF81C
:10C7F0004300C00738B19DF83F000006002802D56D
:0AC80000119800F0C3FE3AB080BDAD
:10C80A0080B582B001900198806B00900099002059
:0EC81A00A1F85E00009800F0B4FE02B080BDF0
:10C8280080B588B00290029800680490049850E897
:10C83800000F0390039820F040000190019902989E
:10C848000068079106900699079A41E8002005902C
:10C8580005980028E7D102992020C1F8880002999C
:0EC8680000208867029800F08DFE08B080BDA9
:10C8760082B001900198406E38B901990120A1F863
:10C886006A000199A1F8680031E010208DF80300D4
:10C896008DF80200019800688068C0F342608DF848
:10C8A6000100019800688068400F8DF800009DF82F
:10C8B60002009DF8002040F63A63C0F60103995C39
:10C8C600484340F64261C0F601018A5CB0FBF2F0D3
:10C8D600019AA2F86A009DF803009DF801209B5C6E
:10C8E6005843895CB0FBF1F00199A1F8680002B0E9
:02C8F600704789
:10C8F80080B584B002900298006841F20001C4F249
:10C90800010188424FD00298006844F20041C4F205
:10C918000001884247D00298006844F60001C4F23A
:10C92800000188423FD00298006844F60041C4F2F2
:10C938000001884237D00298006845F20001C4F22D
:10C94800000188422FD00298006841F20041C4F2E9
:10C958000101884227D00298006847F60001C4F216
:10C96800000188421FD00298006847F60041C4F2CF
:10C978000001884217D00298006841F60001C4F20D
:10C98800010188420FD00298006841F60041C4F2C4
:10C998000101884207D00298006840F60041C5F6B8
:10C9A8000001884200D107E040F6C310C0F601003C
:10C9B80040F23621F7F7ECFE029890F8840001283F
:10C9C80003D102208DF80F0027E00299012081F899
:10C9D800840002992420C1F8880002980068006841
:10C9E800019002980168086820F001000860019829
:10C9F80020F00050019002990020486601980299A1
:10CA08000968086002992020C1F88800029900206E
:10CA180081F8840000208DF80F009DF80F0004B005
:02CA280080BDCF
:10CA2A0080B584B0029001910298006841F2000139
:10CA3A00C4F2010188424FD00298006844F20041D2
:10CA4A00C4F20001884247D00298006844F6000107
:10CA5A00C4F2000188423FD00298006844F60041BF
:10CA6A00C4F20001884237D00298006845F20001FA
:10CA7A00C4F2000188422FD00298006841F20041B6
:10CA8A00C4F20101884227D00298006847F60001E3
:10CA9A00C4F2000188421FD00298006847F600419C
:10CAAA00C4F20001884217D00298006841F60001DA
:10CABA00C4F2010188420FD00298006841F6004191
:10CACA00C4F20101884207D00298006840F600418A
:10CADA00C5F60001884200D107E040F6C310C0F64F
:10CAEA0001004FF41971F7F752FE019898B10198B5
:10CAFA00B0F1005F0FD00198B0F1804F0BD00198D0
:10CB0A00B0F1C04F07D00198B0F1004F03D001989F
:10CB1A00B0F1204F00D107E040F6C310C0F6010083
:10CB2A0040F26521F7F733FE029890F88400012855
:10CB3A0003D102208DF80F002DE00299012081F81F
:10CB4A00840002992420C1F88800029800680068CD
:10CB5A00009002980168086820F0010008600298B5
:10CB6A000068806820F060400199084302990968CA
:10CB7A0088600298FFF77AFE0098029909680860AF
:10CB8A0002992020C1F888000299002081F88400C7
:0ECB9A0000208DF80F009DF80F0004B080BD44
:10CBA80080B584B0029001910298006841F20001BA
:10CBB800C4F2010188424FD00298006844F2004153
:10CBC800C4F20001884247D00298006844F6000188
:10CBD800C4F2000188423FD00298006844F6004140
:10CBE800C4F20001884237D00298006845F200017B
:10CBF800C4F2000188422FD00298006841F2004137
:10CC0800C4F20101884227D00298006847F6000163
:10CC1800C4F2000188421FD00298006847F600411C
:10CC2800C4F20001884217D00298006841F600015A
:10CC3800C4F2010188420FD00298006841F6004111
:10CC4800C4F20101884207D00298006840F600410A
:10CC5800C5F60001884200D107E040F6C310C0F6CF
:10CC6800010040F29521F7F793FD019898B10198DA
:10CC7800B0F1007F0FD00198B0F1806F0BD0019810
:10CC8800B0F1C06F07D00198B0F1006F03D00198E0
:10CC9800B0F1206F00D107E040F6C310C0F60100E4
:10CCA80040F29621F7F774FD029890F88400012865
:10CCB80003D102208DF80F002DE00299012081F8A0
:10CCC800840002992420C1F888000298006800684E
:10CCD800009002980168086820F001000860029836
:10CCE8000068806820F0606001990843029909682B
:10CCF80088600298FFF7BBFD0098029909680860F0
:10CD080002992020C1F888000299002081F8840047
:0ECD180000208DF80F009DF80F0004B080BDC4
:0ECD260081B000900098D0F8800001B07047F6
:10CD340082B001900091009800680199C1F88000C8
:06CD4400002002B0704760
:10CD4A0080B584B003900291002001900298406857
:10CD5A003F2800D807E040F64A60C0F6010040F2DA
:10CD6A006511F7F714FD0298806848B10298806847
:10CD7A00B0F5807F04D002988068B0F5407F00D17A
:10CD8A0007E040F64A60C0F601004FF4B371F7F7C6
:10CD9A00FEFC0298C06848B10298C068B0F5806F7E
:10CDAA0004D00298C068B0F5006F00D107E040F6E1
:10CDBA004A60C0F6010040F26711F7F7E8FC0298F2
:10CDCA00006920B102980069B0F5805F00D107E0E0
:10CDDA0040F64A60C0F601004FF4B471F7F7D7FC89
:10CDEA000298006803998860029948688B68CA6843
:10CDFA0009691843104301430198084301900398B5
:10CE0A00C0684EF2C001CFF6FE710840019908438E
:0ACE1A000399C860002004B080BD39
:0ECE240081B0009000980069C0B201B0704764
:10CE320080B584B003900291029840B10298042810
:10CE420005D00298082802D002980C2800D107E0E9
:10CE520040F64A60C0F601004FF4CA71F7F79BFC36
:10CE6200039802990844143001900198006804B0B4
:02CE720080BD81
:10CE740080B588B006908DF817100492049840F697
:10CE8400FC01C2F200410968C90844F6D352C1F258
:10CE94006202A1FB02218909484301900198411EC5
:10CEA400019118B94FF000400790E5E00698406BF7
:10CEB4000290029901204522C0F220021142009002
:10CEC40004D09DF80900C0F3401000900098C007FA
:10CED4000028E3D10698406B4007002804D5069942
:10CEE400042088630790C7E00698406BC00720B110
:10CEF4000699012088630790BEE00699C520C0F218
:10CF0400200088630698FFF78BFF9DF8171088426E
:10CF140002D001200790AFE006980021FFF787FFB9
:10CF2400039003984EF20801CFF6FF51084202D154
:10CF340000200790A0E09DF80F000006002803D50C
:10CF44004FF00070079097E09DF80F00400600280E
:10CF540002D5402007908FE09DF80F00800600283E
:10CF640002D58020079087E09DF80F00C0060028B6
:10CF740003D54FF4807007907EE09DF80F00000702
:10CF8400002803D54FF40070079075E09DF80F005A
:10CF94004007002803D54FF4806007906CE09DF8AB
:10CFA4000F00C00718B14FF40060079064E09DF8CB
:10CFB4000E000006002803D54FF4805007905BE074
:10CFC4009DF80E004006002803D54FF4005007904A
:10CFD40052E09DF80E008006002803D54FF48040EF
:10CFE400079049E09DF80E00C006002803D54FF4D1
:10CFF4000040079040E09DF80E004007002803D54C
:10D004004FF40030079037E09DF80E0080070028A9
:10D0140003D54FF4802007902EE09DF80E00C00742
:10D0240018B14FF40020079026E09DF80D0000068B
:10D03400002803D54FF4801007901DE09DF80D00E3
:10D044004006002803D54FF40010079014E09DF823
:10D054000D008006002803D54FF4800007900BE0F4
:10D064009DF80C000007002803D54FF4000007903A
:0ED0740002E04FF480300790079808B080BDAE
:10D08200F8B51D4617460C460646184603F0CFFA79
:10D09200002803D407FB04F2A24201D20020F8BD0B
:0ED0A2002846314600F065F8B0FBF4F0F8BD0A
:10D0B00051EC100B21F0004181F0E04181F07F61E3
:0AD0C0000843B0FA80F04009704701
:10D0CA0051EC100B4A0042EAD07010F5001F804163
:10D0DA0040420022C7F6F072114018BF01210840F1
:02D0EA0070478D
:10D0EC0051EC102BC1F30A53002B1CBF40F2FF7CF8
:10D0FC00634500D170471844604506DB0020C7F635
:10D10C00F07060F31E01002208E00028C7BF6FF327
:10D11C001E5141EA005101F00041002241EC102B5C
:02D12C0070474A
:10D12E00CB0648BF704789054CBF3021202103F044
:02D13E0026BA0F
:0AD14000436A08460121FFF79CBF77
:10D14A0083B000B582B0844603A80EC040F6EC0056
:10D15A00C2F2004003AA00680192614603F01FFA76
:0AD16A0002B05DF804EB03B070475B
:06D17400006800F096B80F
:10D17A0040F20000C2F2004003210161416140F621
:10D18A00CF42C0F60102826140F2C441C2F20041BC
:10D19A00C1614FF480610162002181624162C16212
:10D1AA00026640F6C402C2F2004242661022826659
:10D1BA000167C1664167BFF35F8F40F6BE42C0F6A2
:10D1CA00010281F00F03D35C435401311029F8D1D5
:06D1DA00BFF35F8F7047F8
:10D1E0000146C0680A6982426FEA000010449CBF91
:06D1F00089680844704745
:10D1F6002DE9F843144688460546C7684FF00009EE
:10D206002869F943B8420844A96898BF0844CE1B68
:10D21600B04238BF06466868A642384428BF26464C
:10D2260041463246F6F719FAA868F1190F1A18BFDF
:10D236000F46BFF35F8FEF60A41BB044B144DFD14C
:06D246004846BDE8F88334
:10D24C0070B50D4600EB400040F20001C2F2004107
:10D25C0001EBC00000F11806C06A022817D0144672
:10D26C00012807D020B93046FFF7B4FFA04207D2FF
:10D27C0000240AE03046FFF7ADFFA04238BF044659
:10D28C0030462946224603F0EBF9204670BD304665
:0AD29C002946BDE87040FFF7A8BF67
:10D2A600F8B51446064640F20000C2F200400D46AC
:10D2B6000078002808BFFFF75DFFEFF311874FF0F6
:10D2C600200181F31188304629462246FFF7BBFF2D
:06D2D60087F31188F8BD8A
:0ED2DC007F298EBF6FF00100017001207047A6
:0ED2EA00A0F141011A2938BF40F02000704722
:10D2F80080B59EB00BA84C21F6F7DCF90020019010
:10D308000A90099008900790069005900490039061
:10D31800022001F0BBFF0020029044F61800C5F679
:10D3280002000168022262F38F310160006800F494
:10D3380040400290029844F61800C5F602000068C2
:10D3480000F40050B0F5005F00D0F4E7F9F777FC7F
:10D3580044F27041C5F60201086820F01800086020
:10D3680005210B914FF480300C9001200D90022084
:10D37800149015901691282117911890042119914D
:10D388001A9008201B9000201C901D900BA8F9F7FC
:10D398005FFC08B100F014F83F20039003200490CC
:10D3A8000020059006900790089009900A9003A81D
:10D3B8000121FAF71CFA08B100F002F81EB080BD8E
:04D3C80072B6FEE754
:10D3CC0080B5BAB0399000203890379036903590AF
:10D3DC00349006A8B821F6F76BF93998006843F237
:10D3EC000041C4F2010188426AD1002007904FF439
:10D3FC00005006904FF4A0201E9006A8F4F7D0F829
:10D40C0008B1FFF7DBFF44F2F040C5F602000168FB
:10D41C0041F400510160006800F40050059005983B
:10D42C0044F2E040C5F60200016841F010010160D1
:10D43C00006800F01000049004984FF4B040349051
:10D44C0002203590002002903690379005203890BD
:10D45C0041F20000C5F6020034A9F9F725F902994A
:10D46C0040F23030C2F2004003901022C4F20202AB
:10D47C0002605422426040228260C1604FF480629C
:10D48C0002614FF4006242614FF400528261C1614B
:10D49C0001624162F7F746FD08B1FFF78FFF39983B
:10D4AC0040F23031C2F200418167399888635420D0
:10D4BC00019000221146F7F7D8FC019800F0AAF968
:04D4CC003AB080BD35
:10D4D00081B044F2F440C5F60200016841F0020157
:10D4E0000160006800F002000090009801B07047F1
:10D4F00080B540F23030C2F2004000F0E5FE80BD61
:10D5000080B540F2B820C2F2004000F0DDFE80BDE0
:10D5100080B540F24020C2F2004000F0D5FE80BD50
:10D5200080B540F24040C2F20040FCF78EFB80BD67
:10D5300080B540F2A800C2F20040FEF711FE80BDA7
:10D5400080B540F2A830C2F20040FCF77EFB80BDFF
:10D5500080B540F2C410C2F20040FBF7A4F980BDD0
:10D5600080B540F2F430C2F20040FCF76EFB80BDA3
:10D5700080B540F23C10C2F2004001F0C7FF80BD10
:0CD5800082B00190ADF8021002B07047BC
:08D58C0081B0009001B070476E
:10D5940080B592B000210091119110910F910E91DC
:10D5A4000D910C910B910A910991089107910691A3
:10D5B400059104910391029140F2A830C2F2004017
:10D5C400019040F20042C4F2010202601F22426054
:10D5D40081604FF6FF72C260016141618021816107
:10D5E400FBF775FE08B1FFF7EDFE4FF480500E9087
:10D5F40040F2A830C2F200400EA9FDF796F908B136
:10D60400FFF7E0FE40F2A830C2F20040FCF7CAF98E
:10D6140008B1FFF7D7FE0420099050200A900A2091
:10D624000B9000200D9040F2A830C2F2004009A9EE
:10D63400FDF719FE08B1FFF7C5FE0020069007901C
:10D64400089040F2A830C2F2004006A902F010FC93
:10D6540008B1FFF7B7FE0A200290012003900022D0
:10D664000492059240F2A830C2F2004002A9FCF7ED
:0CD6740069FE08B1FFF7A6FE12B080BDF1
:10D6800080B58EB00D9000200C900B900A90099000
:10D6900008900D98006840F20041C4F200018842F1
:10D6A00016D144F2E840C5F60200016841F00201DB
:10D6B0000160006800F00200079007981D200490A8
:10D6C00000221146F7F7D7FB049800F0A9F847E0CD
:10D6D0000D98006840F20041C4F2010188423FD138
:10D6E00044F2F040C5F60200016841F00201016019
:10D6F000006800F002000690069844F2E040C5F68B
:10D700000200016841F004010160006800F00400BB
:10D7100005900598402008900220099001200A9069
:10D72000002003900B9003200C9040F60000C5F6FB
:10D73000020008A9F8F7BEFF039A2E2001901146B7
:10D74000F7F799FB019800F06BF80198039A0F2105
:10D750000291F7F790FB0299039A2C20F7F78BFBC5
:04D760000EB080BDCA
:0CD7640040F2B040C2F200400068704784
:10D7700083B00290029800F0070000904EF60C5122
:10D78000CEF200010868019001984FF6FF021040A8
:10D7900001900198009A40EA02200022C0F2FA5259
:0CD7A000104301900198086003B070472E
:10D7AC004EF60C50CEF200000068C0F30220704719
:10D7BC0088B0079006910592079800F00700049036
:10D7CC000498C0F10700052802D30420019003E05F
:10D7DC000498C0F10700019001980390049804305C
:10D7EC00062802D80020009002E00498033800902C
:10D7FC000098029006980399012202FA01F101396E
:10D80C000840029B984005999A40013A1140084300
:04D81C0008B0704799
:10D8200080B582B0ADF80600BDF90600002800D42E
:10D8300006E040F6A220C0F60100BD21F6F7ACFFDD
:0CD84000BDF9060000F002F802B080BD47
:10D84C0081B0ADF80200BDF9020000280CD4BDF97E
:10D85C00021001F01F02012090404A094EF2001103
:0CD86C00CEF2000141F8220001B070472C
:10D8780081B00090009840F001004EF69451CEF22D
:10D88800000108604EF62451CEF20001086840F409
:10D8980080300860BFF34F8FBFF36F8F01B07047C0
:10D8A80010B582B0019001984078D8B301984078BB
:10D8B800012837D001984078022833D00198407861
:10D8C80003282FD00198407804282BD0019840785D
:10D8D800052827D001984078062823D00198407859
:10D8E80007281FD00198407808281BD00198407855
:10D8F800092817D0019840780A2813D00198407851
:10D908000B280FD0019840780C280BD0019840784C
:10D918000D2807D0019840780E2803D00198407848
:10D928000F2800D107E040F6A220C0F6010040F21F
:10D938004D11F6F72DFF01980078012802D00198C3
:10D94800007800B907E040F6A220C0F601004FF4C5
:10D95800A771F6F71DFF0198007B18B10198007BAD
:10D96800012800D107E040F6A220C0F6010040F2ED
:10D978004F11F6F70DFF0198C07A98B10198C07A57
:10D9880001280FD00198C07A02280BD00198C07ADC
:10D99800032807D00198C07A052803D00198C07AD7
:10D9A800062800D107E040F6A220C0F601004FF497
:10D9B800A871F6F7EDFE0198807A38B10198807A5F
:10D9C800012803D00198807A022800D107E040F6A8
:10D9D800A220C0F6010040F25111F6F7D9FE0198D5
:10D9E800407B012802D00198407B00B907E040F64F
:10D9F800A220C0F601004FF4A971F6F7C9FE0198FC
:10DA0800807B012802D00198807B00B907E040F6AE
:10DA1800A220C0F6010040F25311F6F7B9FE0198B2
:10DA2800C07B012802D00198C07B00B907E040F60E
:10DA3800A220C0F601004FF4AA71F6F7A9FE0198DA
:10DA4800407AFE2800DC07E040F6A220C0F601007C
:10DA580040F25511F6F79CFE0198007A04286BD025
:10DA68000198007A052867D00198007A062863D0C3
:10DA78000198007A07285FD00198007A08285BD0BF
:10DA88000198007A092857D00198007A0A2853D0BB
:10DA98000198007A0B284FD00198007A0C284BD0B7
:10DAA8000198007A0D2847D00198007A0E2843D0B3
:10DAB8000198007A0F283FD00198007A10283BD0AF
:10DAC8000198007A112837D00198007A122833D0AB
:10DAD8000198007A13282FD00198007A14282BD0A7
:10DAE8000198007A152827D00198007A162823D0A3
:10DAF8000198007A17281FD00198007A18281BD09F
:10DB08000198007A192817D00198007A1A2813D09A
:10DB18000198007A1B280FD00198007A1C280BD096
:10DB28000198007A1D2807D00198007A1E2803D092
:10DB38000198007A1F2800D107E040F6A220C0F61D
:10DB480001004FF4AB71F6F723FE019840784EF6CA
:10DB58009851CEF2000108604EF6A051CEF20001B5
:10DB6800086820F001000860019840684EF69C5251
:10DB7800CEF200021060DDF804E09EF80C00000709
:10DB88009EF80B2040EA02609EF800209EF80830BC
:10DB98009EF809C09EF80A4040EAC4409EF80D402D
:10DBA80040EA84409EF80E4040EA44409EF80FE068
:10DBB80040EA0E4040EA0C2040EA43001043086067
:04DBC80002B010BDDA
:10DBCC0083B00290029800790190019800287BD0D4
:10DBDC000198082878D802980168012045F208427B
:10DBEC00C5F602029142009046D0029801680120CD
:10DBFC0045F21C42C5F60202914200903CD00298BC
:10DC0C000168012045F23042C5F6020291420090B3
:10DC1C0032D002980168012045F24442C5F6020256
:10DC2C009142009028D002980168012045F2584298
:10DC3C00C5F60202914200901ED0029801680120A4
:10DC4C0045F26C42C5F602029142009014D0029843
:10DC5C000168012045F28042C5F602029142009013
:10DC6C000AD0029800684AF66C31CAF2FD71084479
:10DC7C00B0FA80F0400900900098C00778B1019983
:10DC8C0045F6FC00C5F6020000EB81000299C8665F
:10DC9C00029945F64010C5F6020008670EE001999E
:10DCAC0040F6FC00C4F2020000EB81000299C86649
:10DCBC00029940F64010C4F2020008670198411E18
:0CDCCC00012088400299486703B07047AF
:10DCD80080B586B00490049818B901208DF8170013
:10DCE800EAE2049890F83500022806D004998020CA
:10DCF800486501208DF81700DEE2049801680120CC
:10DD08001022C4F202029142029000F0918004981D
:10DD1800016801202822C4F202029142029000F018
:10DD280087800498016801204022C4F202029142CF
:10DD380002907DD00498016801205822C4F20202A2
:10DD48009142029074D00498016801207022C4F2B4
:10DD58000202914202906BD0049801680120882247
:10DD6800C4F202029142029062D004980168012034
:10DD7800A022C4F202029142029059D0049801688C
:10DD88000120B822C4F202029142029050D00498B5
:10DD98000168012040F21042C4F20202914202904E
:10DDA80046D004980168012040F22842C4F20202D9
:10DDB800914202903CD004980168012040F2404210
:10DDC800C4F202029142029032D004980168012004
:10DDD80040F25842C4F202029142029028D00498BC
:10DDE8000168012040F27042C4F20202914202909E
:10DDF8001ED004980168012040F28842C4F2020251
:10DE08009142029014D004980168012040F2A04287
:10DE1800C4F20202914202900AD0049800684FF6B8
:10DE28004831CBF6FD710844B0FA80F04009029001
:10DE38000298C007002800F08A800499042081F81D
:10DE48003500049800681021C4F20201884270D09D
:10DE5800049800682821C4F20201884269D0049815
:10DE680000684021C4F20201884262D00498006828
:10DE78005821C4F2020188425BD0049800687021DE
:10DE8800C4F20201884254D0049800688821C4F280
:10DE9800020188424DD004980068A021C4F2020112
:10DEA800884246D004980068B821C4F2020188422A
:10DEB8003FD00498006840F21041C4F20201884241
:10DEC80037D00498006840F22841C4F20201884221
:10DED8002FD00498006840F24041C4F20201884201
:10DEE80027D00498006840F25841C4F202018842E1
:10DEF8001FD00498006840F27041C4F202018842C1
:10DF080017D00498006840F28841C4F202018842A0
:10DF18000FD00498006840F2A041C4F20201884280
:10DF280007D00498006840F2B841C4F20201884260
:10DF380006D104980168086820F00100086005E02F
:10DF480004980168086820F001000860B1E10498AD
:10DF58000168086820F00E00086004980068102125
:10DF6800C4F20201884270D0049800682821C4F2E3
:10DF78000201884269D0049800684021C4F2020175
:10DF8800884262D0049800685821C4F2020188428D
:10DF98005BD0049800687021C4F20201884254D012
:10DFA800049800688821C4F2020188424DD0049880
:10DFB8000068A021C4F20201884246D00498006893
:10DFC800B821C4F2020188423FD00498006840F2A8
:10DFD8001041C4F20201884237D00498006840F228
:10DFE8002841C4F2020188422FD00498006840F208
:10DFF8004041C4F20201884227D00498006840F2E8
:10E008005841C4F2020188421FD00498006840F2C7
:10E018007041C4F20201884217D00498006840F2A7
:10E028008841C4F2020188420FD00498006840F287
:10E03800A041C4F20201884207D00498006840F267
:10E04800B841C4F20201884206D104980168086800
:10E0580020F00100086005E004980168086820F0D5
:10E06800010008600498016801201022C4F202022D
:10E078009142019000F0EA8004980168012028226A
:10E08800C4F202029142019000F0E0800498016815
:10E0980001204022C4F202029142019000F0D68091
:10E0A8000498016801205822C4F2020291420190AA
:10E0B80000F0CC800498016801207022C4F20202AA
:10E0C8009142019000F0C2800498016801208822E2
:10E0D800C4F202029142019000F0B88004980168ED
:10E0E8000120A022C4F202029142019000F0AE8009
:10E0F800049801680120B822C4F2020291420190FA
:10E1080000F0A48004980168012040F21042C4F293
:10E1180002029142019000F0998004980168012060
:10E1280040F22842C4F202029142019000F08E802F
:10E1380004980168012040F24042C4F20202914270
:10E14800019000F0838004980168012040F2584251
:10E15800C4F202029142019078D00498016801202B
:10E1680040F27042C4F20202914201906ED00498CB
:10E178000168012040F28842C4F2020291420190F3
:10E1880064D004980168012040F2A042C4F202025F
:10E19800914201905AD004980168012040F2B84297
:10E1A800C4F202029142019050D004980168012003
:10E1B80045F20842C5F602029142019046D0049801
:10E1C8000168012045F21C42C5F602029142019005
:10E1D8003CD004980168012045F23042C5F602029D
:10E1E8009142019032D004980168012045F24442DE
:10E1F800C5F602029142019028D0049801680120D6
:10E2080045F25842C5F60202914201901ED0049888
:10E218000168012045F26C42C5F602029142019064
:10E2280014D004980168012045F28042C5F6020224
:10E23800914201900AD0049800684AF66C31CAF2FB
:10E24800FD710844B0FA80F0400901900198C007B8
:10E2580008B30498016E086820F480700860049878
:10E26800806D03900498C06D00F01F010120884064
:10E27800039948600498416E806E48600498C06EA7
:10E2880048B10498C16E086820F48070086004984A
:10E29800016F406F48600499012081F835000499A6
:10E2A800002081F834000498006D10B10498016DC5
:10E2B800884700208DF817009DF8170006B080BD2C
:10E2C80080B590B00F9000200B9040F6FC00C2F291
:10E2D8000040006848F2B511C1F64E31A0FB0110AC
:10E2E800800A0A900F98806D09900F98806D0890A9
:10E2F800099800680E90089800680D900F980168BA
:10E3080001201022C4F202029142079000F091808D
:10E318000F98016801202822C4F202029142079056
:10E3280000F087800F98016801204022C4F20202A1
:10E33800914207907DD00F98016801205822C4F2BD
:10E3480002029142079074D00F9801680120702250
:10E35800C4F20202914207906BD00F980168012025
:10E368008822C4F202029142079062D00F98016895
:10E378000120A022C4F202029142079059D00F98BE
:10E3880001680120B822C4F202029142079050D0DD
:10E398000F980168012040F21042C4F20202914233
:10E3A800079046D00F980168012040F22842C4F235
:10E3B8000202914207903CD00F980168012040F278
:10E3C8004042C4F202029142079032D00F9801688D
:10E3D800012040F25842C4F202029142079028D02C
:10E3E8000F980168012040F27042C4F20202914283
:10E3F80007901ED00F980168012040F28842C4F2AD
:10E4080002029142079014D00F980168012040F24F
:10E41800A042C4F20202914207900AD00F98006805
:10E428004FF64831CBF6FD710844B0FA80F0400948
:10E4380007900798C007002800F05F840E980F998E
:10E44800C96D01F01F01C8400007002840F19A80FB
:10E458000F9800681021C4F20201884270D00F980A
:10E4680000682821C4F20201884269D00F98006828
:10E478004021C4F20201884262D00F9800685821F6
:10E48800C4F2020188425BD00F9800687021C4F280
:10E498000201884254D00F9800688821C4F2020112
:10E4A80088424DD00F980068A021C4F2020188422A
:10E4B80046D00F980068B821C4F2020188423FD0C4
:10E4C8000F98006840F21041C4F20201884237D028
:10E4D8000F98006840F22841C4F2020188422FD008
:10E4E8000F98006840F24041C4F20201884227D0E8
:10E4F8000F98006840F25841C4F2020188421FD0C8
:10E508000F98006840F27041C4F20201884217D0A7
:10E518000F98006840F28841C4F2020188420FD087
:10E528000F98006840F2A041C4F20201884207D067
:10E538000F98006840F2B841C4F20201884206D13F
:10E548000F980068006800F00400069005E00F9836
:10E558000068006800F008000690069890B10F98CF
:10E568000168086820F0040008600F98C06D00F08A
:10E578001F0108208840099988600F99486D40F06C
:10E58800010048650E980F99C96D01F01F01C84038
:10E59800C007002800F093800F9800681021C4F28B
:10E5A8000201884270D00F9800682821C4F2020145
:10E5B800884269D00F9800684021C4F2020188425D
:10E5C80062D00F9800685821C4F2020188425BD0DB
:10E5D8000F9800687021C4F20201884254D00F9845
:10E5E80000688821C4F2020188424DD00F98006863
:10E5F800A021C4F20201884246D00F980068B821D1
:10E60800C4F2020188423FD00F98006840F21041DE
:10E61800C4F20201884237D00F98006840F22841BE
:10E62800C4F2020188422FD00F98006840F240419E
:10E63800C4F20201884227D00F98006840F258417E
:10E64800C4F2020188421FD00F98006840F270415E
:10E65800C4F20201884217D00F98006840F288413E
:10E66800C4F2020188420FD00F98006840F2A0411E
:10E67800C4F20201884207D00F98006840F2B841FE
:10E68800C4F20201884206D10F980068406900F080
:10E698008000059004E00F9800680068002005904D
:10E6A800059860B10F98C06D00F01F0101208840E7
:10E6B800099988600F99486D40F0020048650E98E6
:10E6C8000F99C96D01F01F01C8404007002840F1AB
:10E6D80093800F9800681021C4F20201884270D01C
:10E6E8000F9800682821C4F20201884269D00F9867
:10E6F80000684021C4F20201884262D00F98006885
:10E708005821C4F2020188425BD00F98006870213A
:10E71800C4F20201884254D00F9800688821C4F2DC
:10E72800020188424DD00F980068A021C4F202016E
:10E73800884246D00F980068B821C4F20201884286
:10E748003FD00F98006840F21041C4F2020188429D
:10E7580037D00F98006840F22841C4F2020188427D
:10E768002FD00F98006840F24041C4F2020188425D
:10E7780027D00F98006840F25841C4F2020188423D
:10E788001FD00F98006840F27041C4F2020188421D
:10E7980017D00F98006840F28841C4F202018842FD
:10E7A8000FD00F98006840F2A041C4F202018842DD
:10E7B80007D00F98006840F2B841C4F202018842BD
:10E7C80006D10F980068006800F00200049004E089
:10E7D8000F980068006800200490049860B10F98B2
:10E7E800C06D00F01F0104208840099988600F99C6
:10E7F800486D40F0040048650E980F99C96D01F006
:10E808001F01C840C006002840F1BB800F9800686F
:10E818001021C4F20201884270D00F9800682821A4
:10E82800C4F20201884269D00F9800684021C4F2FE
:10E838000201884262D00F9800685821C4F2020190
:10E8480088425BD00F9800687021C4F202018842A8
:10E8580054D00F9800688821C4F2020188424DD034
:10E868000F980068A021C4F20201884246D00F9890
:10E878000068B821C4F2020188423FD00F980068AE
:10E8880040F21041C4F20201884237D00F98006864
:10E8980040F22841C4F2020188422FD00F98006844
:10E8A80040F24041C4F20201884227D00F98006824
:10E8B80040F25841C4F2020188421FD00F98006804
:10E8C80040F27041C4F20201884217D00F980068E4
:10E8D80040F28841C4F2020188420FD00F980068C4
:10E8E80040F2A041C4F20201884207D00F980068A4
:10E8F80040F2B841C4F20201884206D10F9800687C
:10E90800006800F00800039005E00F9800680068B0
:10E9180000F004000390039898B30F98C06D00F0BE
:10E928001F0110208840099988600F9800680068C6
:10E938004003002813D50F980068006800030028DA
:10E9480006D40F98006C10B10F98016C884705E049
:10E958000F98806C10B10F98816C884711E00F9860
:10E9680000680068C005002805D40F980168086889
:10E9780020F0080008600F98006C10B10F98016C27
:10E9880088470E980F99C96D01F01F01C84080068D
:10E99800002840F1F8800F9800681021C4F20201A5
:10E9A800884270D00F9800682821C4F2020188427A
:10E9B80069D00F9800684021C4F20201884262D0F1
:10E9C8000F9800685821C4F2020188425BD00F9862
:10E9D80000687021C4F20201884254D00F98006880
:10E9E8008821C4F2020188424DD00F980068A02106
:10E9F800C4F20201884246D00F980068B821C4F2D8
:10EA0800020188423FD00F98006840F21041C4F2DA
:10EA18000201884237D00F98006840F22841C4F2BA
:10EA2800020188422FD00F98006840F24041C4F29A
:10EA38000201884227D00F98006840F25841C4F27A
:10EA4800020188421FD00F98006840F27041C4F25A
:10EA58000201884217D00F98006840F28841C4F23A
:10EA6800020188420FD00F98006840F2A041C4F21A
:10EA78000201884207D00F98006840F2B841C4F2FA
:10EA88000201884206D10F980068006800F0100063
:10EA9800029005E00F980068006800F002000290FC
:10EAA800029800286FD00F98C06D00F01F01202039
:10EAB8008840099988600F9890F8350004282ED16D
:10EAC8000F980168086820F0160008600F98016820
:10EAD800486920F0800048610F98006C10B90F98C1
:10EAE800806C28B10F980168086820F00800086059
:10EAF8000F98C06D00F01F013F2088400999886079
:10EB08000F99012081F835000F99002081F8340011
:10EB18000F98006D10B10F98016D884780E30F982A
:10EB2800006800684003002813D50F980068006843
:10EB38000003002806D40F98406C10B10F98416C60
:10EB4800884705E00F98C06B10B10F98C16B8847D4
:10EB580019E00F9800680068C00500280DD40F98C8
:10EB68000168086820F0100008600F99012081F8FA
:10EB780035000F99002081F834000F98C06B10B150
:10EB88000F98C16B88470F98406D002800F0B4803B
:10EB98000F98406DC007002800F0A8800F99042046
:10EBA80081F835000F9800681021C4F202018842EC
:10EBB80070D00F9800682821C4F20201884269D0F9
:10EBC8000F9800684021C4F20201884262D00F9871
:10EBD80000685821C4F2020188425BD00F9800688F
:10EBE8007021C4F20201884254D00F98006888212D
:10EBF800C4F2020188424DD00F980068A021C4F2E7
:10EC08000201884246D00F980068B821C4F2020178
:10EC180088423FD00F98006840F21041C4F20201C8
:10EC2800884237D00F98006840F22841C4F20201A8
:10EC380088422FD00F98006840F24041C4F2020188
:10EC4800884227D00F98006840F25841C4F2020168
:10EC580088421FD00F98006840F27041C4F2020148
:10EC6800884217D00F98006840F28841C4F2020128
:10EC780088420FD00F98006840F2A041C4F2020108
:10EC8800884207D00F98006840F2B841C4F20201E8
:10EC9800884206D10F980168086820F001000860D2
:10ECA80005E00F980168086820F0010008600B98DB
:10ECB80001300B900A99884200D905E00F98006846
:10ECC8000068C0070028F2D10F9800680068C007E4
:10ECD80020B10F99032081F8350003E00F99012036
:10ECE80081F835000F99002081F834000F98C06C26
:10ECF80010B10F98C16C884792E20F980168012003
:10ED080045F20842C5F602029142019046D00F989A
:10ED18000168012045F21C42C5F6020291420190A9
:10ED28003CD00F980168012045F23042C5F6020236
:10ED38009142019032D00F980168012045F2444277
:10ED4800C5F602029142019028D00F98016801206F
:10ED580045F25842C5F60202914201901ED00F9822
:10ED68000168012045F26C42C5F602029142019009
:10ED780014D00F980168012045F28042C5F60202BE
:10ED8800914201900AD00F9800684AF66C31CAF295
:10ED9800FD710844B0FA80F0400901900198C0075D
:10EDA800002800F03D820F98006800680C900D98CC
:10EDB8000F99C96D01F01F01C8404007002840F1B4
:10EDC800B7809DF830004007002840F1B1800F98C7
:10EDD800C06D00F01F0104208840089948609DF824
:10EDE80031000006002811D59DF83200C00730B95F
:10EDF8000F98806C10B10F98816C884705E00F98C8
:10EE0800006C10B10F98016C884790E09DF83000B5
:10EE18008006002800F185800F9800681021C4F250
:10EE28000201884270D00F9800682821C4F20201BC
:10EE3800884269D00F9800684021C4F202018842D4
:10EE480062D00F9800685821C4F2020188425BD052
:10EE58000F9800687021C4F20201884254D00F98BC
:10EE680000688821C4F2020188424DD00F980068DA
:10EE7800A021C4F20201884246D00F980068B82148
:10EE8800C4F2020188423FD00F98006840F2104156
:10EE9800C4F20201884237D00F98006840F2284136
:10EEA800C4F2020188422FD00F98006840F2404116
:10EEB800C4F20201884227D00F98006840F25841F6
:10EEC800C4F2020188421FD00F98006840F27041D6
:10EED800C4F20201884217D00F98006840F28841B6
:10EEE800C4F2020188420FD00F98006840F2A04196
:10EEF800C4F20201884207D00F98006840F2B84176
:10EF0800C4F20201884206D10F980168086820F00F
:10EF18000800086005E00F980168086820F0040000
:10EF280008600F98006C10B10F98016C884776E163
:10EF38000D980F99C96D01F01F01C840800700287E
:10EF480040F1BF809DF830008007002840F1B9806B
:10EF58000F98C06D00F01F01022088400899486092
:10EF68009DF831000006002811D59DF83200C00731
:10EF780030B90F98406C10B10F98416C884705E084
:10EF88000F98C06B10B10F98C16B884798E09DF837
:10EF980030008006002800F18D800F98006810214D
:10EFA800C4F20201884270D00F9800682821C4F288
:10EFB8000201884269D00F9800684021C4F202011A
:10EFC800884262D00F9800685821C4F20201884232
:10EFD8005BD00F9800687021C4F20201884254D0B7
:10EFE8000F9800688821C4F2020188424DD00F981A
:10EFF8000068A021C4F20201884246D00F98006838
:10F00800B821C4F2020188423FD00F98006840F24C
:10F018001041C4F20201884237D00F98006840F2CC
:10F028002841C4F2020188422FD00F98006840F2AC
:10F038004041C4F20201884227D00F98006840F28C
:10F048005841C4F2020188421FD00F98006840F26C
:10F058007041C4F20201884217D00F98006840F24C
:10F068008841C4F2020188420FD00F98006840F22C
:10F07800A041C4F20201884207D00F98006840F20C
:10F08800B841C4F20201884206D10F9801680868A5
:10F0980020F01400086005E00F980168086820F067
:10F0A8000A0008600F99012081F835000F990020A7
:10F0B80081F834000F98C06B10B10F98C16B884766
:10F0C800ADE00D980F99C96D01F01F01C840000708
:10F0D800002840F1A4809DF830000007002840F186
:10F0E8009E800F9800681021C4F20201884270D0F7
:10F0F8000F9800682821C4F20201884269D00F984D
:10F1080000684021C4F20201884262D00F9800686A
:10F118005821C4F2020188425BD00F980068702120
:10F12800C4F20201884254D00F9800688821C4F2C2
:10F13800020188424DD00F980068A021C4F2020154
:10F14800884246D00F980068B821C4F2020188426C
:10F158003FD00F98006840F21041C4F20201884283
:10F1680037D00F98006840F22841C4F20201884263
:10F178002FD00F98006840F24041C4F20201884243
:10F1880027D00F98006840F25841C4F20201884223
:10F198001FD00F98006840F27041C4F20201884203
:10F1A80017D00F98006840F28841C4F202018842E3
:10F1B8000FD00F98006840F2A041C4F202018842C3
:10F1C80007D00F98006840F2B841C4F202018842A3
:10F1D80006D10F980168086820F01C00086005E057
:10F1E8000F980168086820F00E0008600F98C06D3D
:10F1F80000F01F01012000FA01F1089A51600F99EF
:10F2080048650F9981F835000F99002081F834007E
:10F218000F98C06C10B10F98C16C8847FFE7FFE7E3
:04F2280010B080BDE5
:10F22C0080B582B00190ADF802108DF80120BDF8C8
:10F23C00020010B1002000B907E040F65A50C0F6A9
:10F24C0001004FF4D571F5F7A1FA9DF8010018B142
:10F25C009DF80100012800D107E040F65A50C0F695
:10F26C00010040F2AB11F5F791FA9DF8010020B1C5
:10F27C00BDF802000199886104E0BDF802000004A9
:08F28C000199886102B080BD08
:10F2940080B584B002900298022802D00298012816
:10F2A40000D107E040F60C30C0F601004FF4A17124
:10F2B400F5F770FA44F60C00C5F602000068C0F3D6
:10F2C400800088B944F60C00C5F60200006800F01E
:10F2D40007000299884203D001208DF80F0027E02F
:10F2E40000208DF80F0023E044F60C01C5F602015E
:10F2F400086820F00700029A10430860FEF730FA0D
:10F30400019044F60400C5F602000068C0F34030E2
:10F3140058B9FEF725FA0199401AB0F57A7F03D956
:10F3240001208DF80F0003E0EBE700208DF80F00BB
:08F334009DF80F0004B080BD3C
:10F33C0082B00190009101993F20086044F2104086
:10F34C00C5F60200006800F007000199486044F21D
:10F35C001840C5F60200016801F47061019A9160D1
:10F36C00016801F00F01019AD160006800F0700093
:10F37C000199086144F21C40C5F60200016801F0D5
:10F38C007001019A5161006800F4E0600199886194
:10F39C0044F22040C5F60200006800F070000199AC
:10F3AC00C86142F20000C5F20020006800F00F00B6
:08F3BC000099086002B07047DF
:10F3C40080B584B00290029801684FF65F70C0F275
:10F3D4000300C860FEF7C4F9019002980068C06891
:10F3E400800600280BD4FEF7BBF90199401AB0F54A
:10F3F4007A7F03D903208DF80F0003E0EDE70020A6
:0CF404008DF80F009DF80F0004B080BDD3
:10F4100080B584B003900398406A00900398806A96
:10F4200020282FD3002002900298072823D8039881
:10F430000068FDF778FC0190019800990870009829
:10F44000013000900198000A00990870009801307E
:10F450000090BDF8060000990870009801300090F7
:10F460009DF80700009908700098013000900298FC
:10F4700001300290D8E70098039948620399886A9E
:08F480002038886204B080BD51
:10F4880080B584B003900398C06900900398006A1F
:10F49800202835D3002002900298072829D8009800
:10F4A8000078019000980130009000980178019848
:10F4B80040EA0120019000980130009000980178FE
:10F4C800019840EA014001900098013000900098AE
:10F4D8000178019840EA016001900098013000909D
:10F4E8000398006801A9FDF721FC029801300290F9
:10F4F800D2E700980399C8610399086A203808621E
:04F5080004B080BD0E
:10F50C0080B588B007900798006800690690079846
:10F51C000068406905900698059908400490079882
:10F52C0000688068039000200290079890F8810092
:10F53C008DF8070007980068303000909DF8150092
:10F54C00000700280ED59DF818000007002809D5E3
:10F55C0007980168886940F4006088610798FEF795
:10F56C000FF85DE19DF810004006002811D49DF8BD
:10F57C001000800600280CD49DF8100040070028CD
:10F58C0007D50798416F88470798016F8847012076
:10F59C0002909DF81000400600280DD49DF8100034
:10F5AC00C00748B19DF810004007002804D4079804
:10F5BC00016F8847012002909DF8100080060028FA
:10F5CC000ED49DF810008007002809D59DF8100076
:10F5DC004007002804D40798416F88470120029007
:10F5EC00029800B11CE19DF810000007002878D5A6
:10F5FC0007980168886940F00800886107980168DD
:10F60C00886940F01000886107980168886940F4A7
:10F61C000060886107980168086920F0080008619B
:10F62C0007980068806810F4404F32D10798B0F802
:10F63C006A0070B30798C06810280AD3079800684E
:10F64C00006B0799496E08600799486E043048664C
:10F65C0018E00798C068082809D300980088079913
:10F66C00496E08800799486E023048660AE0079890
:10F67C00006890F830000799496E08700799486E39
:10F68C00013048660799B1F86A000138A1F86A00A0
:10F69C00CCE70798F9F798FD0799012081F88100CC
:10F6AC000798D0F8840018B10798FDF769FFB7E008
:10F6BC009DF80700052803D10798FDF761FF0FE0BF
:10F6CC009DF80700042803D10798FDF759FF07E0C0
:10F6DC009DF80700032803D10798FDF751FFFFE7BA
:10F6EC009EE0BDF8100010F4587F00F099809DF852
:10F6FC001000400600280CD50799D1F8840040F082
:10F70C000400C1F8840007980168886940F0400043
:10F71C0088619DF81100800700280CD50799D1F855
:10F72C00840040F00100C1F88400079801688869E2
:10F73C0040F4007088619DF81100C00760B1079912
:10F74C00D1F8840040F00800C1F8840007980168E3
:10F75C00886940F4807088619DF81000800600284C
:10F76C000CD50799D1F8840040F08000C1F88400D2
:10F77C0007980168886940F0200088610798D0F8E4
:10F78C00840000284CD007980168086820F001001C
:10F79C00086007980168086940F26B329043086171
:10F7AC00039800F44040B0F5404F32D107980168FF
:10F7BC00886820F4404088600798C06F90B1079823
:10F7CC00C16F4FF63100C0F6000008650798C06F96
:10F7DC00FEF77CFA30B10799D1F8840040F0400074
:10F7EC00C1F884000798806F90B10798816F4FF62D
:10F7FC003100C0F6000008650798806FFEF766FAC6
:10F80C0030B10799D1F8840040F04000C1F8840071
:10F81C0006E00799012081F881000798FDF7B0FEFA
:04F82C0008B080BDE3
:10F8300080B582B001900198806B00900099002003
:10F84000A1F86A000099A1F862000099012081F8EE
:0CF8500081000098FDF79AFE02B080BD18
:10F85C0080B584B00290029800680021C4F20101C6
:10F86C00884274D002980068B0F1804F6FD0029833
:10F87C00006840F20041C4F20001884267D002984F
:10F88C00006840F60001C4F2000188425FD0029883
:10F89C00006840F60041C4F20001884257D002983B
:10F8AC00006841F20001C4F2000188424FD0029876
:10F8BC00006841F20041C4F20001884247D002982E
:10F8CC00006840F20041C4F2010188423FD0029826
:10F8DC00006841F60001C4F20001884237D002985A
:10F8EC00006841F60041C4F2000188422FD0029812
:10F8FC00006842F20001C4F20001884227D002984D
:10F90C00006844F20001C4F2010188421FD0029841
:10F91C00006844F20041C4F20101884217D00298F9
:10F92C00006844F60001C4F2010188420FD002982D
:10F93C0000684EF20001C4F20001884207D0029820
:10F94C0000684EF20041C4F20001884200D107E089
:10F95C0040F65C10C0F6010040F2D311F4F716FF2C
:10F96C00029890F83D00012803D001208DF80F007B
:10F97C0074E00299022081F83D0002980168C86881
:10F98C0040F00100C860029800680021C4F2010137
:10F99C00884244D002980068B0F1804F3FD0029862
:10F9AC00006840F20041C4F20001884237D002984E
:10F9BC00006840F60001C4F2000188422FD0029882
:10F9CC00006840F60041C4F20001884227D002983A
:10F9DC00006840F20041C4F2010188421FD0029835
:10F9EC00006841F60001C4F20001884217D0029869
:10F9FC00006844F20001C4F2010188420FD0029861
:10FA0C0000684EF20001C4F20001884207D002984F
:10FA1C0000684EF20041C4F20001884215D10298F0
:10FA2C00006880680721C0F201010840019001982C
:10FA3C00062809D00198B0F5803F05D002980168DE
:10FA4C00086840F00100086005E002980168086849
:10FA5C0040F00100086000208DF80F009DF80F00A9
:04FA6C0004B080BDA5
:10FA700080B586B0059004910598006A02900599BA
:10FA8000086A20F010000862059840680190059807
:10FA900080690390039848F6FF71CFF6FF61084034
:10FAA0000390039820F44070039004980168039831
:10FAB00040EA01200390029820F020000290049870
:10FAC0008168029840EA0110029005980021C4F272
:10FAD0000101884221D0059840F20041C4F20101A1
:10FAE00088421AD0059844F20001C4F2010188420C
:10FAF00001D1002088B9059844F20041C4F2010107
:10FB0000884201D1002040B9059844F60001C4F2B2
:10FB1000010188421FD10120E8B90498C06818B1DA
:10FB20000498C068082800D107E040F65C10C0F6D1
:10FB3000010041F6B731F4F72FFE029820F0800063
:10FB400002900498C168029840EA0110029002985D
:10FB500020F04000029005980021C4F20101884283
:10FB60001BD0059840F20041C4F20101884214D034
:10FB7000059844F20001C4F2010188420DD00598B5
:10FB800044F20041C4F20101884206D0059844F6CF
:10FB90000001C4F20101884235D104988069B0F5B2
:10FBA000007F02D00498806900B907E040F65C103D
:10FBB000C0F6010041F6C431F4F7EEFD0498406947
:10FBC000B0F5807F02D00498406900B907E040F6A4
:10FBD0005C10C0F6010041F6C531F4F7DDFD019877
:10FBE00020F480600190019820F400600190049856
:10FBF0004169019840EA8100019004988169019867
:10FC000040EA8100019001980599486003980599A0
:10FC1000886104984068059988630298059908628C
:04FC200006B080BDED
:10FC240085B0049003910498006A01900499086ACD
:10FC340020F4803008620498406800900498406D75
:10FC4400029002984FF68F71CFF6FE710840029031
:10FC540003980168029808430290019820F4003048
:10FC6400019003988168019840EA0140019004984A
:10FC74000021C4F2010188421BD0049840F20041E3
:10FC8400C4F20101884214D0049844F20001C4F281
:10FC9400010188420DD0049844F20041C4F20101EC
:10FCA400884206D0049844F60001C4F20101884257
:10FCB40009D1009820F4803000900398416900989D
:10FCC40040EA012000900098049948600298049941
:10FCD4004865039840680499886501980499086206
:04FCE40005B07047B0
:10FCE80086B005900491039202930598006A0090EB
:10FCF8000599086A20F0100008620598806901904B
:10FD0800019820F4407001900399019840EA01207D
:10FD18000190019820F4704001900298000381B28C
:10FD2800019808430190009820F0A00000900498E2
:10FD380000F00A01009840EA011000900198059926
:0CFD4800886100980599086206B07047B9
:10FD540086B005900491039202930598006A00907E
:10FD64000599086A20F4805008620598C0690190DA
:10FD7400019820F4407001900399019840EA012011
:10FD84000190019820F4704001900298000381B220
:10FD9400019808430190009820F4204000900498B2
:10FDA40000F00A01009840EA01300090019805999A
:0CFDB400C86100980599086206B070470D
:10FDC00085B004900391029201930498806800909A
:10FDD000009820F47F40009003980299019A41EA2C
:10FDE000022101430098084300900098049988601C
:04FDF00005B07047A3
:10FDF40085B00490039102920498006A00900499DB
:10FE0400086A20F001000862049880690190019852
:10FE140020F0F00001900299019840EA011001904D
:10FE2400009820F00A00009003990098084300907D
:10FE340001980499886100980499086205B0704794
:10FE440083B00290019102988068009000984FF668
:10FE54008F71CFF6CF710840009001980099084344
:10FE640040F00700009000980299886003B0704742
:10FE740080B586B004900391049800680021C4F210
:10FE84000101884254D004980068B0F1804F4FD0EB
:10FE94000498006840F20041C4F20001884247D04F
:10FEA4000498006840F60001C4F2000188423FD083
:10FEB4000498006840F60041C4F20001884237D03B
:10FEC4000498006841F20001C4F2000188422FD076
:10FED4000498006841F20041C4F20001884227D02E
:10FEE4000498006840F20041C4F2010188421FD026
:10FEF4000498006841F60001C4F20001884217D05A
:10FF04000498006844F20001C4F2010188420FD051
:10FF1400049800684EF20001C4F20001884207D040
:10FF2400049800684EF20041C4F20001884200D1F6
:10FF340007E040F6E030C0F6010040F2CB71F4F780
:10FF440029FC03980068D8B103980068102817D0DA
:10FF540003980068202813D00398006830280FD035
:10FF64000398006840280BD003980068502807D0F5
:10FF740003980068602803D003980068702800D1B3
:10FF840007E040F6E030C0F6010040F2CC71F4F72F
:10FF940001FC03988068802802D00398806800B927
:10FFA40007E040F6E030C0F6010040F2CD71F4F70E
:10FFB400F1FB049890F83C00012803D102208DF84D
:10FFC4001700F5E00499012081F83C00049902200F
:10FFD40081F83D0004980068406802900498006825
:10FFE40080680190049800680021C4F201018842ED
:0CFFF40007D00498006840F20041C4F2FD
:020000040801F1
:100000000101884265D10398406800284FD00398C9
:100010004068B0F5801F4AD003984068B0F5001FD3
:1000200045D003984068B0F5401F40D00398406821
:10003000B0F5800F3BD003984068B0F5A00F36D0E4
:1000400003984068B0F5C00F31D003984068B0F510
:10005000C00F2CD003984068B0F5E00F27D003986C
:100060004068B0F5000F22D003984068B0F5100F3B
:100070001DD003984068B0F5200F18D00398406851
:10008000B0F5300F13D003984068B0F5400F0ED094
:1000900003984068B0F5500F09D003984068B0F558
:1000A000600F04D003984068B0F5700F00D107E0EE
:1000B00040F6E030C0F6010040F2DF71F4F76CFB6F
:1000C000029820F470000290039841680298084357
:1000D0000290029820F07000029003980168029844
:1000E00008430290029804990968486004980068DF
:1000F0000021C4F20101884244D004980068B0F1A4
:10010000804F3FD00498006840F20041C4F20001E3
:10011000884237D00498006840F60001C4F200011C
:1001200088422FD00498006840F60041C4F20001D4
:10013000884227D00498006840F20041C4F20101CF
:1001400088421FD00498006841F60001C4F2000103
:10015000884217D00498006844F20001C4F20101FB
:1001600088420FD0049800684EF20001C4F20001EA
:10017000884207D0049800684EF20041C4F20001A2
:1001800088420CD1019820F080000190039881688A
:1001900001980843019001980499096888600499BE
:1001A000012081F83D000499002081F83C000020E6
:0C01B0008DF817009DF8170006B080BD08
:1001BC0080B596B0059005990020C1F89000FDF728
:1001CC00CBFA0490059800680068000700282FD52A
:1001DC000598049B6A466FF07E4111604FF4001144
:1001EC000022FBF746FF18B3059800680C900C989A
:1001FC0050E8000F0B900B9820F0800003900399AF
:10020C0005980068159114901499159A41E80020EE
:10021C00139013980028E7D105992020C1F8880085
:10022C000599002081F8840003208DF81B0063E001
:10023C00059800680068400700284AD50598049B7B
:10024C006A466FF07E4111604FF480010022FBF78B
:10025C0010FF00283DD0059800680A900A9850E8D5
:10026C00000F0990099820F490700290029905985B
:10027C000068129111901199129A41E80020109087
:10028C0010980028E7D10598006808300890089865
:10029C0050E8000F0790079820F001000190019999
:1002AC000598006808300F910E900E990F9A41E84E
:1002BC0000200D900D980028E5D105992020C1F85B
:1002CC008C000599002081F8840003208DF81B0018
:1002DC0012E005992020C1F888000599C1F88C001E
:1002EC0005990020C866059908670599002081F8D2
:1002FC00840000208DF81B009DF81B0016B080BDFB
:10030C0093B00390039800680990099850E8000F87
:10031C000890089820F49070029002990398006855
:10032C00129111901199129A41E800201090109896
:10033C000028E7D10398006808300790079850E828
:10034C00000F069006984FF6FE71CEF6FF7108402E
:10035C00019001990398006808300F910E900E9946
:10036C000F9A41E800200D900D980028E2D10398D7
:10037C00C06E012817D1039800680590059850E8C5
:10038C00000F0490049820F010000090009903983E
:10039C0000680C910B900B990C9A41E800200A9084
:1003AC000A980028E7D103992020C1F88C00039902
:0C03BC000020C8660399486713B0704722
:1003C80080B588B00790002002900C21009103911D
:1003D8004FF48071049105904FF48050069007996E
:1003E800C86840F08000C8600799C86820F04000DD
:1003F800C860079802A9FCF7A4FC009907984EF278
:100408000012C0F2F552FCF731FD01900799C86857
:1004180020F08000C8600198B0F1007F01D1002071
:080428000190019808B080BDAD
:10043000010002000400060008000A000C00100081
:080440002000400080000001D3
:10044800F4F78BFA4EF68850CEF20000016851F4AA
:0804580070010160F3F710F8D8
:100460000020B4EE400BF1EE10FA68BF0120704797
:0804700051EC100BC80F70479E
:0404780000F000B8D8
:10047C0052EC10CBC2F30A5340F2FF718B4211BF06
:10048C00002B002101607047A3F2FE31016040F2A5
:0C049C00FE3060F31E5242EC10CB7047A3
:0804A800002848BF40427047E4
:1004B000B7EE000B0028B0EE401B11D0014648BF3C
:1004C0004142B7EE001B40F2E842C0F60002CB0703
:1004D0001CBF92ED002B21EE021B08324908F6D119
:0C04E00080EE010B002821FE000B70478D
:1004EC0010B582B0044600698DF8071078B1D4E9D4
:1004FC0000239A4231D26269531C63618154D4E95E
:10050C000501884229D1204600F02CF825E0E0684E
:10051C0050B1D4E9002C62451FD2531CB3EB0C0331
:10052C0018BF0B46835418E0A06858B1D4E9002CCE
:10053C00624512D2531CB3EB0C0318BFCBB240F87C
:10054C0022300AE0236A43B1D4E90001884204D284
:10055C000DF10701204601229847206801302060E8
:04056C0002B010BD0C
:100570004269002A08BF704710B50446036A002B81
:0C0580001CBF216998470020606110BD7D
:10058C00012AB8BF704770B514460D460646304672
:0C059C002946FFF7A5FF013CF9D870BD0F
:1005A80070B514460D46064600F0BAF801463046C6
:0C05B8002A462346BDE8704000F000B861
:1005C4002DE9F04F03AF8DB047F83C3C91460C4603
:1005D400064600F047F80546EB46073020F00700D2
:1005E400ADEB0008C546A7F1380A50460021242285
:1005F400F3F766F84DF24110C0F6000047E90740F2
:100604006FF0004047F8340C47F8146C47F8205C4E
:1006140047F8288C5046494657F83C2CEFF7D6FF4C
:0C062400DD46A7F10C04A546BDE8F08FF0
:1006300040F6EC01C2F2004140F6F0020968091AE6
:10064000C2F2004218BF01211268121A18BF01221B
:10065000114040F6F402C2F200421268101A18BFAC
:080660000120084040427047F0
:040668004020704777
:10066C002DE9F0411546884604464068D4E9021647
:10067C0030448F1BBA42414605D2F2F7EBFF3544AA
:10068C00BFF35F8F0BE03A46F2F7E4FF08EB07018C
:10069C00ED1B60682A46F2F7DDFFBFF35F8FE56064
:0406AC00BDE8F08134
:1006B0000178002904BF0020704700214FF001326B
:1006C0004358C2FA53F30431002BF9D093FAA3F044
:0C06D000B0FA80F001EBD0000438704755
:1006DC0000291CBF0278002A01D10020704700B508
:1006EC00D0F800E00429034609D34FF0013CCCFAC2
:1006FC005EF222B9043953F804EF0329F7D8181A1B
:10070C004FF00132C2FA5EF292FAA2F2B2FA82F21F
:0C071C00B1EBD20F88BFD108084400BD2B
:1007280040F2C040C2F200400068002804BF40F612
:08073800D400C2F2004070473A
:1007400084460020002918BF002A00D1704709788C
:1007500048B2002844BF6FF001007047BCF1000FA1
:1007600018BFCCF800100021C3E90011002818BF01
:0407700001207047AD
:100774007F2884BF0020704740F63952C0F601023A
:10078400515C40F6DA62C0F60102105C0840704722
:0C079400A0F161011A2938BF203870471D
:1007A0007F2884BF0020704740F63952C0F601020E
:1007B000515C40F6DA62C0F60102105C08407047F6
:1007C000443A5C50726F6A656B74655C6563735F15
:1007D000636861726765725C6374726C5C6669728F
:1007E0006D776172655C4D61696E5C437562654DE4
:1007F000585C447269766572735C53544D33324869
:100800003778785F48414C5F4472697665725C5313
:1008100072635C73746D3332683778785F68616CCB
:070820005F646D612E6300AF
:10082700443A5C50726F6A656B74655C6563735FAD
:10083700636861726765725C6374726C5C66697227
:100847006D776172655C4D61696E5C437562654D7C
:10085700585C447269766572735C53544D33324801
:100867003778785F48414C5F4472697665725C53AC
:1008770072635C73746D3332683778785F68616C64
:070887005F7263632E630042
:10088E00443A5C50726F6A656B74655C6563735F46
:10089E00636861726765725C6374726C5C666972C0
:1008AE006D776172655C4D61696E5C437562654D15
:1008BE00585C447269766572735C53544D3332489A
:1008CE003778785F48414C5F4472697665725C5345
:1008DE0072635C73746D3332683778785F68616CFD
:0708EE005F7274632E6300CA
:1008F500443A5C50726F6A656B74655C6563735FDF
:10090500636861726765725C6374726C5C66697258
:100915006D776172655C4D61696E5C437562654DAD
:10092500585C447269766572735C53544D33324832
:100935003778785F48414C5F4472697665725C53DD
:1009450072635C73746D3332683778785F68616C95
:070955005F7370692E63005F
:10095C00443A5C50726F6A656B74655C6563735F77
:10096C00636861726765725C6374726C5C666972F1
:10097C006D776172655C4D61696E5C437562654D46
:10098C00585C447269766572735C53544D333248CB
:10099C003778785F48414C5F4472697665725C5376
:1009AC0072635C73746D3332683778785F68616C2E
:0709BC005F74696D2E6300FA
:1009C300443A5C50726F6A656B74655C6563735F10
:1009D300636861726765725C6374726C5C6669728A
:1009E3006D776172655C4D61696E5C437562654DDF
:1009F300585C447269766572735C53544D33324864
:100A03003778785F48414C5F4472697665725C530E
:100A130072635C73746D3332683778785F68616CC6
:0B0A23005F756172745F65782E6300E0
:070A2E00286E756C6C2900B5
:100A35004A616E7561727900466562727561727997
:100A4500004D6172636800417072696C004D617997
:100A5500004A756E65004A756C7900417567757356
:100A6500740053657074656D626572004F63746FD1
:100A7500626572004E6F76656D62657200446563EE
:070A8500656D62657200005F
:070A8C00414D00504D000038
:0F0A930025612025622025652025542025590046
:100AA200443A5C50726F6A656B74655C6563735F30
:100AB200636861726765725C6374726C5C666972AA
:100AC2006D776172655C4D61696E5C437562654DFF
:100AD200585C447269766572735C53544D33324884
:100AE2003778785F48414C5F4472697665725C532F
:100AF20072635C73746D3332683778785F68616CE7
:0A0B02005F636F727465782E630064
:100B0C00443A5C50726F6A656B74655C6563735FC5
:100B1C00636861726765725C6374726C5C6669723F
:100B2C006D776172655C4D61696E5C437562654D94
:100B3C00585C447269766572735C53544D33324819
:100B4C003778785F48414C5F4472697665725C53C4
:100B5C0072635C73746D3332683778785F68616C7C
:0A0B6C005F7077725F65782E6300FA
:100B7600443A5C50726F6A656B74655C6563735F5B
:100B8600636861726765725C6374726C5C666972D5
:100B96006D776172655C4D61696E5C437562654D2A
:100BA600585C447269766572735C53544D333248AF
:100BB6003778785F48414C5F4472697665725C535A
:100BC60072635C73746D3332683778785F68616C12
:0A0BD6005F7263635F65782E6300B1
:100BE000443A5C50726F6A656B74655C6563735FF1
:100BF000636861726765725C6374726C5C6669726B
:100C00006D776172655C4D61696E5C437562654DBF
:100C1000585C447269766572735C53544D33324844
:100C20003778785F48414C5F4472697665725C53EF
:100C300072635C73746D3332683778785F68616CA7
:0A0C40005F74696D5F65782E630034
:100C4A0053756E646179004D6F6E646179005475F5
:100C5A006573646179005765646E657364617900D0
:100C6A0054687572736461790046726964617900C7
:0A0C7A005361747572646179000023
:020C840043002B
:020C86002E003E
:100C880050726F6772616D207374617274202825C9
:090C9800732C202573292E0A009B
:090CA10031363A31333A323700A2
:050CAA002D494E46003B
:050CAF002D696E6600D6
:050CB4002B494E460033
:050CB9002B696E6600CE
:100CBE00000000000000545452205245474745534F
:010CCE000025
:090CCF005465726D696E616C00E0
:090CD800256D2F25642F257900FC
:090CE10025483A254D3A2553003F
:100CEA0053756E004D6F6E0054756500576564004C
:0D0CFA005468750046726900536174000073
:100D07004A616E00466562004D6172004170720073
:100D17004D6179004A756E004A756C004175670030
:100D2700536570004F6374004E6F7600446563002F
:010D370000BB
:010D380000BA
:0D0D39000007032004170201085710408036
:0C0D46004A616E20323820323032350015
:080D5200000610160006101641
:100D5A00443A5C50726F6A656B74655C6563735F75
:100D6A00636861726765725C6374726C5C666972EF
:100D7A006D776172655C4D61696E5C437562654D44
:100D8A00585C447269766572735C53544D333248C9
:100D9A003778785F48414C5F4472697665725C5374
:100DAA0072635C73746D3332683778785F68616C2C
:080DBA005F6770696F2E630092
:100DC20000000000000000000102030406070809F9
:100DD200443A5C50726F6A656B74655C6563735FFD
:100DE200636861726765725C6374726C5C66697277
:100DF2006D776172655C4D61696E5C437562654DCC
:100E0200585C447269766572735C53544D33324850
:100E12003778785F48414C5F4472697665725C53FB
:100E220072635C73746D3332683778785F68616CB3
:080E32005F756172742E63000C
:080E3A000101010307010000A2
:080E420008040204080101018B
:100E4A00443A5C50726F6A656B74655C6563735F84
:100E5A00636861726765725C6374726C5C666972FE
:100E6A006D776172655C4D61696E5C437562654D53
:100E7A00585C447269766572735C53544D333248D8
:100E8A003778785F48414C5F4472697665725C5383
:100E9A0072635C73746D3332683778785F6C6C5F39
:080EAA0073646D6D632E63009B
:100EB200303132333435363738394142434445468E
:100EC20030313233343536373839616263646566BE
:040ED2004E414E003F
:040ED6006E616E00DB
:100EDA0020202020202020202068282828282020A0
:100EEA0020202020202020202020202020202020F8
:100EFA0048101010101010101010101010101010B0
:100F0A00848484848484848484841010101010104F
:100F1A0010818181818181010101010101010101A8
:100F2A00010101010101010101010110101010105C
:100F3A001082828282828202020202020202020279
:100F4A000202020202020202020202101010102021
:100F5C00AD0F010800000024D4080000BF0F0108E9
:100F6C00D40800247C0F01082D0000008B340008ED
:100F7C0024370008243700082437000824370008D9
:100F8C002437000810000000B4040024B804002426
:100F9C00BC0400240090D0030090D003010000009A
:100FAC00206861680834002200E042540139FCD505
:020FBC0070477C
:100FBE0020686168A2680C3401E08B5C8354013AAE
:040FCE00FBD5704798
:0400000508010449A1
:00000001FF
